:020000040800F2
:10000000000001205D460008D1270008D327000822
:10001000D5270008D7270008D927000800000000CE
:10002000000000000000000000000000DB270008C6
:10003000DD27000800000000DF270008E127000896
:10004000AD460008AD460008E5270008AD460008AB
:10005000AD460008AD460008F1270008F727000864
:10006000AD460008AD46000829280008AD46000846
:10007000FD270008FF270008012800080D280008B8
:100080001928000825280008AD460008AD460008DC
:1000900000000000AD4600082B280008AD4600080F
:1000A000AD460008AD460008AD460008AD46000864
:1000B000AD460008AD460008AD460008AD46000854
:1000C000AD460008AD460008AD460008AD46000844
:1000D000AD46000835280008AD460008AD460008CA
:1000E000AD4600083128000841280008AD46000848
:1000F000AD4600080000000000000000AD4600080A
:10010000AD460008AD4600084D280008AD46000881
:10011000AD460008AD460008AD460008AD460008F3
:10012000AD460008AD460008AD460008AD460008E3
:08013000AD460008AD460008D1
:1001380010B5054C237833B9044B13B10448AFF319
:1001480000800123237010BDBC08002000000000BF
:10015800D046010808B5034B1BB103490348AFF368
:10016800008008BD00000000C0080020D04601083B
:1001780014214160704714207047406A704700009E
:10018800790100087F01000883010008990100082F
:1001980010B5044604F1100000F05CFCC4F8F80047
:1001A8000148C4F87C0110BD88010008F8B5E6B024
:1001B80004460D4616461F460A4906A800F0CAFE20
:1001C80070996F9A05910492009733466E996D9ACB
:1001D800039102922A466C990191214600F060F839
:1001E80067B0F0BD94010008F8B5E6B004460D46C6
:1001F80016461F46094906A800F0ACFE6F996E9A8C
:100208000491039200976D996C9A0291019233467A
:100218002A46214600F087F867B0F0BD940100082F
:1002280038B500281CBF01680029184A23D1184B8B
:100238001C684FF6F0710C404CF24025AC421FBFD1
:100248001B6819404CF27024A14212D1114D296843
:1002580079B911490B68C3F30B03B3F58A6F1FBF54
:100268000968C1F30B0140F28343994204BF01219D
:10027800117028B905E0094B994204BF012111709A
:100288004068BDE8324001F09FBE00BFD80800209A
:1002980000ED00E0002004E00010005C000037489A
:1002A8002DE9F04104460D46216816464A681F4666
:1002B80090478046B8F5403F2ED122680A99936846
:1002C800204698478046B8F5403F25D12368089ACC
:1002D8000799D3F80CC02046E0478046B8F5403F60
:1002E8001AD12368069A39461F692046B8478046BE
:1002F800B8F5403F10D1236829465D69324620464B
:10030800A8478046B8F5403F06D123680B9A09995B
:100318009D692046A847804621680A68204690477C
:100328004046BDE8F0812DE9F04104460D462168BC
:1003380016464A681F4690478046B8F5403F2ED17A
:1003480022680A999368204698478046B8F5403F46
:1003580025D12368089A0799D3F80CC02046E047AE
:100368008046B8F5403F1AD12368069A39461F6976
:100378002046B8478046B8F5403F10D12368294643
:100388005D6932462046A8478046B8F5403F06D109
:1003980023680999DD6900222046A847804621681C
:1003A8000A68204690474046BDE8F0814FF4403047
:1003B80070470000F0B50C4685B0114600281A4673
:1003C8001CBF0568002D0B4B11D082B104B971B95F
:1003D8000D9860B10F9E0E9F0A9B0290049603979A
:1003E8000B980C9E009001962046A8470346184695
:1003F80005B0F0BD020003002DE9F04F0646D0B06D
:100408000868F56DD6F860E0726EB76EF36E00BAE4
:1004180000906C46486800BA60600DF14008886832
:1004280000BAA060C86800BAE060086900BA206134
:10043800486900BA6061886900BAA061C86900BAF1
:10044800E061086A00BA2062486A00BA6062886A95
:1004580000BAA062C86A00BAE062086B00BA2063FA
:10046800486B00BA6063886B00BAA063C86B00BAB7
:10047800E063402058F80C1C58F820CC58F838ACE9
:100488008CEA010158F840CC8AEA01018CEA01099A
:100498004FEAF979401E48F8049BEBD187EA02003D
:1004A80000EA0E00784010EBF5610098DFF824C4EC
:1004B80041186144C81882EABE032B404FEAF06134
:1004C80053405918636859186144CF194FEAB50366
:1004D80083EABE01014081EABE0111EBF765A1681C
:1004E8004D196544A91883EAB0023A404FEAF1650C
:1004F8005A405519E26855194FEAB70282EAB0071F
:1005080065440F4005EBBE0E97EAB00717EBFE6592
:1005180027697D194FEAB10782EA0701654401EAB4
:100528000E01EB18514011EBF36561694D194FEA63
:10053800BE0187EA010E65440EEA030E15EBB00012
:100548008EEA070E0EEBF065D4F818E075446544A2
:10055800AA1881EAB30505404FEAF26E4D40AE4451
:10056800E569AE44E64477444FEAB00080EAB30E4A
:100578000EEA020E8EEAB30E0EEBF765D4F820E011
:1005880075446544691880EAB2053D404FEAF16E4A
:100598004540AE44656AAE44E6440EEBB3034FEA09
:1005A800B70787EAB20E0EEA010E8EEAB20E0EEB1C
:1005B800F365D4F828E075446544281887EAB1053E
:1005C8001D404FEAF06E7D40AE44E56AAE44E64415
:1005D8000EEBB2024FEAB30383EAB10E0EEA000E45
:1005E8008EEAB10E0EEBF265D4F830E0754465443E
:1005F800EF1983EAB00515404FEAF76E5D40AE4447
:10060800656BAE44E6440EEBB1014FEAB20282EAF2
:10061800B00E0EEA070E8EEAB00E0EEBF165D4F8B6
:1006280038E075446544EB1882EAB7050D404FEA97
:10063800F36E5540AE44E56BAE44E6440EEBB000B5
:100648004FEAB10181EAB70E0EEA030E8EEAB70E41
:100658000EEBF065D4F840E07544654481EAB30ECA
:10066800AA180EEA000E4FEAF2658EEA010E7544EA
:10067800DDF844E04FEAB000754480EAB30E654403
:100688000EEA020E15EBB7078EEAB30E0EEBF7650E
:10069800DDF848E04FEAB202754480EA020E65448C
:1006A8000EEA070E69188EEA000E0EEBF165DDF80A
:1006B8004CE07544654405EBB3034FEAB70E1427C5
:1006C8000DF1500CDFF810528EEA010B82EA0B0B89
:1006D8000BEBF36A5CF804BBDA44AA44504483EA9F
:1006E800B10B4FEAF06A8EEA0B0BDA445CF804BBF4
:1006F800DA44AA44524480EAB30B4FEAF26A8BEA1E
:10070800B10BDA445CF804BBDA444FEAB000AA44FF
:1007180080EA020BD6448BEAB30B0BEBFE6A5CF85B
:1007280004BBDA444FEAB202AA4482EA0E0B0AEB8F
:10073800B10180EA0B0B0BEBF16A5CF804BBDA44FD
:100748007F1DAA44282F0AEBB3034FEABE0EBBD382
:100758003C2F61D3502F4DD204EB870CC7F15407BF
:100768005E4CA7FB04A504465D4FA8088EEA010A63
:1007780082EA0A0A5CF804BB0AEBF3655D447D195A
:100788002C1983EAB10A4FEAF4658EEA0A0A55443D
:100798005CF804AB5CF804BB55447D19AA1884EADC
:1007A800B30A4FEAF2658AEAB10A55445D444FEA52
:1007B800B4047D1984EA020AAE448AEAB30A0AEB51
:1007C800FE655CF804AB55444FEAB2027D1982EA33
:1007D8000E0A15EBB10184EA0A0A5CF804BB0AEBBD
:1007E800F1655D447D1915EBB303401E4FEABE0E5B
:1007F800BCD12046F46D1B19F365336EC9183166F8
:10080800716E71447166B36ED218B266F16E40189B
:10081800F06650B0BDE8F08F4EEA010B0EEA010A0F
:100828000BEA020B4BEA0A0A0AEBF36554F827A015
:10083800DFF8B0C0554443EAB10B654403EAB10A96
:100848000BEA0E0B28184BEA0A0A7F1C0AEBF06524
:1008580054F827A0554440EAB30B654400EAB30AAC
:100868000BEAB10BAA184BEA0A0A7F1C0AEBF265DD
:1008780054F827A055444FEAB00040EA020B6544FB
:1008880000EA020A0BEAB30BAE444BEA0A0A7F1CE1
:100898000AEBFE6554F827A055444FEAB20242EA33
:1008A8000E0B654402EA0E0A0BEA000B15EBB101C8
:1008B8004BEA0A0A7F1C0AEBF16554F827A0554455
:1008C8007F1C65443C2F05EBB3034FEABE0EA3D350
:1008D80040E700BF9979825AA1EBD96ECDCCCCCC38
:1008E800D6C162CADCBC1B8F00B581B00168074A5B
:1008F800914200D110B9064801B000BD7C2113F027
:100908004DFE4FF4003001B000BD00BFFC090008E7
:10091800030002002DE9F0410B4A92E8F85188B033
:10092800694681E8F8510268084B9A4200D118B923
:10093800074808B0BDE8F0811422083000F04FFBEA
:1009480008B0BDE8F08100BFDC090008FC09000818
:1009580003000200152904D20268044B9A4200D110
:1009680008B903487047083000F048BBFC09000884
:100978000300020010B481B013460268074CA2427B
:1009880000D118B901B010BC0548704701B000F19A
:10099800240210BC083000F035BB00BFFC09000879
:1009A8000300020010B481B013460268074CA2424B
:1009B80000D118B901B010BC054870470A4601B00B
:1009C80000F1240110BC083000F070BBFC090008DD
:1009D800030002000123456789ABCDEFFEDCBA981E
:1009E80076543210F0E1D2C300000000000000008D
:1009F80000000000F10800081D0900085D09000852
:100A08007D090008AD09000801040008790F0008F5
:100A1800C50F0008810F0008F0B5A3B004460B48C5
:100A280002900D4616461F46094B0822402104A88D
:100A380000F0D1FA28980190009733462A462146BB
:100A480002A800F01BF823B0F0BD00BFFC090008A5
:100A5800100A000810B5040008BF002408D0054893
:100A6800054B20600822402104F1080000F0B3FA89
:100A7800204610BDFC090008100A00082DE9F041C5
:100A880004460E46216817464A681D469047804628
:100A9800B8F5003F19D1226806999368204698470F
:100AA8008046B8F5003F10D123683146DE683A46E3
:100AB8002046B0478046B8F5003F06D12368079A1C
:100AC80029461D692046A847804621680A682046AD
:100AD80090474046BDE8F08110B500F033FA4FF476
:100AE800403400280EBF034C4FF4C07113F056FD7C
:100AF800204610BD0200030010B5044600F022FA9B
:100B080008B9054810BD0021A160D0F87C21116802
:100B180088474FF4403010BD0200030070B504460A
:100B28000D4600F00FFA064E40B1D0F87C0141683E
:100B38008847A84224BF65604FF44036304670BDF0
:100B4800020003002DE9FF4715000C4600D02CB128
:100B5800064600F0F7F95FEA000801D16448C3E0EF
:100B6800D8F8F80001684A689047B0F5003F17D1F7
:100B7800D8F87C118A68404690478146B9F1810FC0
:100B880080F09E80A94508F1FC0A17D2D8F8F80031
:100B98000368D3F80CC02A462146E047B0F5003F69
:100BA80040F08E80D8F8F8000368D3F810C06A4681
:100BB8005146E047B0F5003F76D10AE0002004E056
:100BC800215C0AF800100098401C00900098A84288
:100BD800F6D34FF0000C4749474A484B01AC009800
:100BE800844558D2D3E9007001ADC5E9007010788A
:100BF80000281ABF042086464FF0000E085854F803
:100C08000E5028443E4D05600127D0F800E087606B
:100C1800019D4F681AF80C007D408EEA050585F0A5
:100C2800040E65680F687D4085F0FC05754485F005
:100C3800A30568400AF80C000CF1010CCFE7D3E9D2
:100C4800004501A8C0E9004510782E4D002814BFC2
:100C58004FF0040E4FF0000E01A8744651F80EE054
:100C68000459A6440127CEF80050DEF80040CEF81B
:100C780008704D68019F40687D406C400D68684071
:100C880084F0040480F0FC00041984F057040AF886
:100C98000C400CF1010CCC45D1D3D8F8F800016810
:100CA8004A689047B0F5003F0AD1D8F8F8000368C1
:100CB800D3F80C804A465146C047B0F5003F01D0F2
:100CC800114811E0002006E05AF8201081F06A313E
:100CD8004AF82010401CB0EB990FF5D3B06840F0EB
:100CE8000100B0604FF4403004B0BDE8F08700BFA9
:100CF8000200030068470108D8080020240F0008F4
:100D0800ADBE4ED70DBE75A10100030038B50C4627
:100D1800017A1546CA0702D500F014F908B908483F
:100D280032BDD0F8F80003682146DC682A46A0479F
:100D3800B0F5003F01D0034832BD4FF4403032BD1A
:100D480002000300010003002DE9F84191B00546B7
:100D58000E461746402101A813F020FC297AC8073F
:100D680004D5284600F0EEF8040002D1DFF8A4808C
:100D78004BE0D4F8F800DFF8A0800368D3F810C07F
:100D88006A4601A9E047B0F5003F3ED1D4F8F80023
:100D980001684A689047B0F5003F36D1D4F87C1115
:100DA8008A6820469047D4F8F830024618461B68EF
:100DB800D3F80CC004F1FC01E047B0F5003F24D1A2
:100DC800D4F87C0141688847D4F8F83002461846C0
:100DD8001B68D3F80CC001A9E047B0F5003F14D157
:100DE800D4F8F8000268696893689847B0F5003F3E
:100DF8000BD1D4F8F80003681C693A463146A0477D
:100E0800B0F5003F08BF4FF44038404612B0BDE887
:100E1800F08100BF02000300010003002DE9F84142
:100E2800A5B0074688461646402115A813F0B6FB1C
:100E380000220492402105A813F0B0FB387AC107BC
:100E48005ED5384600F07EF8050059D0D5F8F80090
:100E58002D4C0368D3F810C06A4605A9E047B0F5E1
:100E6800003F3CD1D5F8F80001684A689047B0F5D2
:100E7800003F34D1D5F87C118A6828469047D5F8C8
:100E8800F830024618461B68D3F80CC005F1FC017F
:100E9800E047B0F5003F22D1D5F87C01416888478A
:100EA800D5F8F830024618461B68D3F80CC005A9D7
:100EB800E047B0F5003F12D1D5F8F800026879682C
:100EC80093689847B0F5003F09D1D5F8F800036852
:100ED8001D6904AA15A9A847B0F5003F01D020460E
:100EE8000FE00A4B0A490B4A0396029101924046C9
:100EF8001C68049B009415AA796800F0E5F900E0E5
:100F0800054826B0BDE8F0810100030070470108DC
:100F1800936E030026C703000200030004B001011A
:100F280000170145E10A0008010B0008250B00081D
:100F3800B50300084D0B0008150D0008510D0008F9
:100F4800250E00080168024A914218BF0020704728
:100F58002C0F000810B5040008BF002404D0034873
:100F68002060204609688847204610BD2C0F0008DD
:100F780020225C3013F010BBF0B58468A30800226F
:100F880004F0030407E000F15C0555F8226035BA67
:100F980041F82250521C9A42F5D300220BE000F18E
:100FA8005C0502EB830755F82360D500C5F11805E9
:100FB800EE40CE55521CA242F1D3F0BD30B5C46804
:100FC80003690022E31AD5188C5C0544521C082AD0
:100FD8002C77F8D330BD0360C1600261704738B523
:100FE800044615460022626023685A68904700202C
:100FF8006061A061A5604FF4003032BD81604FF49C
:10100800003070472DE9F84304462079D4F80C8065
:10101800450748BF244845D466691D46A8F1010024
:1010280000EAD60306EBC506B6EBC50F666102D229
:10103800A669761CA6611746A66906EB5576A661D1
:101048000E46E918884225D2A8EB03094A463146DC
:10105800F81813F0A1FA2268136839460FE04246DF
:10106800384613F099FA23681A683946204690479B
:1010780007E0311811F00300F1D122681368204607
:101088009847484600EB0809A9F10101A942F0D3A5
:10109800002300E000202A1A3118F81813F07CFA0F
:1010A8004FF40030BDE8F283040002002DE9FC4F44
:1010B800024685B0D0681369DFF86CC1DFF86C812F
:1010C800A0EB030A506840F004005060002703A812
:1010D80002900DF10C0ED8E9003403A8544DC0E974
:1010E80000342878534D00280CBF00230423994668
:1010F8005CF803305EF80940234401261D601C6833
:101108009E60DCF80430039DDCF80090DEF8046093
:101118005D406540484C654089EA0606474C664094
:101128007519474C6540D8E9006B03AC0028C4E941
:10113800006B0EBF002404200424029E5CF800000B
:10114800345920183F4C04600126046886600398CF
:10115800029E43406340384C7068634089EA00004F
:10116800364C6040034438484340280018BF0120EB
:101178005B1E9B41042F2CBFC0B2D80F02F1140391
:1011880053F8200007F00303C3F10303DB00D84042
:101198000DF807007F1C082F9DD315460C466A6979
:1011A800AB69E868D20842EA4372401E00EA0207C7
:1011B800002302409B420AD8524508D28020E055BD
:1011C8007F1C574516D2AAEB0701E01910E08020D2
:1011D800E05500E0E355E8687F1C8742FAD32A68A7
:1011E800136828469847BAF1000F03D051462046A5
:1011F80013F0D4F92A68069E059F93686946284625
:1012080098472A68D2F8009021462846C8472B6894
:10121800DA683946284690470EB1A86830604FF41E
:10122800003007B0BDE8F08F684701085412000885
:10123800D80800205FC5109304850012FC68017A65
:10124800C0F524FF24AF33D426AF698B04B0010165
:1012580000170145F8B501240094002300240DE08F
:10126800009D065D0F5D7E40F643761CF60F86F006
:10127800010635400095641C009DEB189442EFD39D
:101288001846F2BDF8B5002301240094002A11E0A5
:10129800009C85188F1815F8016C17F8015C6E40D2
:1012A800F643761CF60F86F0010634400094009C45
:1012B800E318521EECD11846F2BD00005D1200087A
:1012C8008D120008010000002DE9F84F1D46DDF8D9
:1012D80028900B9F0D9C4FF0FF3300930E469246CB
:1012E800D9F800B0804632465146D847834664B3A1
:1012F800D9F8043032465146404698476FEA0B0207
:10130800521C42EA0B0200996FEAD2735B1C194027
:10131800C2430091521C024300996FEAD2735B1CCE
:101328001940009186F05531484087EA000181F064
:101338005531216080F05531C943491C0843009A52
:101348006FEAD070401C82430092D9F80800012847
:1013580009D17540E943491C0D4300986FEAD572DD
:10136800521C90430AE0F11C85EA9102D243521CB8
:10137800154300986FEAD5735B1C984386F0AA362C
:10138800009086EA0B0686F0AA33F243DB430C98FA
:10139800C2F3C0725B1C42EAD3720099D243521C5A
:1013A80091430091774000998843009987F0AA37C4
:1013B8000F403843BDE8F28F034613F8012B002A8B
:1013C800FBD1181A0138704781F0004102E000BFD4
:1013D80083F0004330B54FEA41044FEA430594EAED
:1013E800050F08BF90EA020F1FBF54EA000C55EA28
:1013F800020C7FEA645C7FEA655C00F0E2804FEAF9
:101408005454D4EB5555B8BF6D420CDD2C4480EADA
:10141800020281EA030382EA000083EA010180EA0A
:10142800020281EA0303362D88BF30BD11F0004F58
:101438004FEA01314FF4801C4CEA113102D040428E
:1014480061EB410113F0004F4FEA03334CEA1333C9
:1014580002D0524263EB430394EA050F00F0A780E1
:10146800A4F10104D5F1200E0DDB02FA0EFC22FADC
:1014780005F2801841F1000103FA0EF2801843FAD0
:1014880005F359410EE0A5F120050EF1200E012AC1
:1014980003FA0EFC28BF4CF0020C43FA05F3C018FF
:1014A80051EBE37101F0004507D54FF0000EDCF178
:1014B800000C7EEB00006EEB0101B1F5801F1BD321
:1014C800B1F5001F0CD349085FEA30004FEA3C0C25
:1014D80004F101044FEA445212F5800F80F09A801B
:1014E800BCF1004F08BF5FEA500C50F1000041EB1F
:1014F800045141EA050130BD5FEA4C0C404141EB23
:101508000101013C28BFB1F5801FE9D291F0000F1D
:1015180004BF01460020B1FA81F308BF2033A3F1CC
:101528000B03B3F120020CDA0C3208DD02F1140CC3
:10153800C2F10C0201FA0CF021FA02F10CE002F1FE
:101548001402D8BFC2F1200C01FA02F120FA0CFCF7
:10155800DCBF41EA0C019040E41AA2BF01EB045140
:10156800294330BD6FEA04041F3C1CDA0C340EDC3E
:1015780004F11404C4F1200220FA04F001FA02F381
:1015880040EA030021FA04F345EA030130BDC4F13F
:101598000C04C4F1200220FA02F001FA04F340EA34
:1015A8000300294630BD21FA04F0294630BD94F0E5
:1015B800000F83F4801306BF81F480110134013DCC
:1015C8004EE77FEA645C18BF7FEA655C29D094EA3D
:1015D800050F08BF90EA020F05D054EA000C04BFBB
:1015E8001946104630BD91EA030F1EBF00210020A6
:1015F80030BD5FEA545C05D14000494128BF41F045
:10160800004130BD14F580043CBF01F5801130BDA8
:1016180001F0004545F0FE4141F470014FF0000033
:1016280030BD7FEA645C1ABF194610467FEA655CE4
:101638001CBF0B46024650EA013406BF52EA033586
:1016480091EA030F41F4002130BD00BF90F0000F74
:1016580004BF0021704730B54FF4806404F13204B0
:101668004FF000054FF0000150E700BF90F0000F69
:1016780004BF0021704730B54FF4806404F1320490
:1016880010F0004548BF40424FF000013EE700BF60
:1016980042004FEAE2014FEA31014FEA02701FBFF0
:1016A80012F07F4393F07F4F81F06051704732F022
:1016B8007F4208BF704793F07F4F04BF41F4002179
:1016C800704730B54FF4607401F0004521F00041D7
:1016D8001CE700BF50EA010208BF704730B54FF061
:1016E80000050AE050EA010208BF704730B511F062
:1016F800004502D5404261EB41014FF4806404F19A
:1017080032045FEA915C3FF4D8AE4FF003025FEA1F
:10171800DC0C18BF03325FEADC0C18BF033202EBA3
:10172800DC02C2F1200300FA03FC20FA02F001FAFD
:1017380003FE40EA0E0021FA02F11444BDE600BFA0
:101748004FF0FF3C06E000BF4FF0010C02E000BF85
:101758004FF0010C4DF804CD4FEA410C7FEA6C5C68
:101768004FEA430C18BF7FEA6C5C1BD001B050EA0B
:10177800410C0CBF52EA430C91EA030F02BF90EAF6
:10178800020F0020704710F1000F91EA030F58BFB5
:10179800994208BF90422CBFD8176FEAE37040F017
:1017A800010070474FEA410C7FEA6C5C02D150EAB5
:1017B800013C07D14FEA430C7FEA6C5CD6D152EA70
:1017C800033CD3D05DF8040B704700BF8446104635
:1017D80062468C461946634600E000BF01B5FFF734
:1017E800B7FF002848BF10F1000F01BD4DF808ED04
:1017F800FFF7F4FF0CBF012000205DF808FB00BFD5
:101808004DF808EDFFF7EAFF34BF012000205DF82E
:1018180008FB00BF4DF808EDFFF7E0FF94BF01207B
:1018280000205DF808FB00BF4DF808EDFFF7CEFF7C
:1018380094BF012000205DF808FB00BF4DF808EDBB
:10184800FFF7C4FF34BF012000205DF808FB00BF8C
:101858004FEA410212F5001215D211D56FF47873D0
:10186800B3EB625212D94FEAC12343F0004343EA73
:10187800505311F0004F23FA02F018BF404270474E
:101888004FF00000704750EA013005D111F00040D8
:1018980008BF6FF0004070474FF00000704700BF6E
:1018A80080F0004002E000BF81F0004142001FBF0D
:1018B8005FEA410392EA030F7FEA226C7FEA236C16
:1018C8006AD04FEA1262D2EB1363C1BFD21841400B
:1018D80048404140B8BF5B42192B88BF704710F0A1
:1018E800004F40F4000020F07F4018BF404211F044
:1018F800004F41F4000121F07F4118BF494292EAAC
:10190800030F3FD0A2F1010241FA03FC10EB0C00D7
:10191800C3F1200301FA03F100F0004302D5494264
:1019280060EB4000B0F5000F13D3B0F1807F06D311
:1019380040084FEA310102F10102FE2A51D2B1F109
:10194800004F40EBC25008BF20F0010040EA0300FE
:101958007047490040EB0000013A28BFB0F5000F7E
:10196800EDD2B0FA80FCACF1080CB2EB0C0200FA34
:101978000CF0AABF00EBC25052421843BCBFD04083
:101988001843704792F0000F81F4000106BF80F4FD
:1019980000000132013BB5E74FEA41037FEA226CC0
:1019A80018BF7FEA236C21D092EA030F04D092F08B
:1019B800000F08BF0846704790EA010F1CBF0020BF
:1019C800704712F07F4F04D1400028BF40F000401C
:1019D800704712F100723CBF00F50000704700F03C
:1019E800004343F0FE4040F4000070477FEA226263
:1019F80016BF08467FEA23630146420206BF5FEA34
:101A0800412390EA010F40F4800070474FF0000333
:101A180004E000BF10F0004348BF40425FEA000CFA
:101A280008BF704743F0964301464FF000001CE0A2
:101A380050EA010208BF70474FF000030AE000BFF8
:101A480050EA010208BF704711F0004302D5404236
:101A580061EB41015FEA010C02BF844601460020A8
:101A680043F0B64308BFA3F18053A3F50003BCFAC3
:101A78008CF2083AA3EBC25310DB01FA02FC634470
:101A880000FA02FCC2F12002BCF1004F20FA02F277
:101A980043EB020008BF20F00100704702F120026A
:101AA80001FA02FCC2F1200250EA4C0021FA02F2CB
:101AB80043EB020008BF20EADC7070474FEA40029F
:101AC800B2F1FE4F0FD34FF09E03B3EB12620DD964
:101AD8004FEA002343F0004310F0004F23FA02F0CE
:101AE80018BF404270474FF00000704712F1610F75
:101AF80001D1420205D110F0004008BF6FF000404C
:101B080070474FF00000704753B94AB9002908BF21
:101B180000281CBF4FF0FF314FF0FF3000F070B9C4
:101B2800ADF1080C6DE904CE00F006F8DDF804E02C
:101B3800DDE9022304B070472DE9F047089E0D4601
:101B480004460F46002B4AD18A42944665D9B2FA18
:101B580082F343B102FA03FCC3F120029F4020FA4A
:101B680002F217439C404FEA1C4E1FFA8CF5B7FB54
:101B7800FEF1220C0EFB117742EA074201FB05F049
:101B880090420AD91CEB020201F1FF3780F01B8159
:101B9800904240F2188102396244121AA4B2B2FB90
:101BA800FEF00EFB102244EA024400FB05F5A542B4
:101BB8000AD91CEB040400F1FF3280F00681A5422B
:101BC80040F203816444023840EA0140641B00216A
:101BD8001EB1DC400023C6E90043BDE8F0878B4214
:101BE80008D9002E00F0EC800021C6E9000508465F
:101BF800BDE8F087B3FA83F1002949D1AB4202D39B
:101C0800824200F2F780841A65EB0302012017462E
:101C1800002EE2D0C6E90047DFE702B9FFDEB2FADC
:101C280082F3002B40F08F808A1A4FEA1C471FFA74
:101C38008CFE0121B2FBF7F507FB1520220C42EAC6
:101C480000420EFB05F0904208D91CEB020205F198
:101C5800FF3802D2904200F2CA804546121AA4B256
:101C6800B2FBF7F007FB102244EA02440EFB00FE29
:101C7800A64508D91CEB040400F1FF3202D2A645A0
:101C880000F2BA801046A4EB0E0440EA05409FE734
:101C9800C1F120078B4022FA07FC4CEA030C05FA35
:101CA80001F420FA07F3FD40234300FA01F94FEA53
:101CB8001C401FFA8CFEB5FBF0F81C0C00FB1855F5
:101CC80044EA054408FB0EF5A54202FA01F20BD9D5
:101CD8001CEB040408F1FF3A80F08780A54240F22B
:101CE8008480A8F102086444641B9DB2B4FBF0F33D
:101CF80000FB134445EA044403FB0EFEA64508D93D
:101D08001CEB040403F1FF306BD2A64569D9023BF2
:101D1800644443EA0840A0FB0283A4EB0E049C42FF
:101D2800C6461D4655D352D056B1B9EB0E0364EBE7
:101D3800050404FA07F7CB40CC401F43C6E90074FA
:101D48000021BDE8F087C3F1200102FA03FC20FA64
:101D580001F225FA01F19D402A434FEA1C471FFA78
:101D68008CFEB1FBF7F007FB1015110C41EA054199
:101D780000FB0EF58D4204FA03F408D91CEB0101AF
:101D880000F1FF382FD28D422DD902386144491B0A
:101D980092B2B1FBF7F507FB151142EA014205FBC8
:101DA8000EF1914208D91CEB020205F1FF3816D258
:101DB800914214D9023D6244521A45EA004139E77A
:101DC8003146304609E73946E7E61046FCE6C145A4
:101DD800AAD2B8EB020E63EB0C050138A4E745461E
:101DE800EAE7034695E74046D1E7D0467CE7023D5F
:101DF800624433E708460BE76444023843E700BF10
:101E0800704700BF1348144A08B54FF00043C0E9B3
:101E180000230422002342610122C2614FF4805151
:101E280007220383C0E90233C0E90933C0E90C1271
:101E38000361837680F8203080F82C30826380F844
:101E48003C30C36405F00EFB18B1BDE8084000F053
:101E580017BC08BDDC080020002401400268084BBC
:101E68009A4282B00AD14FF0B0431A6E42F400721F
:101E78001A661B6E03F400730193019B02B070474E
:101E8800002401400268054B9A4201BF4FF0B0425E
:101E9800136E23F400731366704700BF00240140DB
:101EA80030B585B000240546CDE901440394FFF719
:101EB800A9FF144805F06EFE08B100F0E1FB1148D7
:101EC800039401A9CDE9015405F02AFC08B100F0FA
:101ED800D7FB0C4805F088FD08B100F0D1FB4FF0A6
:101EE800FF31084805F0BEFB064805F035FE0548F9
:101EF80005F012FC0446034805F0D8FD204605B05D
:101F080030BD00BFDC080020014B024A1A60704750
:101F1800DC0800200024014008B50948FFF7C0FF8D
:101F280068B1084BB3F8AA304FF6FF72934216BF58
:101F380040F6E442044B5343B3FBF0F398B208BDB8
:101F4800002000B40075FF1FD8084C0013B500230B
:101F5800ADF80630FFF7E0FF04461948FFF7A0FF89
:101F6800184BB3F8C820B3F8A8108A4204FB00F055
:101F780018D040F6E443B0FBF3F364205B1A434304
:101F8800521A93FBF2F31E331BB2ADF80630BDF8BC
:101F980006305BB21B02ADF80630BDF8060000B291
:101FA80002B010BD4FF47A7240F6FF73B0FBF3F342
:101FB8005343A3F53923A3F50C6340F6C412E0E7B5
:101FC800001000B00075FF1F4FF0B04382B09A6A4E
:101FD80022F480529A629A6C42F480529A649B6C02
:101FE80003F480530193019B002002B070474FF027
:101FF800B04382B09A6C02439A649B6C034001938D
:10200800019B02B0704708B50420FFF7F0FF0120DC
:10201800FFF7EDFF0220FFF7EAFF002211460B2031
:1020280005F056FE0B2005F085FE002211460C2017
:1020380005F04EFE0C2005F07DFE002211460D2015
:1020480005F046FE0D2005F075FE002211460E2013
:1020580005F03EFE0E2005F06DFE002211460F2011
:1020680005F036FE0F2005F065FE0022114610200F
:1020780005F02EFE102005F05DFE0022114611200D
:1020880005F026FE112005F055FE002236201146E7
:1020980005F01EFEBDE80840362005F04BBE0000E6
:1020A80008B506F08FF810B16FF0040008BD064BB4
:1020B8009A6942F040429A614CF2FA321A6106F08B
:1020C80093F80028F2D0EFE700400058F0B585B04B
:1020D80000230C4600930646A8B3FFF7E1FF054628
:1020E80070BB06F06FF888BB1A481B4A022301939D
:1020F800D0F8E01506F1784302EA8121B3FBF1F745
:1021080001FB1733DB0A0293D0F8E00504F17841AC
:102118000139314402EA8022B1FBF2F002FB1011CE
:10212800C3EBD1230133694601A8039306F0DCF819
:1021380020B102280CBF01256FF0010506F054F804
:10214800284605B0F0BD6FF00505F9E76FF0040506
:10215800F6E700BF0070FF1F00FCFF03014B18608B
:1021680000207047400900202DE9F04F89B0B0F1F8
:10217800006F06460F460092C0F0C580DFF89881D0
:10218800664DD8F8E03505EA832303F10063013B87
:10219800984200F2B880002800F0B880002900F0CA
:1021A800B58040EA02035B0740F0B080FFF778FF94
:1021B8000446A0BB06F006F8002840F0AA80D8F82C
:1021C800E01506F1784205EA8121B2FBF1F301FB43
:1021D8001322009B03F17843013B3344B3FBF1F036
:1021E80001FB1033DB0A01334FEAD22AA3EBD222D8
:1021F800012A039388BFC6F30A050AF58038C6F199
:10220800080398BF009D069388BFC5F500654FEA8F
:10221800C828B346039B9A4505D305F0E5FF204639
:1022280009B0BDE8F08FA6F10803069A1A44954252
:1022380019D804950197CDF814B04FF00009059B03
:1022480009EB0301049B99453ED3009BAB442F4403
:102258005D1BB5F5006F28BF4FF400650AF1010A50
:1022680008F50068D6E753F8081F5A68B2F1FF3F2F
:1022780008BFB1F1FF3FD8D0294B186810B96FF0EB
:102288000504CAE7B8F1000F04D04FF400624146D4
:1022980011F016FDDFF88890D9F80030CBF30A006A
:1022A80039461844AAB211F00BFD4FF400614046BC
:1022B800FFF70CFF08BBD9F8003001934FF4006317
:1022C800CDF814800493B8E7019B07914B4402931F
:1022D8000120D3E9002305F0C1FF88B90799019BC4
:1022E800D1E9000259F80310029B5B689A4208BFC3
:1022F800884205D109F10809A1E76FF001048CE7CC
:102308006FF0030489E74FF0FF3488E76FF00504A6
:1023180085E76FF0040482E70070FF1F00FCFF03ED
:1023280040090020B1F1006F70B511D30B4BD3F801
:10233800E0650B4B03EA862303F10063013B9942F6
:1023480006D840B139B192B211F0BAFC002070BD84
:102358004FF0FF30FBE76FF00500F8E70070FF1F54
:1023680000FCFF03B0F1006F10B40DD3084BD3F895
:10237800E045084B03EA842303F10063013B9842DC
:1023880002D810BCFFF7A2BE4FF0FF3010BC704758
:102398000070FF1F00FCFF034FF0B04382B0DA6CFF
:1023A8000243DA64DB6C03400193019B02B070477F
:1023B80070B586B01422002101A812F0B9F80120E6
:1023C800FFF7EAFF0220FFF7E7FF0420FFF7E4FF2B
:1023D8004FF4007101224FF0904006F0F9F8012502
:1023E80002234FF4041401A94FF09040CDE90134C1
:1023F800224E039505F0C6FF4FF4441301A94FF090
:102408009040CDE90235019505F0BCFF2023CDE9C8
:10241800013401A900243046039405F0B3FF4FF4BA
:10242800007301A94FF09040CDE90135CDE903547F
:1024380005F0A8FF04230DEB03013046CDE9013573
:10244800CDE9034405F09EFF22462146062005F00B
:102458003FFC062005F06EFC22462146072005F0C9
:1024680037FC072005F066FC22462146162005F0B9
:102478002FFC162005F05EFC06B070BD0004004875
:1024880008B51248124A134BC0E900230023012261
:10249800C0E90232C0E90433C0E90633036206F03A
:1024A8000BFA08B100F0ECF80848002106F084FBAC
:1024B80008B100F0E5F80548002106F0A3FB18B1C3
:1024C800BDE8084000F0DCB808BD00BF040A0020E1
:1024D800005800405D3E302070B596B00546142285
:1024E800002103A812F024F83822002108A812F0CD
:1024F8001FF82A68304B9A425BD18023089308A8BA
:102508004FF440230E9307F0D9F808B100F0B8F85B
:102518004FF0B0444FF4C050E36C43F00103E36460
:10252800E36C03F001030293029B12230026CDE91A
:1025380003030323CDE905634FF09040042303A967
:10254800079305F01FFFA36DDFF870C043F4800305
:10255800A365A36D1A4C03F480030193019B2662C3
:102568000D23C4E900C320468023C4E90266C4E9F8
:102578000436C4E9066605F03DFC08B100F080F8B1
:10258800104AEC63A562104C0E23C4E90023102105
:10259800002380222046C4E90213C4E90423C4E9C5
:1025A8000633236205F026FC08B100F069F8AC6335
:1025B800A56216B070BD00BF00580040440002403C
:1025C8004409002058000240A409002000B59BB02F
:1025D8004822002108A811F0ABFF1822002102A808
:1025E80011F0A6FF06F034FB4FF0B0420120D2F8FC
:1025F800903023F01803C2F89030D2F8003423F456
:10260800C06343F40073C2F80034D2F8003403F412
:10261800C0630193019B2423089381230B93002318
:10262800CDE91003B02208A8CDE9122306F088FCF2
:1026380008B172B6FEE74F23CDE90230CDE90400B8
:10264800CDE90600022102A806F014FF08B172B60F
:10265800FEE71BB05DF804FB08B504F0B1FEFFF718
:10266800B5FFFFF7A5FEFFF7CEFCFFF709FF00F067
:10267800F8FD40F6B83000F049FA00F0F9FDFCE743
:1026880072B6FEE700B58DB02C22002101A811F02A
:102698004FFF1748174B03601F2383604FF080429A
:1026A8000023C0E90433C0E9072383614FF4807332
:1026B800436207F089F908B1FFF7E2FF0C4807F019
:1026C800AFFA08B1FFF7DCFF4FF000530022079381
:1026D800074808924FF4807301A9029206920B935F
:1026E80007F0D2F908B1FFF7CBFF0DB05DF804FB96
:1026F800580A00200028004010B5044690B038223F
:10270800002102A811F014FF2268194B9A422CD11B
:102718004FF48033029302A84FF480730F9306F0AE
:10272800CDFF08B1FFF7ACFF4FF0B0430220D3F85C
:10273800902042F40042C3F890209A6D42F48062DF
:102748009A659B6D002203F4806311460193019BF7
:1027580005F0BEFA022005F0EDFA00222A20114603
:1027680005F0B6FA2A2005F0E5FA10B010BD00BF52
:10277800002800407047000008B504F037FE044BFD
:102788000120C3F88800BDE8084006F0B9BA00BFC8
:102798000004005804F031BE08B504F02EFE00F025
:1027A80063FCFFF705FEFFF72EFCBDE80840FFF7C6
:1027B80067BE08B504F01AFEBDE8084001210020F4
:1027C80006F04EBA70477047FEE7FEE7FEE7FEE701
:1027D800FEE770477047704770470000014807F0F0
:1027E80045BA00BF580A0020012005F0F7BE0220B4
:1027F80005F0F4BE70477047014805F075BC00BF8E
:1028080044090020014805F06FBC00BF300B0020D0
:10281800014805F069BC00BFD00A0020FFF7F2BFED
:102828007047202005F0DABE70470000014807F025
:10283800E1BD00BF900B0020014807F049B800BF78
:10284800580A0020014807F03CBC00BFBC0A002021
:102858002DE9F04389B080460020109E07908946F4
:1028680015461F46FDF7DCFCF0B9104CCDE9009089
:10287800CDE9020407AB0E480593142304933A46A6
:10288800434629460068FDF795FD2346324604F184
:10289800140153F8044B42F8044B8B42F9D1079BBF
:1028A800337509B0BDE8F0830120FAE7900A0020EB
:1028B800644701087FB5124C00253C2302A86375C4
:1028C800CDE90255257500F0C3F8042303AA009446
:1028D80012210C48FFF7BCFF0B491422204611F0C7
:1028E80017FE0646B0FA80F0400960750090074B65
:1028F8002A462946022011F0DBF8304604B070BDA4
:10290800A40A0020AA4701083E0E00208C470108AF
:10291800054808B50823036007F0EEF918B1BDE8CB
:102928000840FFF7ADBE08BDBC0A00204FF0B04319
:1029380007B55A6E42F001025A665B6E002203F038
:102948000103019311463220019B05F0C1F93220A1
:1029580003B05DF804EB05F0EDB900000CB407B561
:10296800054A05AB1021019311F0B4FC03B05DF8E2
:1029780004EB02B0704700BFBC47010830B585B012
:10298800044602A80D4611F0D1FABDF90C30064AEA
:1029980000931021029B2046FFF7E0FF2046FEF738
:1029A8000BFD288005B030BDBC4701084FF0B04290
:1029B80010B5936823F40043936011F03FFB0E4B6E
:1029C80001241C7000F0B6F811F008F80B4811F05B
:1029D8001FF80B4B4FF400421A61032011F01EF848
:1029E800FFF792FA00F012F911F014F92146204687
:1029F800BDE8104011F02EB9C80A0020852900084A
:102A08000040005811F03CB908B5FFF785FA40F6C8
:102A1800B83398420CD8B0F5E16F0BD3FE23A0F57C
:102A2800E16058434FF49663B0FBF3F0C0B208BDC1
:102A3800FE20FCE70020FAE77FB5684600F0CAF8F8
:102A48000198FFF73BF800B207B05DF804FB0000FF
:102A5800194A38B5D2F88035591C044619D104F002
:102A6800D3FC054604F0DCFC054404F0D3FC2B0E33
:102A7800E3712B0CA3712B0A6371030EE370C0F38F
:102A88000742C0F307232571C0B2A270637020709B
:102A980038BD190AC3718171190C1B0E417103717C
:102AA800D2F88435C370D2F88405C0F30722C0F386
:102AB8000743000EE9E700BF0070FF1F38B5094B58
:102AC800D3F8803503600133054609D104F09CFC36
:102AD800044604F09FFC444004F0A2FC44402C60EF
:102AE80038BD00BF0070FF1F0121022011F09CB803
:102AF8000021022011F098B800207047024B187886
:102B080008B100F0BBB87047C80A002082B0019035
:102B1800019802B000F04EB94FF0B04382B0DA6CC1
:102B280042F00202DA64DB6C03F002030193019BBA
:102B380002B070472DE9F043254C87B004F076FCCD
:102B480004F07CFC04F082FC0123002502934FF47E
:102B58008059032301A9204604934FF40058039594
:102B68000595FFF7D9FFFFF7D7FFFFF7D5FFFFF769
:102B7800D3FFCDF8049005F005FC01A920464FF4D9
:102B88000067CDF8048005F0FDFB01A920464FF44D
:102B98000046019705F0F6FB01A92046019605F0CD
:102BA800F1FB2A464946204605F012FD2A464146D1
:102BB800204605F00DFD2A463946204605F008FD59
:102BC8002A463146204605F003FD07B0BDE8F083EC
:102BD8000004004810B50446FFF7B8F9074BA36096
:102BE80040F30F20FEF716FF054B064A2360064BFD
:102BF8006060C4E90323002010BD00BF0000484204
:102C080000007A440D093E00AB0305000020704720
:102C1800014B1868704700BFCC0A0020032070479A
:102C280008B501464FF47A7200238002890DFEF739
:102C38006BFF08BD4FF47A73A0FB0303800A40EAD8
:102C480083507047034B98689A689042FBD1C04301
:102C5800704700BF0028004008B5FFF7F3FF014B9D
:102C6800186008BDCC0A002008B5FFF7EBFF024B3F
:102C78001B68C01A08BD00BFCC0A0020024B187898
:102C880008B1FFF7DFBF7047C90A002010B5074B2E
:102C9800074C0122DA654FF48071204606F0DEFD0C
:102CA8004FF0FF332363002010BD00BF0028004011
:102CB800580A002002460021014806F0E8BF00BF7C
:102CC800580A002002460121014806F0E0BF00BF73
:102CD800580A002010B58CB02C220021044601A807
:102CE80011F026FCFFF7D2FF0C4B0D481B681C4463
:102CF8000023089306934FF00053E44307930122FF
:102D08004FF4807301A902940B9306F0BDFE08B13D
:102D1800FFF7B6FC00200CB010BD00BFCC0A0020A5
:102D2800580A002038B50546FFF78CFF02210446F3
:102D3800074806F0B3FFC4F309024FF47A71A2FB07
:102D48000121920AA30A2A8043EA805038BD00BFB5
:102D5800580A00200148002106F0A0BF580A0020A8
:102D68000148012106F09ABF580A0020F8B50F4D16
:102D78002E78CEB90E4C4FF0FF372763FFF782FC51
:102D8800FFF784FF4FF48071204606F067FD204668
:102D9800276306F027FF32462046022106F077FF18
:102DA800FFF75AFF01232B700020F8BDC90A002045
:102DB800580A0020014610B54FF47A7200238002A9
:102DC800890DFEF7A1FE0146FFF73CFF0446FFF719
:102DD80039FF031B8B4200D310BD00BFF7E711F08A
:102DE80035BA000010B5064C0221204606F056FF01
:102DF8000221421C2046BDE8104006F048BF00BF33
:102E0800580A00201648174A08B54FF4E133C0E9BC
:102E1800002300230C22C0E90233C0E90523C0E9DE
:102E28000733C0E90933036108F0C5F808B1FFF7B3
:102E380027FC0B48002108F03AFA08B1FFF720FCFC
:102E48000748002108F053FA08B1FFF719FC0448B5
:102E580008F00DFA18B1BDE80840FFF711BC08BD2D
:102E6800900B00200044004070B596B0054614222F
:102E7800002103A811F05CFB3822002108A811F0FA
:102E880057FB2A68334B9A4261D10223089308A85A
:102E9800314B0A9306F012FC08B1FFF7F1FB4FF033
:102EA800B0430C219A6D2D4C42F400329A659A6D0C
:102EB80002F400320292029ADA6C42F00102DA64F9
:102EC800DB6C03F001030193019B02230026CDE98B
:102ED80003130323CDE905634FF09040072303A9AB
:102EE800079305F04FFA1E4826621423C4E900032D
:102EF8001023C4E9023620468023C4E90436C4E915
:102F0800066604F077FF08B1FFF7BAFB154AEC67CD
:102F1800A562154C1323C4E9002320460023802210
:102F2800C4E90233C4E90423C4E90633236204F084
:102F380061FF08B1FFF7A4FB2520C5F880400022F7
:102F48000221A56204F0C4FE252004F0F3FE16B0A9
:102F580070BD00BF0044004004000C00300B00208E
:102F6800800002406C000240D00A002002680E4B2C
:102F78009A4210B5044616D14FF0B0420C21936D19
:102F880023F4003393654FF0904005F0A7FAE06F03
:102F980004F0A4FFD4F8800004F0A0FFBDE81040BE
:102FA800252004F0D5BE10BD0044004008B50A46EF
:102FB8000146024807F082F9002008BD900B002066
:102FC80013B5114B114C18604FF40013009302AB6A
:102FD80013E90600204608F0EEF82368DA69D10301
:102FE800FCD4DA695202FCD59A68084842F4800297
:102FF8009A6008F026F906490448012208F094F876
:10300800002002B010BD00BF240C0020900B00204F
:103018002C0C002008B5074B1860FEF7F4FFFFF7EB
:10302800F1FE054AD2F8803043F00063C2F88030E0
:10303800002008BD280C00200008005808B54FF0F3
:10304800B04308489A6B42F400329A639A6B22F4B0
:1030580000329A63FFF78AFF0F2004F079FE002000
:1030680008BD00BF900B002008B5074807F0A3FF74
:1030780008B1FFF705FB054804F0BCFE18B1BDE830
:103088000840FFF7FDBA08BD900B0020300B002068
:103098000268044B9A4203D1034B00201B6818476F
:1030A800704700BF00440040280C002002680B4B0A
:1030B8009A4210B504460FD1094B1B682BB1D0F8C2
:1030C800902012B907480121984720460549BDE8D4
:1030D8001040012208F028B810BD00BF004400408D
:1030E800240C00202C0C002002480122102105F09D
:1030F8006FBA00BF0004004802480022102105F002
:1031080067BA00BF0004004813B5134C23785BB9B5
:10311800E37C03F0FF023BB9104B1146022002B0DA
:10312800BDE8104010F0C4BCFFF7C4FB00380C4BDE
:1031380018BF0120400018701A78022A02BF002226
:103148002270E2741B7800930022064B114603207C
:1031580010F0AEFC02B010BD3E0E00201848010869
:10316800340C00203448010838B5184C23785BBB70
:10317800E37C03F0FF023BBB154D2B68012B0CD9F8
:103188002B68042B09D81146124B022010F090FC32
:10319800114A0421012000F079FB2B68042B13D974
:1031A80000220E4B1146022010F082FCFFF782FB32
:1031B80000380B4B18BF0120400018701B78022BF9
:1031C80002BF00232370E37438BD00BF3E0E002009
:1031D800300C00204B480108704801087548010868
:1031E800340C002008B5FFF77FFF0022054B11467D
:1031F800032010F05DFC01F015FDBDE80840FFF765
:103208007BBF00BFA8480108022801D8FFF76CBFA0
:103218007047022801D8FFF76FBF7047022808B52A
:103228001BD8012210210D4805F0D2F93220FFF7F2
:103238006DFC0A480022102105F0CAF9012210216C
:10324800064805F0C5F93220FFF760FCBDE80840E4
:1032580002480022102105F0BBB908BD000400484F
:10326800704708B5FFF7A2FBBDE8084000F0D8BCDE
:103278004FF0FF3010F068BD70477047014BD870B1
:10328800704700BF5C000020014B1874704700BFF6
:103298005C00002007B5064B00221B5C009311461A
:1032A800044B022010F004FC03B05DF804FB00BFDF
:1032B800E4480108CA48010808B50220002110F0B6
:1032C8000BFDBDE80840014810F06EBF8C0D0020D2
:1032D8000021012010F000BD13B50D4CA0B12060F5
:1032E8000C4810F013FF21680A4810F097FF0948AE
:1032F80010F05AFF236800930022074B1146032061
:1033080010F0D6FB02B010BD42F210732360E7E75D
:10331800740000208C0D0020E848010813B50D4CFE
:10332800206023680BB90C4B23600C4810F0EEFEAC
:1033380021680A4810F072FF084810F035FF23682A
:1033480000930022064B1146032010F0B1FB02B097
:1033580010BD00BF0C000020A0860100A40D0020B5
:103368001149010837B5044600283AD090F90650AB
:10337800002D38D11F4810F0C9FE2A4629461E4B99
:10338800022010F095FBE379012B0CBF1B4B1C4B63
:103398002A46294602201B4D10F08AFBE3792B7040
:1033A800194B1868FFF7BAFF184B1868FFF794FF16
:1033B8002978174A174B012918BF13460022009392
:1033C8001146154B032010F073FB94F90530019357
:1033D80094F9043000930022104B1146022010F09B
:1033E80067FB03B030BD00220D4B1146022010F0E0
:1033F8005FFBEAE7280D0020564901086B490108E0
:1034080088490108580D00200C0000207400002095
:10341800514901084D490108A5490108DD4901083C
:10342800C449010838B504460D4607484FF4006101
:10343800FEF798FF30B92A4621460348BDE83840D0
:10344800FEF792BE38BD00BF00F003080A460149E6
:10345800FEF768BF00F0030870B5164810F056FE76
:1034680008F0AAFB044650B10022134B1146022073
:1034780010F01EFBBDE87040104810F095BE104DCE
:10348800104B02460146022010F012FB01260E4B9B
:103498002E7022462146022010F00AFB0B4808F045
:1034A8001DFA2878314607F06FFF024810F07CFEBD
:1034B800E0E700BF8C0D0020064A01085C0D0020E3
:1034C80000000020244A0108384A01085C00002056
:1034D80030B587B0FFF798FA044608F04BF8054670
:1034E80080B10024434810F011FE434B414819684D
:1034F800A14238BF214610F091FE3E4810F054FE1C
:1035080007B030BD01464FF4807010F0E5FB02A80B
:1035180001F09EF923B203EB4303FE2203EB4313AE
:10352800B3FBF2F3354A0B2111703549506809781D
:10353800DBB28DF8143001705068457050681A2459
:10354800847050680124C470506803712D4B18783A
:1035580040B11D700C231370536861F07F0119701E
:10356800052314E0284B2948197811B90178002956
:10357800F6D0002101701970536802215971BDF805
:1035880008305168180A88715168CB71082320499E
:10359800204C0978012988BF00235370637A33B11E
:1035A80007F0D4FF012802D1204610F0AFFD1A4BD6
:1035B8001248D978002207F0F3FF044630B90146D3
:1035C800164B0122032010F073FA8BE7063488D1DA
:1035D80007F0B6FF0446002884D001224FF47A731E
:1035E8000021B0FBF3F3104600930D4B10F060FA86
:1035F80078E700BF8C0D0020740000200400002034
:10360800270D0020BC0D0020530E00203D0E002089
:10361800340C0020280D00205C000020574A0108C7
:10362800664A010800B503468DB000282CD04078C2
:1036380002280AD003282AD0164B0022114602205D
:103648000DB05DF804EB10F033BA1A7F0B92DA7EF6
:103658000A929A7E09925A7E08921A7E0792DA7D19
:1036680006929A7D05925A680492DA68039293F951
:1036780014200292B3F9122001921B7C00930022BD
:10368800054B114610F014FA0DB05DF804FB034B1E
:10369800D3E700BF844A01089B4A01080D4B010883
:1036A80001284FF000020CBF024B034B11460220C9
:1036B80010F0FEB92C4B01083E4B01081FB504461B
:1036C800002831D00378002B2ED01D4810F06CFD57
:1036D800002211461B4B022010F0EAF994F9183029
:1036E800039394F90A300293237C0193E3680093CF
:1036F80000221146144B032010F0DAF90022134B74
:103708001146032010F0D4F9237A012B0ED1617AE7
:103718000F4A104B002908BF134600220093114698
:103728000D4B032010F0C4F904B010BD00220B4B60
:103738001146032004B0BDE8104010F0B9B900BF2D
:10374800740D0020574B0108884B0108B94B01083C
:10375800524B0108534B0108C64B0108D74B0108CF
:1037680008B5104B0122002102201A7010F0B4FA9B
:103778000D4810F019FD0D4B1B788BB10C4B1A78C6
:1037880072B9DB7C63B90B4B1A68042A9EBF1A68AE
:1037980001321A600021BDE80840102010F09CBAE0
:1037A80008BD00BFBC0D0020A40D0020580D00204E
:1037B8003E0E0020300C0020044B1B78022B03D156
:1037C8000021082010F088BA704700BF00000020D0
:1037D80008B508F0FAF980B907F0B8FE01280CD14D
:1037E800BFF34F8F0549064BCA6802F4E0621343E2
:1037F800CB60BFF34F8F00BFFDE708BD00ED00E0D1
:103808000400FA0510B508F073FA10F1080F07D193
:10381800064B0022BDE810401146022010F048B9BE
:10382800013001D1024BF4E710BD00BFE54B0108A0
:10383800FB4B010870477047022813B5014618D0A2
:10384800202819D001281AD14FF0904004F0BAFE70
:103858000022044600900B4B1146032010F028F973
:10386800012C0CD10021022002B0BDE8104010F05C
:1038780033BA00210820F7E7034B01221A7002B07F
:1038880010BD00BF134C0108B80E002073B50546E3
:103898000C46164607F06EFE0346002838D0002472
:1038A800264810F033FC264B24481968A14238BF3B
:1038B800214610F0B3FC214802B0BDE8704010F07A
:1038C80073BC4A68F05CD0540133DAB2A242F8D330
:1038D8001C4B0D701B78012B88BF00244C701A4CB0
:1038E800637A33B107F032FE012802D1204610F086
:1038F8000DFC164B1648D978002207F051FE0446F5
:1039080040B90146134B0122032010F0D1F8C7E754
:103918000F49DAE70634C2D107F012FE0446002840
:10392800BED04FF47A730122B0FBF3F30021009369
:103938000320094B10F0BCF8B2E700BF8C0D002043
:1039480074000020340C0020280D00205C000020AA
:1039580004000020574A0108664A0108044B1B78F6
:1039680023B9044A05210120FFF790BF704700BF23
:10397800340C0020314C010810B5002490B03C22D2
:10398800214601A8009410F0D3FD2F4B2022DA72B3
:1039980019788DF8001059788DF8011099788DF8FC
:1039A8000210D9788DF8031019798DF80410597917
:1039B8008DF8051099798DF80610D9798DF80710CA
:1039C800197A8DF80810597A8DF80910997A8DF8B6
:1039D8000A108DF80B2021460DF10B025818013101
:1039E800007B02F8010F1C29F8D193F828208DF8E4
:1039F800282093F829208DF8292093F82A208DF87B
:103A08002A2093F82B208DF82B2093F82C206AB1CC
:103A180093F83F2052B10DF12B0100229818013282
:103A280090F82C0001F8010F142AF7D107484FF439
:103A38000061FEF797FC20B9044840226946FEF76A
:103A480093FB10B010BD00BF7800002000F80308F9
:103A58000149402210F034B900F8030870B52A4D26
:103A680028796B794D2BC0B233D1C0EB00108000A0
:103A78000A2838BF0A204FF47A735843234BAC798D
:103A88001860EB794D2BE4B22BD1C4EB0414A400DD
:103A980095F82C301E4E63BB95F83F304BBB42F275
:103AA8001070FFF719FC3068FFF738FC2B7A194AB9
:103AB8001949DBB213706B7A184ADBB21370002312
:103AC800EA1892F82C20D2B2CA540133142BF7D139
:103AD80070BD6B79482B0ABF4FF461636B7958430B
:103AE800C6E7EB79482B0ABF4FF46163EB795C4377
:103AF800CEE7FFF7F1FB012C38BF01244FF47A73AE
:103B08005C433460CFE700BF7800002074000020D9
:103B18000C000020520E00203E0E0020340C002025
:103B280010B590B000213C2201A8009110F000FDD2
:103B380040223749684610F0C3F89DF800203AB98A
:103B48009DF801001A2803D19DF80210012914D00C
:103B5800002211462F4B03200FF0AAFFFFF70CFF9E
:103B68002D481422002110F0B5F84FF47A70FEF7B2
:103B7800CDFFFFF773FF10B010BD284B1A705870B7
:103B880099709DF80310D9709DF8041019719DF86B
:103B9800051059719DF8061099719DF80710D97193
:103BA8009DF8081019729DF8091059729DF80A10AD
:103BB80099729DF80B1001F03F01D972D87AD1B2F1
:103BC80088421BD89DF8282083F828209DF82920B2
:103BD80083F829209DF82A2083F82A209DF82B2095
:103BE80083F82B200DF12B0100229818013211F8CF
:103BF800014F80F82C40142AF7D1BAE701F14000B0
:103C08006844194410F8340C08730132D6E700BF31
:103C180000F80308374C01083E0E00207800002009
:103C2800F0B50B238BB0122200240125CDE9063212
:103C380003271A231721CDE9043122465F4B039449
:103C48002146CDE901550097284609940FF030FF29
:103C58005B4B009522462146CDE9017402200FF006
:103C680027FF02260523CDE900632246554B02941F
:103C7800214630460FF01CFF534B00952246214643
:103C8800CDE9017430460FF013FF09A9204607F06B
:103C98007FFF099BC3F307220292C3F307421B0E5F
:103CA800019200932246494B214630460FF000FF0F
:103CB80009A9284607F06CFF099BDAB20392C3F3FF
:103CC80007220292C3F307421B0E01920093224679
:103CD8003F4B214630460FF0EBFE3E4B3E480094EA
:103CE80022464FF4FA7110F0B3F93C4B3C4800946B
:103CF80022464FF4FA7110F0ABF93A4B3A48009467
:103D08002A464FF4FA7110F0A3F92046FEF726FA76
:103D180008B1FEF7B5FC354B009400224FF4FA6168
:103D2800334810F095F9334A0021012010F090F83B
:103D3800314A0021022010F08BF8304A002104207B
:103D480010F086F82E4A0021082010F081F800F0C3
:103D580005FC2C492C4807F0D1FE2C4807F0BEFD85
:103D6800214810F021FA2A4B0021187807F00CFBA3
:103D780028490094284B09682848002210F068F95F
:103D8800264810F011FAFFF7CBFE254A0021102033
:103D980010F05EF8234A00214FF4807010F058F8B4
:103DA800214B22481968224B0094002210F050F948
:103DB8001E4810F0F9F90BB0F0BD00BF794C0108AE
:103DC800C04C0108E14C0108024D0108234D0108CF
:103DD800444D010881320008740D00203F38000866
:103DE800400D00203D380008280D0020C13700088C
:103DF8005C0D0020DDB60008D93400080D38000835
:103E08006134000800000301100000205C0000205D
:103E18000000002074000020C13200088C0D002032
:103E280071310008ED3100080C000020A40D0020BD
:103E38006937000830B50024A5B021467C2205A8C2
:103E4800049410F075FB53238DF810304FF48D73E4
:103E5800ADF812300123ADF80C408DF81430FEF7A0
:103E6800D3FD00B200EB4000FE2300EB4010B0FB96
:103E7800F3F08DF8150003A800F0FAFC2246009034
:103E880021461C4B054603200FF012FE07249DB95E
:103E980058238DF8163030228021174810F048FB3F
:103EA800224604A9144810F07CFB134A214601203D
:103EB800FFF7ECFC25B030BD8DF816408DF8175093
:103EC80000F0B0FE0D4B1A6812128DF818201A680F
:103ED8008DF819205A6812128DF81A205A688DF830
:103EE8001B209A689B688DF81D3012128DF81C20D3
:103EF8000E24D0E7684D0108BD0D0020E40E002017
:103F0800F0B50378592B95B0044640F01082052986
:103F18005FD84378443B162B5BD8DFE813F03401B5
:103F28005A0024015A002C015A005A005A005A001B
:103F38008E005A000F015A005A005A00AB015A006D
:103F48005A00B2005A005A005A0017008578482DC6
:103F580017D1BC4A14210120FFF798FC41F28830A0
:103F6800FEF7D4FD0022B84B114603200FF0A0FD48
:103F780040F6B830FEF7CAFD15B0BDE8F040FFF7CF
:103F880027BC532D0ED130228021B04810F0D0FA32
:103F9800FFF750FF41F28830FEF7B8FDAB4A152114
:103FA800012083E0432D16D1002404A88DF8104089
:103FB80007F00CFCA54A4C2313701A2393709DF844
:103FC8001030547001204133D07013710521FFF770
:103FD8005DFC15B0F0BD442DFBD19C4C59232370DA
:103FE8005A236370A57000F024FC2C228021201D28
:103FF80010F09EFA00232570637001251A23A37020
:10400800E5702571FEF700FD9149FE23B0FBF3F042
:104018004B6864229BB2B3FBF2F3A3714B6800EBCD
:1040280040009BB200EB4010B3FBF2F102FB1133EE
:104038006071E37122460821B2E78378303BDBB236
:10404800092BC6D8834C844A23702378DBB2537279
:104058007E4A592313704D2353702378303393705D
:1040680003210120FFF712FC2378009300227B4BE9
:10407800114601200FF01CFD15B0BDE8F040FFF718
:104088007BBC8578482D16D1704A562313700023BF
:1040980053701A23937003231371172353710B233F
:1040A800012093711223D070D371082115B0BDE897
:1040B800F040FFF7EBBB432D8BD1644C00213C2231
:1040C80005A8049110F034FA04A8FFF7C1FC2422D3
:1040D800802104F10C0010F02BFA9DF81030637069
:1040E8009DF81130A3709DF81230E3709DF81330DD
:1040F80023719DF8143063719DF81530A3719DF8F4
:104108001630E3719DF8173023729DF8183025702A
:1041180063729DF81B509DF81930A3729DF81A30F0
:10412800E3722A4607A9257304F10D0010F039FA45
:1041380005F10D012246C9B2012048E780783928E7
:104148000CD83038C0B2FFF75FF8404A23781370B4
:1041580063785370A3789370032121E715B0BDE805
:10416800F040FFF7FBBB80783928F7D83038C0B269
:10417800FFF74FF8E9E780783928EFD83038C0B230
:10418800FFF74CF8E1E78378303BDAB2092AE5D843
:10419800C578303DEAB2092AE0D80179A1F1480290
:1041A800D2B20B2ADAD82E4840FA02F2D007D5D478
:1041B8000A224D2902FB03553FD13C235D43294B7D
:1041C8004FF47A7068431860274B1860FFF784F83B
:1041D8001E4A2378137063785370A3789370E3783A
:1041E800D3702379137105210120FFF74FFB1A4B78
:1041F8001A2200261E705A7001229A70DA70A1786D
:10420800303901EB8100E178303901EB4001C9B266
:10421800197122795A71154A1278D2B21A720D4A56
:104228001278D2B25A72FFF7A7FB114B00953246AB
:10423800314603200FF03CFCCBE64829BFD14FF4B0
:104248006163BBE7754D01088A4D0108BD0D00206B
:10425800E40E0020340C002078000020AC4D01084A
:10426800DEF7FFFF740000200C000020520E002033
:10427800D54D01088378303BDAB2092A3FF66EAF94
:10428800C578303DEAB2092A3FF668AF0179A1F155
:104298004802D2B20B2A3FF661AF734840FA02F2E5
:1042A800D2073FF55BAF0A224D2902FB035539D1EE
:1042B8003C235D436D4A4FF47A736B431360106877
:1042C800FFF72CF86A4A2378137063785370A37841
:1042D8009370E378D3702379137105210120FFF7D8
:1042E800D5FA644B1A2200261E705A7001229A7061
:1042F800DA70A178303901EB8100E178303901EBCF
:104308004001C9B299712279DA715B4A1278D2B246
:104318001A725A4A1278D2B25A72FFF72DFB584BCA
:10432800009584E74829C5D14FF46163C1E7502B54
:104338005DD102297FF64DAE4378303B012B3FF625
:1043480048AE8378312B7FF444AE0B2904D8FFF7AD
:1043580005FB0021464A23E6464D4A4F0234002613
:1043680014F8012FA919303AD2B20A730B7BCDE9A0
:10437800026323780022CDE9006311463B460320FF
:1043880001360FF095FB0C2EEAD1FEF769FF384B8A
:1043980050221A701A229A70002401225C70DA7076
:1043A80003F8042F2A190134127B0C2C02F1300275
:1043B80003F8012FF6D10022502311460093032061
:1043C800314B0FF075FB00232B701A236B70012300
:1043D800AB70EB70284B1B78DBB22B72274B1B782A
:1043E800DBB26B72EC72FFF7C7FA1121B2E7412B0F
:1043F8007FF4EFAD4378432B7FF4EBAD16297FF4C0
:10440800E8AD224D421C002312F8011FE954013384
:10441800142BF9D1FEF778FE1D4B5B7D012B19D1CA
:1044280014490023EA5CC8180133D2B2142B80F86F
:104438002C20F7D1114B00221A701B78DBB24B727B
:10444800FFF79AFA0A4A631E15349C4206D1084AB5
:104458001621A5E5094B02221A70F3E713F8011F8C
:1044680002F8011BF1E700BFDEF7FFFF0C00002098
:10447800BD0D002078000020520E0020340C0020D2
:104488000C4E0108574E01087F4E01083E0E0020D1
:10449800A40A002070B5054686B00C4600293BD01A
:1044A80028480FF081FE2678EEB1002D48D06868C4
:1044B8002E78C0B1032E0BD00B2E2FD0022E12D186
:1044C800697801290FD00B060DD4FFF719FD0AE012
:1044D8006B78012B07D10078012802D0022800D080
:1044E80008B907F029F9237C052B15D894F90A2077
:1044F800059294F909200492134A52F82330039341
:1045080094F90830CDE901630022E368009311466D
:104518000E4B03200FF0CCFA06B070BD6B78012B60
:10452800E1D102780A4B02F001021A702AB9094B4C
:10453800114603200FF0BCFAD5E7074B0022F7E736
:104548002E46D0E7400D0020044F0108AD4E01086B
:10455800270D00209A4E0108A44E0108034B0022A3
:10456800C3E902220122C3E900227047540E002049
:1045780000487047540E00204FF0B04382B0DA6C08
:104588000243DA64DB6C03400193019B02B070477D
:104598002DE9F04186B000240220154D0594FFF75F
:1045A800EBFF0420FFF7E8FF124F03944FF48076E7
:1045B80001230DEB0001CDE9016328460323049391
:1045C8004FF4005803F0DEFE01A93846CDF8048008
:1045D80003F0D8FE22464146384603F0F9FF284644
:1045E8002246314603F0F4FF204606B0BDE8F081CC
:1045F8000004004800080048032810B50ED8012818
:1046080010D868B902460B484FF4807103F0E0FFF8
:10461800002209484FF4005103F0DAFF002010BDD2
:104628000122F0E7002203484FF4807103F0D0FF25
:104638000122EEE700040048000800480220704705
:10464800002070470120704700280CBF0F2016205B
:10465800704700000D48854602F0B0FE0C480D4931
:104668000D4A002302E0D458C4500433C4188C42C5
:10467800F9D30A4A0A4C002301E013600432A2422B
:10468800FBD30FF05DFFFDF7E7FFFEE70000012019
:1046980000000020BC080020305D0108BC08002094
:1046A800BC2C0020FEE74FF0B04382B0DA6C42F039
:1046B8000102DA64DB6C03F001030193019B02B091
:1046C8007047000030B587B0FFF7EDFF4FF4805119
:1046D80001224FF0904003F07BFF01224FF400616C
:1046E8004FF0904003F074FF4FF4C0551123CDE90B
:1046F800015301A901234FF09040039303F042FEB8
:1047080008240A2500224FF480514FF0904003F00E
:104718005FFF0120FEF7FAF901224FF480514FF0B4
:10472800904003F055FF0120FEF7F0F9013DE9D173
:104738004FF400614FF0904003F044FF08B9013C8A
:10474800DFD14FF400614FF0904003F03BFF68BBAE
:10475800FFF7A9FF04240123039001A92A48CDE902
:10476800014303F00FFE284C01220421204603F0E8
:104778002FFF2120FEF7CAF900220421204603F06A
:1047880027FF2120FEF7C2F901220421204603F069
:104798001FFF2120FEF7BAF920460022042103F06A
:1047A80017FF4FF42570FEF7B1F9DDE7FFF77BFF40
:1047B8004FF0B04300249A6D42F480029A659B6DD5
:1047C80003F4800300934FF4C052009B1223CDE9F9
:1047D80001230323CDE9034304230DEB03014FF029
:1047E8009040059303F0CEFD08480949094B8460C1
:1047F800C0E900130123C0E90334C0E90744446158
:1048080004F05AF807B030BD00040048640E0020D8
:10481800005800401A091020FFF754BF40B94B1E3A
:104828005A425A414FF400714FF0904003F0D0BE05
:10483800704708B50120FEF7E7FC6420FEF766F92B
:1048480000F0F0F9BDE808400120FEF7E2BC0000E6
:10485800054B1A6802805A689B684381034B0281A2
:1048680001221A70704700BFE40E00203D0E0020A0
:1048780030B585B0044600F017F810F0FF051FBFEB
:10488800EE232370AA2363706378029323780022AF
:10489800CDE900531146034B03200FF009F92846D0
:1048A80005B030BD1C4F01082DE9F04F0025484EDA
:1048B800484C356089B029462846FFF7AFFF29469E
:1048C8000120FFF7ABFF29460220FFF7A7FFDFF81B
:1048D8000881DFF80891424F94F8640152230121BE
:1048E8004FF0000A84F86031C4F868A1FFF796FF1A
:1048F8000320FEF70BF952468821204602F0C4FC3B
:104908000DF11E02C021204602F00CFD024650B1F6
:10491800344B5246114603200FF0CAF80021E8B282
:10492800FFF77CFF3DE0BDF81E304EF6AA618B42D2
:104938004AD14FEA450A0AF1540A5FFA8AFA059001
:104948005146204600F006FA834610B1264B059AD8
:10495800E0E70DF11E02C021204684F860A102F0B4
:10496800E1FC824610B1214B5A46D3E7204600F0BD
:10497800B5FB0246F0B93168012319443160396842
:10498800C4F86831AB400B433B60029394F8603144
:104998000193D4F8643100930146154B03200FF0BE
:1049A80087F80135032D04F5C87495D1306809B02E
:1049B800BDE8F08FBDF81E30009352464B461146B5
:1049C80003200FF075F8A9E700934346F7E700BF07
:1049D800DC0E0020BC000020F14F0108D64F010872
:1049E800D80E00203F4F0108514F0108744F0108AD
:1049F8008D4F01082DE9F04F4FF4804387B04FF4F5
:104A08009012CDE90232684CDFF8A0A1DFF8A0B11E
:104A180005464FF00A094FF00E0848F2E80700264D
:104A2800D4F86831002B00F0AE800022614B00966C
:104A3800114603200FF03CF8204600F043FE28B151
:104A480000225D4B114603200FF032F80DF11202DF
:104A58000DF11101204600F0EFFB28B1002253466A
:104A6800114603200FF024F80DF1130205A9204682
:104A780000F02DFF28B10022504B114603200FF003
:104A880017F80021204600F069F928B100224C4BA4
:104A9800114603200FF00CF801220021204600F0F7
:104AA80021FA28B10022474B114603200FF000F8E5
:104AB80001221146204600F015FA28B10022414B88
:104AC800114603200EF0F4FF022D65D83E4B33F853
:104AD800153002933D4B53F8253003933C4B53F864
:104AE80025703C4B13F805803B4B13F80590029A50
:104AF8000121204600F041FA28B10022374B114627
:104B080003200EF0D5FF039A0021204600F035FA65
:104B180028B10022314B114603200EF0C9FF394657
:104B2800204600F035F928B100222D4B114603200C
:104B38000EF0BEFF42460021204600F02BF928B1B6
:104B480000225B46114603200EF0B2FF4A460121BF
:104B5800204600F01FF928B100225B4611460320C9
:104B68000EF0A6FF0DF112020DF11101204600F022
:104B780063FB28B100225346114603200EF098FF2C
:104B88000123C4F87C310136032E04F5C8747FF480
:104B980047AF07B0BDE8F08F0022124B1146032043
:104BA8000EF086FFA3E700BFBC00002048500108B4
:104BB80041510108035001082D5001086E500108A9
:104BC80097500108B55001081C52010824520108E9
:104BD800305201083C5201083F520108E7500108D1
:104BE8000A510108D950010810B50B7E9BB9D0F8BD
:104BF8007C21098912B1C0E95E1310BD084BD0F8B9
:104C080078411A68C2F580734B4304FB02331B12C8
:104C1800C0F87831F1E70123C0F87C31EDE700BF37
:104C2800B80000202DE9F04FDFF80491414E87B01D
:104C3800FFF7F2FDD9F800300BB133684BB9FFF735
:104C480033FE002230603C4B0090114603200EF0EA
:104C58002FFF3368394D0024A3422C606C60AC6090
:104C68005BDDDFF8DC80374EDFF8DCA02046FFF79D
:104C7800C1FE88F80040D6F868B1BBF1010F35D104
:104C88000BFA04F304930A272F49304600F07AFC04
:104C9800C8B9059051463046FFF7A6FF9AF8183074
:104CA800059A002B3CD1D6F8783145F82430049A7F
:104CB800D9F800301343C9F8003098F8003043F0B1
:104CC800010388F800300120FDF720FF9AF818301A
:104CD8001BB1013F17F0FF07D6D1D6F8783140F65F
:104CE800C412002B08BF134645F8243005200134B0
:104CF800FDF70CFF032C06F5C876BCD198F80030F8
:104D08005BB12B686A68A9680093CDE9012100228C
:104D18000E4B114601200EF0CBFE07B0BDE8F08F18
:104D2800CDE9004B0A4B114602200EF0C1FECAE73E
:104D3800D80E0020E00E0020DD510108E40E00200E
:104D48003D0E0020BC000020BC0E00208E51010842
:104D5800FB5101084A088A2102F096BA152906D89B
:104D6800044BCB40DB0702D50174002070476FF07D
:104D7800070070470B00300010B50A460C460921A1
:104D880002F0A4FA18B9237803F00103237010BDC8
:104D980001F06BBE01F053BD01F04DBEF7B5002325
:104DA8000C46174601210DF1070206468DF807301B
:104DB80002F08CFA0546D8B9012F9DF8073026D1A4
:104DC800042C3AD8DFE804F003171A1D200043F03A
:104DD8001004A3420CD022460121304602F054FAB6
:104DE800054628B9716986F830413046FFF7D0FF8B
:104DF800284603B0F0BD43F02804EAE743F0040472
:104E0800E7E743F04004E4E743F08004E1E7042CDB
:104E180013D8DFE804F00306090C0F0003F0EF04D1
:104E2800D7E703F0D704D4E703F0FB04D1E703F096
:104E3800BF04CEE703F07F04CBE76FF00305D7E7A5
:104E480013B500230C460DF1070201218DF8073038
:104E580002F03CFA78B99DF80730C3F300122270CB
:104E6800C3F3C002A270C3F380026270C3F380125E
:104E7800DB09E270237102B010BD37B50D460DF1A4
:104E88000202F821044602F04DFA70B901AA042181
:104E9800204602F067FA40B9BDF802201AB1019B1A
:104EA800B3FBF2F32B602B68A36103B030BD037F23
:104EB8000B700020704737B50D460DF10602202112
:104EC800044602F02FFA28B9BDF8063023B9236A40
:104ED8002B60207703B030BDDB002B6023620123F9
:104EE8002377F7E70529F8B504460E46154635D861
:104EF80062B100EB810301215A6B0023701E042864
:104F080007D8DFE800F00E171A1D24001146012308
:104F1800F4E784F828103444E5B984F828500020D0
:104F280007E0C2F34F224421204602F0BDF90028D1
:104F3800F1D0F8BD84F82A10EDE784F82B10EAE7E1
:104F48005B00FE226021204602F0D5F9EFE71B0145
:104F5800EF22F7E7012384F82830E0E76FF0030039
:104F6800E7E7052996BF4018002390F8283013700A
:104F780094BF00206FF00300704770B543180446D3
:104F880093F828000E46154618B904EB810672639B
:104F980070BD05291BD8DFE801F0030912141616A5
:104FA800626304EB860400206563F1E7C2F34F22D5
:104FB8004421204602F078F90028E9D1F1E7E263BC
:104FC800EFE72264EDE7C2F34F226421F1E76FF0C7
:104FD8000300DDE737B50446154605292CD8DFE878
:104FE80001F0030717191B1B436B2B60002021E0FE
:104FF8000DF10602442102F095F9D8B9BDF8062052
:1050080053029AB12B60A363012384F8293011E07D
:10501800C36BEAE7036CE8E70DF10602642102F0CE
:1050280081F938B9BDF806305B02DEE7A36B2B6067
:1050380084F8290003B030BD6FF00300FAE737B5F4
:105048000D460DF107020121044602F03FF938B977
:105058009DF8073084F83031DB092B7084F84C3028
:1050680003B030BD2DE9F843037C0C4601F8083B3A
:105078000546FFF702FF40BB207304F110012846E4
:10508800FFF719FF08BB04F11401284600F021FCC2
:10509800D8B904F1240705F1270904F117080646D1
:1050A8003A46B1B22846FFF795FF70B9013619F8AC
:1050B800013F08F8013F062E07F10407F0D104F17B
:1050C8003C012846FFF7BBFF08B1BDE8F883211D66
:1050D8002846BDE8F84301F030BD0000F0B50022D5
:1050E800054693B0882102F0CFF84FF47A72A5F8FC
:1050F80052214FF4C872A5F854214C4AC5F85821DA
:1051080000234B4A85F8F030C5F8D4202B6202A959
:105118002846FFF7A7FF044670B9ADF8080002AEAD
:105128000FCE05F110070FC70FCE0FC70FCE0FC751
:1051380096E80F0087E80F003E4BC5F834314FF46E
:10514800FA730126A5F838314FF42063A5F83C31ED
:105158003246802185F85061284602F095F832469B
:105168000746FF21284602F08FF800221146074320
:10517800284602F089F83C4364B204430DF1070263
:105188009121284602F0A2F864B29DF8073085F80C
:105198003A31044332460021284602F075F864B2D9
:1051A80004430022FF21284602F06EF864B204434B
:1051B80000228021284602F067F864B2204340B2FA
:1051C800002488BBA1B2012228460134FFF78AFED9
:1051D800062CF6D140BB04466885024604212846C1
:1051E800FFF780FE00BB024605212846FFF77AFE3E
:1051F800D0B94FF490136B634FF4804201212846D5
:10520800FFF7BBFE80B94FF40C13FF22C5E90F303E
:1052180085F830210121284602F036F8012385F867
:10522800323108B985F8154113B0F0BD856B01001E
:10523800A470090064008403012300F079BD2DE9FE
:10524800F0428EB00C460C2304AA1421054602F045
:1052580005F8844600286CD19DF81A309DF81B602B
:105268009DF817209DF81810A07506EB03269DF8E9
:105278001630206002EB03229DF81930606003EBC2
:1052880001239BB25B029DF8121023619DF8133035
:10529800B5F8520103EB012392B252029BB2E260CD
:1052A800A382B0F57A7F9DF8101095F83171B6B2E7
:1052B8000AD0704300F5FA704FF47A76B0FBF6F036
:1052C8002E7F002E39D186B2002F40D0B001C0B257
:1052D800B608E0750DF10F002681CDE9004028469B
:1052E80001F086FE844620BB9DF80FE084F818E0A4
:1052F80005F150060FCE07AF0FC796E80700E37D0C
:1053080087E80700D4E90301A28AADF83020D4E980
:105318000149CDE90A01CDE9084907AC8DF83330D8
:105328008DF834E00FCC50350FC597E8070086E8B4
:10533800070060460EB0BDE8F0822E8C5E43B2EBEB
:10534800262F4FEA262C04D157B948F6E02600202C
:10535800BFE780B25043A2EB0C06B0FBF6F0B2E711
:1053680042F2B826B2E70000F7B517460E210DF154
:1053780006021D460B4C064601F0D4FFBDF8063068
:1053880004EA43433B6050B90DF106020C21304654
:1053980001F0C8FFBDF8063004EA43442C6003B0AE
:1053A800F0BD00BF0000FE1F73B590F8DA30013B76
:1053B800022B06460C4634D801AB6A460121FFF79A
:1053C800D3FF009BB3F57F0F054603D8019BB3F5C8
:1053D8007F0F23D915BB34B11349304602B0BDE85D
:1053E800704001F00FBC0422FF21304601F04CFF51
:1053F8002A4604467021304601F046FF2A460443F7
:10540800FF21304601F040FF64B204432A46802160
:10541800304601F039FF64B2044365B2284602B051
:1054280070BD0025FAE700BF5F06002037B50446C7
:1054380001228021057C01F027FF0122FF2120465F
:1054480001F022FF00221146204601F01DFF94F8CA
:105458003A219121204601F017FF01220021204620
:1054680001F012FF0022FF21204601F00DFF00226B
:105478008021204601F008FF012D29D0032D37D0C7
:10548800002D3CD101222946204601F0FDFE0123D2
:105498008DF80730A0B103B030BD01460DF1070209
:1054A800204601F013FF9DF80730DB0705F10105E1
:1054B80008D538B9B5F5FA6FEFD16FF00600EAE70D
:1054C8000546F0E7B5F5FA6F08BF6FF00600E2E7AA
:1054D80018B929462046FFF767FF02220021204617
:1054E80001F0D2FE0028D6D1042384F83231D2E765
:1054F80018B901212046FFF757FF0422EEE76FF0A5
:105508000700C8E738B5057C044625B1204600F0F9
:1055180054FD28B138BDFFF789FF0028F6D0F9E718
:10552800002DF7D1032384F83231F3E773B506462B
:10553800002501220B21304601F0A6FE0022044678
:105548000B21304601F0A0FE0DF1070204431321A0
:10555800304601F0BBFE9DF8073064B204430135C4
:105568005B0760B2EDB205D0032D08D00028E0D06B
:1055780002B070BD032D08BF6FF00B00F8E76FF0A5
:105588000B00F5E738B50023037404460D46FFF712
:10559800B9FF50B929462046FFF751FE28B9014600
:1055A8002046BDE83840FFF7C1BF38BD152970B5A2
:1055B800054616461C4667D10122FF2101F064FE0C
:1055C800002211460446284601F05EFE00220443EC
:1055D800FF21284601F058FE64B2044301228021CD
:1055E800284601F051FE64B2044302228521284670
:1055F80001F04AFE64B204430422FF21284601F068
:1056080043FE64B204430022CD21284601F03CFE4B
:1056180064B204431122CC21284601F035FE64B25D
:1056280004430722FF21284601F02EFE64B20443FA
:105638000022BE21284601F027FE64B20443062258
:10564800FF21284601F020FE64B204430922CC2140
:10565800284601F019FE64B204430022FF212846BF
:1056680001F012FE64B204430122FF21284601F032
:105678000BFE64B2002204431146284601F004FEE2
:1056880064B2204340B270BD042A17D80A2101F041
:10569800FBFD0028F7D1231E18BF01231B01EF22B1
:1056A8008421284601F027FE0028ECD185F8DA602D
:1056B80001462846BDE87040FFF738BF6FF00A0082
:1056C800E1E7000070B594B005464022002104A827
:1056D8000EF02EFF002301212846ADF806308DF884
:1056E80003308DF80430029300F0B8FC95F81421CB
:1056F80095F81311012A04D840F0AD80202940F212
:10570800AC8001AA02A9284600F02DFB0446002817
:1057180040F09E8095F85031002B40F0A280D5F8DB
:105728004C11284601F06EFA0446002840F090809B
:105738002346214604222846FFF738FF044600285E
:1057480040F086800122FF21284601F09DFD0DF1E1
:10575800060206468421284601F0E4FD2246064357
:10576800FF21284601F090FD76B2064374B2002C62
:105778006ED1BDF806301B01C5F8D43004A92846FF
:10578800FFF770FC0446002862D10DF1030128469A
:10579800FFF7F2FA044600285AD19DF8033085F83D
:1057A800313104AE0FCE05F110040FC40FCE0FC473
:1057B8000FCE0FC496E80F0084E80F000DF1030226
:1057C8000121284601F082FD0446002840D19DF8B9
:1057D800033085F83031024601462846FFF7DEFAE5
:1057E8000446A8BB024602212846FFF7D7FA04461A
:1057F80070BB0323014685F832310DF105022846B6
:1058080001F019F9044618BB9DF8053085F8E83011
:105818000DF105020121284601F00DF90446B8B939
:105828009DF8053085F8E03003AA0321284600F0EA
:1058380001FF044660B9039BC5F8E43003AA0421BC
:10584800284600F0F7FE044610B9039BC5F8DC3083
:10585800204614B070BD0C2951E7284600F010F915
:1058680054E701495DE700BF6C05002013B50C46FD
:105878000DF10702132101F029FD9DF8073013F0FF
:10588800180F03F0070218BF6FF00500226002B07E
:1058980010BD13B590F8DA30042B0C460BD101A9D2
:1058A800FFF7E4FF019B042B01D1012300E0002353
:1058B800237002B010BD01AA142101F007FD0028D1
:1058C800F7D19DF80430DB07EFD42070F1E700F042
:1058D8004ABA13B50C460DF10602282101F022FD43
:1058E80078B9BDF80620C2F30B0312F4006F18BF95
:1058F800A3F580534FF0FA0214BF13FB02F353438E
:10590800236002B010BDF0B54FEAD20C4FF0FF345F
:105918001C6002F00702664600278E4200D207B1DB
:10592800F0BD845D664503BF1441E4B215463D46AB
:1059380014F0010704D005EBC6051D600136ECE73D
:105948000135082D4FEA5404F2D1F7E7034B8009DB
:1059580053F82000003818BF0120704718080020AD
:1059680010B5B1EBD20F4FEAD20402F0070381BFA2
:1059780001229A40035D13438ABF03556FF031003B
:10598800002010BD0A460623B02101F049BC0A4692
:105998000623B02101F062BC2DE9F04F85B08046A6
:1059A800109E0E9D01968A4693461C464FF00009AC
:1059B800119B994508D10023129A1660F3B16FF034
:1059C800310005B0BDE8F08F01AB32462946584694
:1059D800FFF799FF019F7B1C0DD00F9BF818FFF76D
:1059E800B5FF504507D13A462046FFF7B9FF7E1C60
:1059F80009F10109DCE76FF03103DDE72146404694
:105A0800FFF7C0FF0028DCD102A94046FFF7BFFF1F
:105A18002544234602AAAB42D3D013F8014B12F80F
:105A2800011B8C42F7D0CAE770B5C02288B00E4679
:105A3800012190F83041054601F026FCF0B901A992
:105A48002846FFF79FFDC8B90122FF21284601F02B
:105A58001BFC98B93246B621284601F063FC68B9A8
:105A68000246FF21284601F00FFC38B922460121E1
:105A7800284601F009FC08B985F8304108B070BD26
:105A8800F0B50F4689B01646FF210122044601F001
:105A9800FBFB0246A8B94F21204601F0F5FB80B96F
:105AA8002C224E21204601F0EFFB024648B9FF2187
:105AB800204601F0E9FB20B9B422B621204601F0C6
:105AC800E3FB0025C4F82451A4F82851DEB9354673
:105AD80007ABB422CDE903730623CDE90032029562
:105AE80004F5927304F5957231462046FFF754FF8A
:105AF80030B9012384F8153184F8137184F81461DE
:105B080009B0F0BD013505F1B400FFF71FFF00280B
:105B1800DED12C2DF6D1DBE710B541F001020021D2
:105B2800044601F0B1FB78B9204600F046FA58B9AE
:105B380001462046FFF7FAFC30B9024601462046E6
:105B4800BDE8104001F0A0BB10BD2DE9F74F4FF0A4
:105B5800000B88461746FF21012205461E469DF880
:105B680038A09DF83C908DF807B001F08DFB5A469F
:105B780004465946284601F087FB5A460443FF214C
:105B8800284601F081FB64B2044364B2B8F1000F07
:105B980032D0BAF1000F06D00C9ACB21284601F07A
:105BA80095FB204344B2B9F1000F07D00DF107026D
:105BB800EE21284601F08AFB204344B20122FF214E
:105BC800284601F061FB012204430021284601F028
:105BD8005BFB64B204430022FF21284601F054FB1A
:105BE80064B29DF807300D9A204323F0100340B2A9
:105BF800137003B0BDE8F08FBAF1000F06D03A4633
:105C0800CB21284601F040FB204344B2B9F1000FF4
:105C1800D4D033468022EE21284601F06CFBCBE736
:105C28002DE9F04387B091460022054688468DF855
:105C380017201E461BB390F83071012211462846E2
:105C480001F022FB044658BB40212846FFF764FFB9
:105C5800044628BBB9F1010F13D10DF11703CDE9A3
:105C68000290CDE900830246034649462846FFF7DD
:105C78006CFF40B10446204607B0BDE8F0831F46DC
:105C8800DBE788F80000002EF5D03A4601212846C7
:105C980001F0FAFA04460028EDD185F83071EAE7F8
:105CA800002388F800302046E4E72DE9F043054654
:105CB80087B0884691461E4623B390F83071022279
:105CC8000121284601F0E0FA044660BB0146284657
:105CD800FFF722FF044630BBB9F1010F14D10DF1D3
:105CE8001703CDE90209009302460346CDF8048064
:105CF80049462846FFF729FF40B10446204607B029
:105D0800BDE8F0831F46DAE788F80000002EF5D0DA
:105D18003A460121284601F0B7FA04460028EDD199
:105D280085F83071EAE7002388F800302046E4E778
:105D3800F8B51D46164600232A4690F830710446E9
:105D4800FFF76EFF70B903462A4631462046FFF733
:105D5800ACFF38B93A460121204601F095FA08B956
:105D680084F83071F8BD2DE9F04F002393B0CDE9E8
:105D78000A12C0F82431A0F828310122FF21CDE908
:105D88000E33B0F83C818DF8343005468DF8353047
:105D980001F07AFA0446002840F0E38002464F21D9
:105DA800284601F071FA0446002840F0DA802C22D7
:105DB8004E21284601F068FA0446002840F0D180B8
:105DC8000246FF21284601F05FFA0446002840F009
:105DD800C880B422B621284601F056FA04460028A5
:105DE80040F0BF8002468021284601F04DFA044663
:105DF800002840F0B68003460DF135020DA928466B
:105E0800FFF796FF0446002840F0AB800323CDE956
:105E18000203B421062305F5957A05F592790EAEAD
:105E2800CDE90031049601464B4652462846FFF715
:105E3800B3FD0446002840F094800DF13601284651
:105E48000E9FFFF7F1FD0446002840F08A80BDF858
:105E58003630434540F2AA80C5F82401A5F8280148
:105E680007F1B400FFF772FD08B92B2F7DD906237F
:105E7800B4224FF0030BCDE90032CDE9027B049642
:105E88004B46524601212846FFF786FD002840F080
:105E98008B800DF1360128460E9FFFF7C5FD06469B
:105EA80000287CD1BDF83630434540F28280012677
:105EB8000696BDF83630434560D2A3EB080383EA63
:105EC800E372A2EBE3729DF81860099205F59273EC
:105ED8004FF0030B0793079B18689B881090ADF849
:105EE80044303A460FAB06215046FFF70CFD0F9F92
:105EF8007B1C56D007F1B400FFF728FD069B98429B
:105F08003CD10BF101033A4648460893FFF728FDB8
:105F1800002849D149462846FFF734FD002843D1D7
:105F28000DF136012846FFF77FFD00283CD1BDF86A
:105F38003620A2EB0803002BB8BF5B42424516D9B6
:105F4800099A934218D910A92846FFF71BFD079A0A
:105F58000799034610981060BDF844208A806BB1F9
:105F68001C46204613B0BDE8F08F013778E7DDF80E
:105F780020B009930137AEE7DDF820B00A9BC3F8DB
:105F880000B00B9B1E70012385F815310A9B1B6816
:105F980085F813310B9B1B7885F81431E1E704462B
:105FA800DFE76FF03104DCE70446DAE70026B346A2
:105FB8007EE70123834606937BE737B50023044633
:105FC8008DF807304FF4FA650DF107012046FFF709
:105FD80060FC58B99DF80730012B07D0013D03D06C
:105FE800204601F0E5F9EFE76FF0060003B030BD99
:105FF80002464FF08043934202D8002013B97047FD
:106008009B08F8E7C11891424FEA50009CBFC0189E
:10601800521A9B08F2E773B500228321054601F066
:1060280033F9044688B94FF4FA660DF10702832163
:10603800284601F04BF99DF807300343DBB20446CC
:106048001BB9013EF1D16FF00604012283212846D5
:1060580001F01AF9204340B202B070BD2DE9F04FAB
:1060680090F8F06091B04FF00009072ECDE907993C
:1060780004460F4600F0A2820122802101F004F9B3
:1060880001228046FF21204601F0FEF84A4648EAF0
:1060980000084946204601F0F7F84FFA88F848EA20
:1060A80000080622FF21204601F0EEF84FFA88F892
:1060B80048EA00080DF115028321204601F006F98F
:1060C8009DF815204FFA88F848EA000842F00402C3
:1060D8008321204601F0D8F84FFA88F848EA0008EA
:1060E8000722FF21204601F0CFF84FFA88F8012255
:1060F800812148EA0008204601F0C6F84FFA88F8DE
:1061080048EA0008204601F053F94FFA88F848EAAF
:10611800000801228021204601F0B6F84FFA88F8DD
:1061280048EA000517F0010B6DB200F01E82F20775
:1061380000F11E826B229421204601F0A5F88046CA
:106148002046FFF768FF06AA48EA00089021204683
:1061580001F008F945EA0805069B6DB2242294214E
:1061680005432046C3F3062AC3F3C03901F08CF86F
:106178006DB205432046FFF74EFF6DB2054306AAF0
:106188009021204601F0EEF8069B6DB21BBA25223D
:10619800942105432046099301F076F86DB2054332
:1061A8002046FFF738FF6DB2054306AA9021204626
:1061B80001F0D8F8069B6DB21A0E05431B0C6DB2A0
:1061C8008DF828208DF8293017F00203029300F08B
:1061D800DB8016F0020840F0D78002229421204686
:1061E80001F052F801902046FFF715FF019B0DF1D1
:1061F80016020343902120461D4301F067F86DB253
:106208007B2294210543204601F03EF86DB20543F8
:106218002046FFF700FF6DB205430DF117029021EC
:10622800204601F053F86DB27722942105432046A9
:1062380001F02AF86DB205432046FFF7ECFE6DB277
:10624800054306AA9021204601F08CF8069B5A0EB9
:106258008DF82C20C3F386428DF82D20C3F3C62277
:106268008DF82E206DB2C3F30612DB0003F078031D
:10627800942105438DF82F20204678228DF815307B
:1062880001F002F86DB205432046FFF7C4FE6DB277
:10629800054306AA9021204601F064F8069B9DF864
:1062A800152002EB53728DF83020C3F386528DF817
:1062B8003120C3F3C6328DF83220C3F306228DF89D
:1062C80033206DB2C3F346029B0103F040039421CF
:1062D80005438DF83420204679228DF8153000F0DA
:1062E800D3FF6DB205432046FFF795FE6DB2054317
:1062F80006AA9021204601F035F8069B9DF8152046
:1063080002EB93628DF83520C3F3C6428DF8362030
:10631800C3F306328DF837206DB2C3F346129B00E3
:1063280003F07C03942105438DF8382020467A2217
:106338008DF8153000F0A8FF6DB205432046FFF731
:106348006AFE6DB2054306AA9021204601F00AF8BC
:10635800069B9DF815208DF83E8002EB93728DF810
:106368003920C3F3C6526DB28DF83A20C3F3064202
:1063780005438DF83B20C3F34622C3F386036DB271
:106388008DF83C208DF83D3017F00403019300F0A0
:10639800F180730700F1EE807B229421204600F003
:1063A80073FF80462046FFF736FE07AA48EA000832
:1063B8009021204600F0D6FF45EA08084FFA88F8F1
:1063C80048EA00057C229421204600F05DFF6DB26A
:1063D80005432046FFF71FFE6DB2054308AA90212A
:1063E800204600F0BFFF6DB273229421054320467A
:1063F80000F04AFF6DB205432046FFF70CFE6DB270
:10640800054306AA9021204600F0ACFF069B6DB21A
:106418001B0274229421054320461FFA83F800F0DA
:1064280033FF6DB205432046FFF7F5FD6DB2054316
:1064380006AA9021204600F095FF6DB29DF81B300A
:10644800752294210543204643EA080800F01CFF02
:106458006DB205432046FFF7DEFD6DB2054306AA7F
:106468009021204600F07EFF069B6DB21B029BB276
:106478007622942105432046039300F005FF6DB270
:1064880005432046FFF7C7FD6DB2054306AA9021D4
:10649800204600F067FF6DB29DF81B20039B054363
:1064A8006DB21343002281212046039300F0ECFED5
:1064B80006220543FF21204600F0E6FE6DB20543A3
:1064C8000DF115028321204600F000FF9DF81520EC
:1064D8006DB2054302F0FB028321204600F0D4FE92
:1064E8006DB205430122FF21204600F0CDFE6DB2BA
:1064F800054301220021204600F0C6FE6DB2054387
:106508000022FF21204600F0BFFE6DB205430022A5
:106518008021204600F0B8FE6DB205436DB2039BA2
:10652800FDB9BBF1000F29D1029AAABB019AAAB101
:10653800720713D4079AC4F81821089AC4F81C21C2
:106548004FEA4822C4F820213BB1A3F5C8534FF4C1
:106558007A7253431B095B421BB2E3603E4384F8E3
:10656800F060284611B0BDE8F08FD946DA462BE630
:10657800CA4629E64FF00008434693E7F007D3D40C
:106588000998BDF8282084F813A184F81491C4F858
:106598002A01A4F82E21C7E7B107C7D49DF8162011
:1065A80084F8F1209DF8172084F8F2200BA904F153
:1065B800F30002930DF0E8FF029BB7E74D46D0E7E2
:1065C80050B10138002330F0FF019AB203F1010302
:1065D80003D100EB022080B270474008F3E7C3B252
:1065E800000A03FA00F0013070470000084B5A43D4
:1065F8004FF47A7302F5FA724FF4FA60B2FBF0F0D6
:10660800B2FBF3F203FB0100B0FBF2F0704700BFEE
:10661800002F3A00064B5A434FF47A7002F5FA728B
:10662800B2FBF0F24A4302F5FA72B2FBF0F070479F
:10663800002F3A002DE9FF4102294FF000050746D7
:1066480016468DF80350ADF804501CD80DF102021F
:106658002946FEF7A1FB044630B90DF10302462195
:10666800384600F033FE04469DF80300FFF7B7FFF5
:1066780081B29DF802203846FFF7CCFF30602046F3
:1066880004B0BDE8F081032918D10DF102022946B2
:10669800FEF782FB0446002846D101460DF10202AE
:1066A8003846FEF779FB044628B901AA5121384635
:1066B80000F038FE0446BDF80400D7E7042935D1B8
:1066C80002A9FEF7BDFB9DF80B30ABB10DF102023C
:1066D80029463846FEF760FB044658B901AA5121FD
:1066E800384600F01FFE0446BDF80400FFF777FFA8
:1066F80085B214B1002015E01D460DF102020121FA
:106708003846FEF749FB04460028F3D10DF106028E
:106718007121384600F006FE0446BDF80600FFF772
:106728005EFF80B2401BA3E72846A7E728462C4611
:10673800A4E7F0B5022985B0054616461ED80DF126
:1067480005020021FEF728FB0446A0B99DF80520A4
:1067580031462846FFF74AFF83B2B3F5807F9ABFD8
:1067680000F1FF32D2B2FF22A5F8D82046212846F0
:1067780000F08AFD0446204605B0F0BD03291FD16C
:106788000DF105020021FEF707FB9DF805203146B3
:1067980004462846FFF72AFF80B2FFF711FF02469A
:1067A800ADF80600A5F8D800002CE4D15121284600
:1067B80000F07AFD04460028DDD1C5F8E460DAE788
:1067C800042939D102A9FEF73BFB9DF80B70B7B13C
:1067D8000DF1050200212846FEF7DEFA04460028DE
:1067E800C9D10DF106025121284600F09BFD04464F
:1067F800BDF80600FFF7F3FE87B2002CBBD10DF100
:10680800050201212846FEF7C7FA04460028B2D13E
:106818009DF8052031462846FFF7E8FE3844FFF783
:10682800CFFE71210246284600F03EFD04460028AE
:10683800A1D1C5F8DC609EE76FF003049BE7F0B5D3
:1068480085B000238DF80330D30705460F4616465A
:1068580005D439B9A2F10C03DAB2062A11D96FF0BE
:106868000300E6E0012921D1A2F10803DAB2062AE1
:10687800F5D8062B1AD8DFE803F03B1969198A19ED
:106888009D00062B12D8DFE803F004112D112F11FB
:10689800310018225721284600F0F6FC082256211C
:1068A800284600F0F1FC002840F0C3807408013C41
:1068B800E4B2002F00F09180012FD0D101AA042169
:1068C8002846FFF7B7FE50B922467021284600F047
:1068D800DBFC20B9019A04212846FFF72AFF85F836
:1068E800E06099E03022D5E74022D3E75022D1E793
:1068F8001022482100F0C8FC08224721284600F051
:10690800C3FC022204463221284600F0BDFC0C22BA
:1069180004433021284600F0B7FC64B20443012246
:10692800FF21284600F0B0FC64B2044364B2302270
:106938003021284600F0A8FC00220443FF21284605
:1069480000F0A2FC64B2204340B2ACE72822482100
:1069580000F09AFC08224721284600F095FC032203
:1069680004463221284600F08FFC044364B2092211
:106978003021284600F088FC01220443FF212846E4
:1069880000F082FC64B2044364B22022D0E73822CB
:10699800482100F079FC08224721284600F074FCC1
:1069A800032204463221284600F06EFC044364B2F8
:1069B8000822DDE74822114600F066FC082247213C
:1069C800284600F061FC032204463221284600F0E4
:1069D8005BFC044364B20722CAE702AA03212846E3
:1069E800FFF728FEB0B903AA02212846FFF722FEC6
:1069F80080B922465021284600F046FC50B9029A38
:106A080003212846FFF795FE20B9039A022128465C
:106A1800FFF78FFE85F8E86058B969692846FEF7E0
:106A2800B7F930B9024601230DF103012846FFF7F3
:106A38003CF905B0F0BD13B5144629B1012910D0B1
:106A48006FF0030002B010BD0DF10702502100F0F5
:106A58003DFC0028F6D19DF8073001335B00237018
:106A6800F0E70DF107027021F1E7F0B5002385B0DA
:106A78004FF4FA62CDE9002344F61F6399420646B3
:106A88000F4604D86FF00305284605B0F0BD02A9EB
:106A9800FEF7D6F905460028F6D19DF809209DF89D
:106AA800083013439DF80A201343A7F636341BD049
:106AB8006A4602213046FFF7BDFD00283BD19DF80C
:106AC80008302BB1009B03F24E239C42DAD9E41A1A
:106AD8009DF80A3023B3009B03F2B223B4EB430FB3
:106AE8004FEA4302CED9A41A9DF80B305BB101AA34
:106AF80003213046FFF79EFD019B03F52573A34252
:106B0800C0D2C0B9E41A9DF80C30002BBCD0A4F256
:106B1800262204213046FFF70CFE77610546B3E7CD
:106B28009DF80930002BDFD0009B03F525739C42AC
:106B3800A8D9E41AD8E70546A6E770B54FF4FA6273
:106B480086B00023CDE9022340F636330B600C46AD
:106B580004A90646FEF774F90546002836D19DF8C3
:106B680011209DF8103013439DF81220134319D0BB
:106B780002AA02213046FFF75DFD002840D19DF8AA
:106B880010302BB1029B03F24E222368134423607A
:106B98009DF81230EBB1029B03F2B222236803EB9B
:106BA800420323609DF81330EBB99DF814305BB1B4
:106BB80001AA04213046FFF73DFD019B03F226227E
:106BC800236813442360D8B923687361284606B044
:106BD80070BD9DF81130002BE4D0029B03F525729F
:106BE80023681344DDE703AA03213046FFF722FD9B
:106BF800039B03F525722368134423600028D4D02F
:106C08000546E3E72DE9F743002406460D462046EE
:106C180015F80480B8F1000F00D010B103B0BDE83A
:106C2800F083671CB8F1FF0F15F8079029D1A71C4E
:106C3800EB5DB9F1030F36D8DFE809F0020B131B3F
:106C4800271D2C44E27802EB0323A6F834313C4696
:106C5800DEE7271D2C44E27802EB0323A6F8363141
:106C6800F5E7271D2C44E27802EB0323A6F8383118
:106C7800EDE7271D2C44E27802EB0323A6F83C310C
:106C8800E5E7B8F1040F0ED802344246291901A8E5
:106C98000DF087FC434601AA4946304604EB080735
:106CA80000F0BEFAD3E76FF00300D0E773B5002316
:106CB8000E4613600DF1070105461446FEF7F7F876
:106CC80040B99DF807302BB1B38A2A6A5343803301
:106CD8001B0A236002B070BD13B5CB68136014465D
:106CE80001AAFFF7E3FF18B92368019A1344236048
:106CF80002B010BDF8B5B0F85451D0F85801684347
:106D08008030000A0E464543DDE90717144652B1A4
:106D1800B60206EB5202B2FBF4F202EB4202524315
:106D280002F50042140C069A534301F50042120C76
:106D380006200332B2FBF0F2C2EBC202B2F5803F8A
:106D480038BF033103F500433EBFB1FBF0F1C1EB9F
:106D5800C10101F500414FEA134334BF090C1B4937
:106D680003FB03F338BF494303EB57030B44B3FB5F
:106D7800F7F39B03FE2205F120007F33B3FBF2F308
:106D88005C434FF47A7704F5FA748009B4FBF7F49E
:106D98002401FFF72DF904F5FA74BC4228BF4FF41B
:106DA800FA63064629BFB4FBF3F300205B19B4FB72
:106DB800F7F428BFB3FBF4F0FFF71AF9099B8642F2
:106DC80094BF1E6018600020F8BD00BF0000F0FFEF
:106DD8002DE9F04F91B0CDE90723036A0E930B69B3
:106DE80009930546CB680B930F460FAAFFF774FF6C
:106DF8000EAA39462846FFF759FF58BB0F9C95F84D
:106E0800E0B0D5F8DC3005934FF47A7606FB04F150
:106E180001F5004104910E990A910499D5F8E430DE
:106E28000693BBF1080F04F180040CBF022303236F
:106E380024F0FF0A090C95F8E820DFF8A081CDF8C6
:106E48003CA00C9109D1079BC3F80080089BC5F8AA
:106E58004081186011B0BDE8F08F06990D9328465F
:106E6800FFF7C4FB5A46059981462846FFF7BEFB43
:106E78000D9B5B490C9A814403FB09F94FEAC92928
:106E880040F2776309F5FA79240AB9FBF6F903FBAE
:106E980009F909F5FA79B9FBF6F909FB04F404F1E3
:106EA8008003099C74430C40B4FBF2F44D4A1B0A5E
:106EB800944228BF1446012B38BF01230C204FF4FD
:106EC800167258435443FFF793F83B7E3A894FEACA
:106ED800400B002B7FD14249049B0B4003F5FA710C
:106EE800414B5A4341F25C23B2FBF3F20A9B7343D2
:106EF800B3F5481F28BF4FF44813A1EB4303B1FB78
:106F0800F6F1B3FBF6F31B02B3FBF1F63602C6F556
:106F18008036564306F50046360C06F58036760868
:106F28007643B60B4FF44870704304F5004300F500
:106F380000401B0C5B43000C00FB0030FFF758F8C7
:106F480003046422323341F28837B3FBF2F340F68C
:106F5800B532B3FBFBF302FB0377244B9F429CBF84
:106F680042F21073B7FBF3F7DDE90532134403F57A
:106F7800FA734FF47A7B4FF4FA62B3FBFBF0B3FB7E
:106F8800F2F202F5C812B2FBF0F088BF4FF4704776
:106F9800FFF72EF8000200F5FA70B0FBFBF0404353
:106FA80007FB0700FFF724F80BFB00F0079B0B9A81
:106FB800404528BF40461860089BC5F84001CDE908
:106FC80002934FF448730093019433465146284680
:106FD800FFF790FE3EE74FF48036A3E7AE878F02B7
:106FE8000000FFFF666666009A9906000F279F2437
:106FF8002DE9F04F8BB0002711F0780FDDE914B8B8
:107008000446019299468DF80E708DF80F708DF830
:1070180010708DF81170ADF812700997C1F3C30A9A
:1070280000F0AF80AAF10503DBB20A2B01D86B4A46
:10703800D75C0DF10E0200212046FDF792FF9DF866
:107048000E500646D5B1002840F09D8009AB05AA30
:1070580059462046FFF7BCFE002840F09680099B61
:10706800ABF80A30014606AA2046FDF7B3FF069D95
:1070780025B1059B9D422CBF0025012520B904AAF6
:1070880002212046FDF76DFF9DF8106026B3002809
:107098007DD107AA02212046FDF79CFF88B901226D
:1070A800FF21204600F0F0F858B90DF11202B62180
:1070B800204600F037F920B90246FF21204600F0AB
:1070C800E3F8BDF81230079E5B02C4F848311EB1E0
:1070D8009E422CBF0026012628B90DF1110203217A
:1070E8002046FDF73EFF9DF8113093B1002873D17B
:1070F800B9F1000F03D0019B1B02B3FBF9F908AAF1
:1071080003212046FDF766FF089B4B4594BF0023EB
:10711800012320B9012F3CD1FF2288F8002098F8DC
:1071280000200AB9ABF80A200DF10F020121204610
:107138000193FDF716FF08BB9DF80E20019B002A5E
:1071480008BF0125BAF1040F18BF9DF80F2084F875
:107158002E501ABFB2FA82F25209012284F82F2067
:107168009DF81020002A9DF8112008BF0126002A4A
:1071780008BF012384F8306084F831300BB0BDE8D3
:10718800F08F012755E700257EE735467CE7002686
:10719800A9E70AF1FF32092A0AD8DFE802F0050553
:1071A80005090907090B070B0522B6E70422B4E70E
:1071B800012E01D10322B0E7BAF1040F01D0012B4F
:1071C80001D10222A9E7012D1BBF002388F8003056
:1071D80088F800502B46A2E70023A0E74252010896
:1071E80007B502F10A03009393B20A4690F86011BA
:1071F800D0F85C0101F0B2FB03B05DF804FB13B5F5
:1072080002F10A0390F860410093D0F85C0193B250
:107218000A4644F0010101F037FC02B010BD00003D
:107228003F2BF8B50E46054611461C4611D80A4FA5
:1072380038461A4600F8016B0DF0B3F9621C39465E
:107248002846FFF7CDFF00280CBF00206FF0130081
:10725800F8BD6FF00300FBE7F00E002073B515468C
:107268008DF8071001220DF1070104461E46FFF7AD
:10727800B7FF28B9324629462046FFF7C0FF08B1B4
:107288006FF0130002B070BD08B5064B19705A7044
:1072980019460222FFF7A4FF002814BF6FF013005D
:1072A800002008BDF00E002008B5074B1970110A20
:1072B80059709A7019460322FFF792FF002814BFED
:1072C8006FF01300002008BDF00E002037B51546FA
:1072D8008DF8071001220DF107010446FFF780FF22
:1072E80028B9012229462046FFF789FF08B16FF027
:1072F800130003B030BDF7B515460DF10702064679
:107308000F461C46FFF7E2FF50B99DF807301D40B5
:1073180044EA0502394630468DF80720FFF7B4FFE6
:1073280003B0F0BD73B514468DF8071001220DF1B6
:1073380007010646FFF754FF18B16FF0130002B0BB
:1073480070BD074D022229463046FFF758FF002836
:10735800F3D12A786B7803EB02232380EFE700BF91
:10736800F00E002073B514468DF8071001220DF1B8
:1073780007010646FFF734FF18B16FF0130002B09B
:1073880070BD0A4D042229463046FFF738FF002811
:10739800F3D16B782A781B0403EB0263EA78134471
:1073A800AA7803EB02232360E9E700BFF00E002070
:1073B80008B50220FBF7AAFB002008BD70470000B3
:1073C80010B5032000F072FC01F0AAFD064B18600E
:1073D8000F20FBF791FB044618B9FBF7F4F9204698
:1073E80010BD0124FBE700BF280800204FF0E02271
:1073F800136923F00203136170474FF0E022136909
:1074080043F0020313617047014BD3F890057047AE
:107418000070FF1F014BD3F8940570470070FF1FE1
:10742800014BD3F8980570470070FF1F024A536854
:1074380023F0010353607047002004E0024A5368B8
:1074480023F0020353607047002004E0024A5368A7
:1074580023F0040353607047002004E08068C0F301
:1074680080007047F7B5002301930446002800F018
:10747800E980856D25B9FAF7F1FCE56584F8545083
:1074880023689A68D00040F1A1809A68D10000F181
:10749800B480A26D42F01002A265E26D42F00102D2
:1074A800E26501251846FFF7D9FFA26D02F0100228
:1074B800024340F0C980A26D206922F4817242F033
:1074C8000202A2659A68D2075DD4226BA67E94F860
:1074D8002CC0003A18BF01221703D4E902120A434C
:1074E800217E42EA8132617E42EAC13242EA463274
:1074F800002842EA4C02B4BF20F000414FF40011CA
:107508003A430A4394F82010012903D1002E76D17A
:1075180042F48032616A21B1A66A01F4E071314314
:107528000A43D968E66C21F4FE3121F4FF71114356
:10753800D96094F83C206168012A01F0404C4CEA7B
:10754800060609D1D4E910273A433243A66C3243E0
:1075580042EA0C0242F001061F693E4A3A403243B1
:107568001A6121F00042B2F1804F0CD0B1F1004F06
:1075780009D0394ED6F8082701F4701122F4701298
:107588000A43C6F808275A69666BA16B22F00702FE
:1075980032435A615A6922F0700242EA01125A6172
:1075A800002835D19A6A62F00F029A625B6903F08B
:1075B80007039E423CD10023E365A36D23F0030338
:1075C80043F00103A365284603B0F0BD9A68234938
:1075D80022F0104222F0170242F080529A60204AAC
:1075E8001268B2FBF1F2013252000192019A002AAC
:1075F8003FF44BAF019A013AF7E7002552E7A16D36
:1076080041F02001A165E16D41F00101E16581E7EB
:10761800B0F5001FCAD19A6AE269013A92006FF088
:107628000F0102F01C0201FA02F2216E0A43BCE7C4
:10763800A36D23F0120343F01003A365E36D43F039
:107648000103E3650125BEE7A36D43F01003A365BD
:10765800F8E700BF02FCFF1F00200140400D0300B7
:1076680028080020F8B54569082D04460E460AD0BA
:107678000368DB68D80705D5A36D43F02003A3652D
:107688000120F8BD0425FBF739FA074623681A6874
:107698002A4221D0A26D42F40072A265DA6812F47F
:1076A800406F14D1A27E92B91A6812070FD51846F6
:1076B800FFF7D4FE28BB5A6822F00C025A60A26D6C
:1076C80022F4807222F0010242F00102A265207EBB
:1076D80000BB0C221A60D4E7711CD8D0FBF70EFA55
:1076E800C01BB04201D8002ED0D123681B682B40A4
:1076F800CCD1A26D84F8543042F00402A265032074
:10770800BFE7A26D42F02002A265E26D42F00102DD
:10771800E265DCE70020B4E70368186C70470000F6
:10772800F7B50023019390F85430012B044600F07C
:10773800C58005680669012380F854302846FFF79C
:107748008DFE002840F0B480D1E90020022826F000
:10775800040300F08280B3F1004FC2F3110E13D17D
:10776800AB6A43EA0E03AB628B68686903EA0223DB
:1077780023F07C4323F0FF0320EA02210B43002A75
:107788006B6126DB002055E0236E00F01F074FF0E9
:107798000F0C0CFA07FC6FEA0C0623EA0C0CBEF17E
:1077A800000F11D1C2F38463BB4043EA0C03236684
:1077B8008008E36901309842D6D8A86AC2F3836387
:1077C800BB4006403343CEE792FAA2F3B3FA83F301
:1077D800EAE73B493B48D1F80837824203F0E075B5
:1077E80019D11B02CED4D1F8083723F0E0732B430C
:1077F80043F40003C1F80837334B1A68334BB2FB24
:10780800F3F20C2302FB03330193019B002BB9D045
:10781800019B013BF8E72E48824210D113F080709B
:10782800B0D1D1F8083723F0E0732B4343F08073CD
:10783800C1F80837002384F8543003B0F0BD254858
:1078480082429FD113F480009CD1D1F8083723F0ED
:10785800E0732B4343F48003EAE7B3F1004F01BF21
:10786800AB6AC2F311018B43AB62002A8ADA15486E
:1078780013498242D1F8083709D1D1F8082703F013
:10788800A07322F0E0721343C1F808377AE7104872
:10789800824204D1D1F8082703F44003F1E70D48E8
:1078A80082427FF46FAFD1F8082703F0C073E8E78E
:1078B800A26D42F02002A2651846BBE70220BCE791
:1078C80000200140001000B028080020400D0300EF
:1078D800004000B8002000B4026838B504461046DD
:1078E800FFF7BCFD08B9002038BD9368990707D495
:1078F800936823F0004323F0170343F010039360C9
:10790800FBF7FCF8054623689B685B07EBD5FBF79C
:10791800F5F8401B0228F6D923689B685A07F2D568
:10792800A36D43F01003A365E36D43F00103E36522
:107938000120D9E773B50023026801939368DD0736
:10794800044602D5002002B070BD9168214B19424F
:1079580009D0A36D43F01003A365E36D43F0010361
:10796800E3650120EFE7936823F0004323F0170352
:1079780043F001039360184BD3F8083718021CD45E
:10798800637E012BDED0FBF7B9F8144E054622685A
:107998001368DB07D6D49368D9075FBF9368334071
:1079A80043F001039360FBF7A9F8401B0228EED9C6
:1079B80023681B68DA07EAD4CBE7094B094A1B6836
:1079C800B3FBF2F301330193019B002BD8D0019B49
:1079D800013BF8E71700008000200140E8FFFF7F27
:1079E80028080020400D030038B504460068FFF75A
:1079F80035FD054620BB94F85430012B20D00123D7
:107A080084F854302046FFF795FFB0B9A36D22687B
:107A180023F4706323F0010343F48073A3651C23EC
:107A2800E065136084F85400936823F0004323F062
:107A3800170343F00403936038BD84F85450FBE700
:107A48000220F9E7026838B5936891680446C807C8
:107A580001D4002038BD9907FBD4936803F00503CF
:107A6800012B19D1936823F0004323F0170343F047
:107A78000203936003231360FBF740F8054623686D
:107A88009B68DB07E5D5FBF739F8401B0228F6D9D8
:107A980023689B68DA07F2D5A36D43F01003A3654A
:107AA800E36D43F00103E3650120D3E770B50446B5
:107AB80000284BD0836D43F002038365FFF70CFF6A
:107AC800054668B92046FFF7BDFF054608B90123FA
:107AD800A3652268936823F0104323F0170393608B
:107AE80023685A6822F4677222F003025A6040F24F
:107AF8009F321A60D968164A0A40DA601A6922F079
:107B080040421A615A6922F007025A611A6A02F061
:107B1800F0221A625A6A02F0F0225A62DA6A02F015
:107B2800F022DA629A6A0B4A00269E62D2F8083777
:107B380023F0FE73C2F808372046FAF7A3F9E66582
:107B48002666A66584F85460284670BD0125FBE7C3
:107B580000023E830020014010B590F85430012BFC
:107B6800044615D0012380F85430FFF7B5FE58B904
:107B78002046FFF767FF38B9A36D23F4807323F01D
:107B8800010343F00103A365002384F8543010BDBA
:107B98000220FCE7F7B50023019390F85430012B3D
:107BA80004467FD0012380F85430FFF74BFF236849
:107BB8009A6812F00102054607D0A36D43F010033E
:107BC800A365002384F854302DE0A16D364F21F4CD
:107BD800817141F00201A165DE68D96826F4FF468B
:107BE80026F07C0621F40041360421F00301360C0E
:107BF800D96008209968394041F000419960996836
:107C0800002913DA0199013101910199B1F52E3F4B
:107C1800F5D3A36D23F0120343F01003A3650023EB
:107C280084F854300125284603B0F0BDD3F8B410C9
:107C3800013801F07F010A44DCD199681A480140F3
:107C480041F001019960D3F8B41021F07F0141EAB5
:107C5800D202C3F8B4209A68024042F002029A6045
:107C6800FAF74CFF074623689A68D20708D4DA68FF
:107C78003243DA60A36D23F0030343F001039FE767
:107C8800FAF73CFFC01B0228EDD923689B68D90787
:107C9800E9D5A36D43F01003A365E36D43F0010339
:107CA800E365BFE70225BEE7E8FFFF7F0749CA682B
:107CB80022F4E0620302120403F4E063120C13439B
:107CC80043F0BF6343F40033CB60704700ED00E03E
:107CD800164B30B5DC68C4F30224C4F10703251D34
:107CE800042B28BF0423062D4FF0FF358CBF033C1F
:107CF800002405FA03F321EA0303A54022EA05025A
:107D0800A340002843EA0203ACBF00F16040084AE0
:107D18004FEA0313B8BF00F00F00DBB2AABF00F5AB
:107D28006140135480F8003330BD00BF00ED00E01F
:107D380014ED00E0002807DB044A4109012300F0A4
:107D48001F00834042F82130704700BF00E100E087
:107D580000280CDB4309064900F01F0020330122EC
:107D6800824041F82320BFF34F8FBFF36F8F7047D6
:107D780000E100E070B5D0E913456560446D14B1C9
:107D8800D0E916456560D0E9105404F01C060124BA
:107D9800B4406C60046863608368102B0BBFA260FA
:107DA800A160E160E26070BD0268416CD3B210B5B9
:107DB800083B1424B3FBF4F30B4CA24288BF0B4AD4
:107DC80021F0030199BF01F1804202F502325218F5
:107DD80007338264064AC26403F01F03012202FAD1
:107DE80003F3036510BD00BF070402401C080240EE
:107DF8008008024038B500285ED002682F4B9A42AE
:107E08004FF014014CD82E4B1344B3FBF1F32D491A
:107E18009B00C0E91013022380F825301368056918
:107E280023F4FF4323F070031360D0E90243234394
:107E38002B43456911682B4385692B43C5692B433F
:107E4800056A2B430B431360FFF7AEFFB4F5804F71
:107E580004BF002343604268816C02F07F030B601B
:107E6800D0E91314013A032A4C6020D8164A17495E
:107E780081651A44013B9200012103F0030301FAD2
:107E880003F300214265C3651160114A536400235E
:107E98000122C36380F8243080F82520184638BDB5
:107EA8000C4B1344B3FBF1F30B499B00B1E70023E0
:107EB800C0E91533C365EAE70120F0E7070402408B
:107EC800F8FFFDBF000002403F8200104009024059
:107ED80000090240F8FBFDBF0004024038B5002845
:107EE80041D00268136823F0010313601F4B9A42C4
:107EF8004FF0140130D81E4B1344B3FBF1F31D4966
:107F08009B00C0E91013012403F01C0304FA03F3D7
:107F1800002515604B60FFF747FF836C41681D60C3
:107F2800D0E913325A604A1E032A06D8124B0B4472
:107F38009B0094401D60114B5C640023C363C0E93F
:107F48001533C0E90B33C0E90D33C36580F825301C
:107F580080F82430184638BD094B1344B3FBF1F3BD
:107F680008499B00CDE70120F5E700BF0704024060
:107F7800F8FFFDBF000002403F82001000090240E8
:107F8800F8FBFDBF0004024070B590F82450012DA5
:107F980004463BD090F825600125AE4280F8245075
:107FA8004FF000062CD1022580F825500568C663DD
:107FB8002E6826F001062E60FFF7DCFE036BBBB1CE
:107FC8002B6843F00E032B60A36C1A68D20342BFE0
:107FD8001A6842F480721A60636D1BB11A6842F421
:107FE80080721A602B6843F001032B60002070BD7B
:107FF8002B6823F004032B602B6843F00A03E2E7A5
:108008008023C36380F824602846F0E70220EEE767
:10801800034640B190F82520022A06D00422C26304
:10802800002280F82420012070470268806C1168C3
:1080380021F00E011160016821F48071016011685E
:1080480021F001011160D3E9100202F01C010122A4
:108058008A404260D3E9132151605A6D32B11168E8
:1080680021F480711160D3E91621516001220020AA
:1080780083F8252083F82400704710B590F8253040
:10808800022B03D00423C363012010BD03681A68C0
:1080980022F00E021A601A6822F001021A60826C3D
:1080A800136823F480731360D0E9101303F01C02E3
:1080B800012393404B60D0E913325A60436D33B1CA
:1080C8001A6822F480721A60D0E916325A600123C5
:1080D80080F82530836B002480F8244013B198473A
:1080E8002046D2E71846D0E770B4426C046C0368A7
:1080F80026681D6802F01C020421914031420FD00D
:1081080015F0040F0CD01A6892065EBF1A6822F0A8
:1081180004021A60036B6160002B33D070BC1847EF
:1081280002219140314217D015F0020F14D01A687D
:10813800940606D41A6822F00A021A60012280F80E
:108148002520114A93428CBF104B114B59600023D4
:1081580080F82430C36ADFE708219140314211D00A
:1081680029070FD5196821F00E011960012303FAB8
:1081780002F26260C36380F82530002380F824305F
:10818800436BC9E770BC704780000240000402409E
:10819800000002400A4A536943F4802330B5536112
:1081A800EFF3108472B60023CD58C5500433B3F5ED
:1081B800807FF9D11369DB03FCD484F3108830BDC8
:1081C80000400058064B5A69002ABFBF054A9A600A
:1081D80002F188329A60BABF5869C00F0020704710
:1081E8000040005823016745044B5A6942F0004299
:1081F8005A615869C043C00F704700BF004000581B
:1082080070B50546FAF77AFC124E04463369D9036D
:1082180013D43369DA0744BF012232614CF2FA32CF
:10822800134011D10B4E306910F480200BD0FAF7AF
:1082380065FC001BA842F6D304E0FAF75FFC001BBC
:10824800A842E3D3032070BD024A1361024A012009
:108258005360F8E700400058300F00202DE9F04146
:10826800184D98462B78012B06460C46174626D003
:1082780001232B704FF47A7000236B60FFF7C0FF67
:10828800A0B9012E16D1104A536943F00103536176
:108298002760BFF36F8FC4F804804FF47A70FFF73C
:1082A800AFFF094A536923EA0603536100232B7081
:1082B800BDE8F08139462046FFF76CFFEDE7022064
:1082C800F6E700BF300F002000400058054A536908
:1082D80023F47E7343EAC00040F4803040F002008B
:1082E80050617047004000582DE9F041234F3B781A
:1082F800012B054688463FD001233B704FF47A7026
:1083080000237B60FFF77CFF044688B92B68042BA9
:1083180013D11B4A536943F4803343F00403536178
:108328004FF47A70FFF76CFF0446154B1A681B6808
:1083380000233B702046BDE8F0814FF0FF33C8F8BA
:1083480000306E68D5E901321344B3420AD9304689
:10835800FFF7BCFF4FF47A70FFF752FF50B1C8F82F
:1083680000600446064A536923F47E7323F002032F
:108378005361DAE70136E5E70224DBE7300F002036
:10838800004000582DE9F04F524C00234FF00F09E0
:108398000A6832FA03F501D1BDE8F08F012505FA24
:1083A80003F818EA020200F08E804E68032706F0F0
:1083B80003054FEA430E07FA0EFC6F1E012F6FEA02
:1083C8000C0C32D8876807EA0C0ACF6807FA0EF750
:1083D80047EA0A078760476827EA0808C6F30017CC
:1083E8009F4047EA08074760C76807EA0C088F6894
:1083F80007FA0EF747EA0807022DC76017D14FEAB8
:10840800D30800EB880803F0070AD8F820704FEA71
:108418008A0A09FA0AFB27EA0B0B0F6907FA0AF717
:1084280047EA0B07C8F8207001E0032DDCD1076884
:1084380005FA0EF507EA0C073D4316F4403F0560C0
:1084480041D023F0030707F1804707F5803703F091
:10845800030CBD684FEA8C0C4FF0070E0EFA0CFEA9
:10846800B0F1904F25EA0E0E2FD01B4DA8422ED00A
:1084780005F58065A8420CBF0225072505FA0CF50D
:1084880045EA0E05BD602568D74316F4801F0CBF6A
:108498003D4015432560656816F4001F0CBF3D403C
:1084A80015436560D4F8805016F4803F0CBF3D40FA
:1084B8001543C4F88050D4F88450B60354BF3D40E7
:1084C8001543C4F88450013362E70025D6E7012537
:1084D800D4E700BF0008005800040048374A2DE9D7
:1084E800F04F00234FF0010A4FF0070B4FF00F0930
:1084F80031FA03F401D1BDE8F08F0AFA03FC1CEA53
:10850800010654D023F0030404F1804404F58034B8
:1085180003F00307A568BF000BFA07F8B0F1904F06
:1085280008EA050E45D0264DA84244D005F58065D9
:10853800A8420CBF02250725BD40754517D1D2F8C2
:10854800805025EA0605C2F88050D2F8845025EA02
:108558000605C2F88450156825EA060515605568B1
:1085680025EA06055560A56825EA0805A560056899
:1085780003265C0006FA04F423FA06F6254300EB0A
:108588008606056003F00705376AAD0009FA05F5A8
:1085980027EA05073762856825EA04058560456886
:1085A80025EA0C054560C56825EA0404C460013362
:1085B8009EE70025C0E70125BEE700BF0008005878
:1085C800000400480369194214BF012000207047C5
:1085D8000AB181617047816270470000044AD1681E
:1085E800014208B502D0D060FBF726F908BD00BFEC
:1085F8000008005803689A69910744BF00229A62EC
:108608009A69D2075EBF9A6942F001029A6170477F
:1086180030B5039D04682B4343EA0243064A606869
:10862800C1F309010B4342EA555223F0004320EA03
:1086380002000343636030BDFF63FF0303682DE955
:10864800F0419C6914F0100405460F4616466FD099
:1086580010220024DA61A0462B689A69900661D43A
:10866800B8F1000F35D044F0040401202E68B36936
:10867800D90541BF4FF48072F26144F00104012032
:108688005A0541BF4FF4806244F00804F2610120AA
:108698009B054FD54FF4007344F00204F36128465C
:1086A800FFF7A8FF736823F0FF7323F48B3323F4D9
:1086B800FF7323F0010373606B6C23436B64202307
:1086C80085F84130002385F8423085F84030012094
:1086D80032E07A1CC1D0FAF711FA801BB84201D8EF
:1086E800002FB9D12B68596895F842209869000481
:1086F800D2B20AD5490408D4202A06D05A6842F4CE
:1087080080425A60FAF7FAF906462B689B699B067D
:10871800A2D4FAF7F3F9801B1928F6D920244FF0D0
:10872800010899E7B8F1000F9DD12022DA619AE794
:1087380020469BE70028B2D1BDE8F08170B5044619
:108748000D46164623689B699B0701D5002070BD1E
:10875800324629462046FFF771FFA0B96A1CF1D0BE
:10876800FAF7CCF9801BA84201D8002DEAD1636C36
:1087780043F020036364202384F84130002384F805
:10878800423084F840300120E1E770B504460D46D8
:10879800164623689B695B070ED432462946204655
:1087A800FFF74CFF38BB23689A69910625D59A696B
:1087B800520703D5228D0AB1002070BD9A6912F0C4
:1087C80010021CBF1022DA614FF0200118BF0422EA
:1087D8006264D9615A6822F0FF7222F48B3222F463
:1087E800FF7222F001025A60002384F8411084F8D5
:1087F800423084F840300120DFE7FAF77FF9801B28
:10880800A84201D8002DC4D1636C43F020036364EF
:10881800202384F841300023EBE72DE9F041069F3F
:108828000446884616461D462268936938EA0303BB
:108838000CBF01230023B34201D0002015E06B1CBC
:10884800F3D0FAF75BF9C01BA84201D8002DEBD191
:10885800636C43F020036364202384F841300023D1
:1088680084F8423084F840300120BDE8F08170B5CA
:1088780004460D46164623689B699B0601D50020D1
:1088880070BD324629462046FFF7D8FE90B9FAF760
:1088980035F9801BA84201D8002DECD1636C43F058
:1088A80020036364202384F84130002384F8423095
:1088B80084F840300120E3E710B5044600284AD088
:1088C80090F8413003F0FF021BB980F84020F9F717
:1088D80003FE242384F8413023681A6822F0010239
:1088E8001A60626822F070621A619A6822F4004283
:1088F8009A60D4E90221012924D142F400429A6005
:108908005A6842F0007242F400425A60DA6822F46F
:108918000042DA60D4E904210A43A16942EA01224B
:10892800DA60D4E907210A431A601A6842F00102A2
:108938001A6000202023606484F84130206384F8A2
:10894800420010BD42F4044202299A6004BF4FF469
:1089580000625A60D4E70120F3E700002DE9F347ED
:10896800984690F841300A9F202B04460E469146BF
:1089780040F0868090F84030012B00F081804FF065
:10898800010A80F840A0FAF7B9F8192305460090C3
:1089980052464FF400412046FFF73FFF18B101202F
:1089A80002B0BDE8F087212384F84130102384F811
:1089B80042306064A4F82A80638DC4F824909BB286
:1089C800FF2B60632F4B26D9FF22228500934FF09F
:1089D800807331462046FFF71BFE638D9BB22A4603
:1089E80039462046FBB9FFF742FF0028D7D1236854
:1089F8002021D9615A6822F0FF7222F48B3222F4C6
:108A0800FF7222F001025A6084F8411084F8400095
:108A180084F84200C4E7628D009392B222854FF039
:108A28000073D2B2D5E7FFF789FE0028B7D1636A91
:108A3800226813F8011B91626362638D228D013BEA
:108A48009BB26385638D013A92B29BB22285002B5B
:108A5800C3D0002AC1D100953B4680212046FFF7AC
:108A6800DCFE00289BD1638D9BB2FF2B03D9FF222C
:108A780022850090ABE7628D009092B22285CEE706
:108A880002208DE7002000802DE9F347984690F8F2
:108A980041300A9F202B04460E46914640F08780BD
:108AA80090F84030012B00F082804FF0010A80F8E6
:108AB80040A0FAF723F819230546009052464FF4D0
:108AC80000412046FFF7A9FE18B1012002B0BDE819
:108AD800F087222384F84130102384F84230606400
:108AE800A4F82A80638DC4F824909BB2FF2B60639E
:108AF800304B26D9FF22228500934FF080733146F0
:108B08002046FFF785FD638D9BB22A4639462046ED
:108B1800FBB9FFF7ACFE0028D7D123682021D96123
:108B28005A6822F0FF7222F48B3222F4FF7222F08C
:108B380001025A6084F8411084F8400084F8420029
:108B4800C4E7628D009392B222854FF00073D2B2CF
:108B5800D5E7FFF71AFE0028B7D123685A6A636A77
:108B68001A70636A228D01336362638D013B9BB285
:108B78006385638D013A92B29BB22285002BC2D0E5
:108B8800002AC0D100953B4680212046FFF745FECC
:108B980000289AD1638D9BB2FF2B03D9FF2222852F
:108BA8000090AAE7628D009092B22285CDE702205C
:108BB8008CE700BF0024008010B590F84120202ADF
:108BC8000346D4B21CD190F84020012A18D02422A0
:108BD80080F841200268106820F0010010601068D9
:108BE80020F4805010601068014311601168002063
:108BF80041F00101116083F8414083F8400010BD45
:108C08000220FCE710B590F84120202A0346D4B290
:108C18001BD190F84020012A17D0242280F8412047
:108C28000268106820F001001060106820F470607D
:108C380040EA012111601168002041F00101116032
:108C480083F8414083F8400010BD0220FCE7000093
:108C5800024A136843F48073136070470004005895
:108C68000D4B10B55B690C4628B99A0507D500F07D
:108C780027F820B110BD9B0501D400F019F8074A68
:108C88001369012C23F00403136101D130BFF1E70C
:108C980040BF20BF20BFEDE70004005800ED00E012
:108CA800024B186800F4C060704700BF0004005809
:108CB800024A136843F48043136070470004005865
:108CC8000C4A136823F4804313600B4B1B68322152
:108CD8004B430A49B3FBF1F35169890500D533B910
:108CE800536913F4007F14BF032000207047013B31
:108CF800F2E700BF000400582808002040420F0097
:108D08000B4A136823F0070343F002031360094B6F
:108D18001A69012842F004021A6105D130BF1A69A4
:108D280022F004021A61704740BF20BF20BFF6E757
:108D38000004005800ED00E04FF0B0431868C0F39D
:108D4800404070474FF0B0431868C0F34000704788
:108D58004FF0B042536823F47F4343EA0023536043
:108D680070474FF0B0431868C0F340607047000088
:108D78007FB54FF0B0432C4AD3F80831C0F3031045
:108D880003F00F0352F82040284A52F82330B4FB6E
:108D9800F3F4FFF785FF264B054693E80700B5F582
:108DA800007F04AB03E9070010D0224B9C4218D384
:108DB80003F5B70303F67F539C4229D903F57413CF
:108DC80003F510639C4225D802230BE01A4B9C4202
:108DD80007D91A4B9C421BD903F5370303F5D8531F
:108DE800F0E7002304AA02EB830353F80C4C144D5C
:108DF8002B6823F0070323432B60F9F77FFE064611
:108E08002B6803F007039C4206D1002004B070BD14
:108E18000123E7E70024EAE7F9F770FE801B022840
:108E2800EED90320F2E700BFB05201085052010802
:108E3800E8460108C0CF6A00BFEA21013F93340227
:108E4800004000584FF0B04310B59A68D96812F046
:108E58000C0205D00C2A4AD101F00303012B50D192
:108E68004FF0B0412B480B6813F0080306D00B688D
:108E780013F0080337D1D1F8941007E00C682407E1
:108E880056BFD1F894300968C3F3032350F8233050
:108E9800002A0CBF184600204FF0B0418A6802F043
:108EA8000C020C2A1ED1CA6802F00302022A2ED034
:108EB800032A06D10B68184A13F4801F174B18BFF2
:108EC80013464FF0B042D068D168D268C0F306208C
:108ED8005843C1F302130133B0FBF3F0530F0133CE
:108EE800B0FBF3F010BD0B68C3F30313CEE7042AFD
:108EF8000AD0082A05D11B6813F4801304D1074847
:108F0800CAE700231846C7E703480023C4E7024B13
:108F1800D7E700BFB05201080024F4000048E80178
:108F280008B5FFF78FFF4FF0B043044A9B68C3F3BF
:108F3800031352F82330B0FBF3F008BD5052010878
:108F48002DE9F0410446002853D04FF0B0439D6806
:108F5800DE6803689B0605F00C0506F0030668D575
:108F6800026A1DB10C2D46D1012E44D1002A40D0F1
:108F78004FF0B043A16A1A68170756BFD3F8943068
:108F88001B681B0903F0F00399421FD90846FFF735
:108F9800EFFE00282DD14FF0B042136843F00803CC
:108FA80013601368A16A23F0F0030B431360606A2F
:108FB800FFF7CEFEFFF7B4FFAB4B1860AB4B18685A
:108FC800F9F79AFD002834D0BDE8F0814FF0B0429F
:108FD800136843F008031360136823F0F0030B438E
:108FE8001360606AFFF7B4FE0846FFF7C1FE002869
:108FF800E0D00120E8E74FF0B043002A54D01A68C7
:1090080042F001021A60F9F779FD0746FFF79AFE68
:10901800002842D04FF0B042136843F008031360B1
:109028001368A16A23F0F0030B431360606AFFF72B
:109038008FFE2368D80748D42368990700F18C80ED
:1090480023681E0740F1FA80A3694FF0B046002B51
:1090580000F0E180D6F89430E16903F01002914203
:1090680000F0C48003F00302022AC2D0D80740F1FE
:10907800B380D6F8943023F00103C6F89430F9F79A
:109088003DFD0746D6F89430990740F1A580F9F7D9
:1090980035FDC31B112BF5D904E0F9F72FFDC01BD3
:1090A8000228B3D903208FE71A6822F001021A6058
:1090B800F9F724FD0746FFF745FE0028B9D0F9F770
:1090C8001DFDC01B0228F6D9ECE7082D03D00C2D96
:1090D80005D1032E03D16368002BADD189E74FF08A
:1090E800B043A1681A6822F480120A431A606268C1
:1090F800B2F5803F10D11A6842F480321A60F9F74D
:10910800FDFC0746FFF718FE002895D1F9F7F6FC95
:10911800C01B6428F6D9C5E7B2F5041F04D11A6844
:1091280042F400121A60E6E7196821F480311960E8
:10913800196821F400111960002AE0D1F9F7DEFC62
:109148000746FFF7F9FD00283FF476AFF9F7D6FC9C
:10915800C01B6428F5D9A5E7042D236903D00C2D7D
:109168000ED1022E0CD1002B3FF443AF4FF0B0428A
:109178006169536823F0FE4343EA016353605FE784
:109188004FF0B046BBB1336843F480733360F9F7EE
:10919800B5FC074633685A0507D57368626923F03A
:1091A800FE4343EA026373604AE7F9F7A7FCC31B6F
:1091B800022BEFD976E7336823F480733360F9F72D
:1091C8009DFC074633685B057FF53AAFF9F796FCD7
:1091D800C31B022BF6D965E74FF0B042E169D2F81C
:1091E800943023F010030B43C2F894304FF0B0478B
:1091F800D7F8943043F00103C7F89430F9F77EFCB0
:109208000646D7F894309A0718D4F9F777FC831BE9
:10921800112BF6D946E7D6F8943023F00103C6F8A7
:109228009430F9F76BFC0746D6F894309B0705D5C0
:10923800F9F764FCC31B112BF6D933E723685807E9
:1092480054D50B4F3B68D90514D4FFF701FDF9F746
:1092580055FC06463B68DA050CD4F9F74FFC831B2E
:10926800022BF7D91EE700BF280800202C08002091
:1092780000040058E3684FF0B046002B58D023F0A4
:109288008003052B02BFD6F8903043F00403C6F8DC
:1092980090304FF0B046F9F731FCD6F8903043F0F3
:1092A80001030746C6F8903041F28838D6F8903066
:1092B8009B0705D4F9F722FCC31B4345F6D9F1E611
:1092C800E36823F00403812B1BD1F9F717FCD6F8C8
:1092D800903043F08003C6F8903007464FF0B04610
:1092E80041F28838D6F89030180504D5E06A00288D
:1092F8004AD1002068E6F9F701FCC01B4045F1D9C6
:10930800D0E6F9F7FBFBD6F8903023F08003C6F8D7
:10931800903007464FF0B04641F28838D6F8903082
:109328001905E3D5F9F7EAFBC01B4045F6D9B9E6BC
:10933800F9F7E4FBD6F8903023F080030746C6F827
:10934800903041F28838D6F890301A0516D4F9F7DB
:10935800D5FBD6F8903023F00103C6F890300746C5
:109368004FF0B04841F28836D8F890309B07BDD509
:10937800F9F7C4FBC31BB342F6D993E6F9F7BEFB72
:10938800C01B4045DFD98DE60C2D4ED04FF0B043C1
:1093980002281A6822F080721A6033D1F9F7AEFBFE
:1093A8000546FFF7DEFC38BBD4E90C314FF0B0427C
:1093B8000B43D0682D4901400B43E16B0B43216CF3
:1093C8000B43616C0B43A16B43EA0123D360136821
:1093D80043F080731360D36843F08053D360F9F788
:1093E8008DFB0446FFF7BDFC002882D1F9F786FB08
:1093F800001B0A28F6D955E6F9F780FB401B0A2816
:10940800CFD94FE6F9F77AFB0446FFF7AAFC30B943
:109418004FF0B042164BD1680B40D360D4E5F9F752
:109428006DFB001B0A28F0D93CE601283FF4CCADBF
:109438004FF0B043226BDB6803F0030191427FF4E5
:10944800D8AD616B03F070028A427FF4D2ADA16B94
:1094580003F4FE42B2EB012F7FF4CBAD626C03F054
:10946800604393423FF445AFC3E500BF8C80C11110
:10947800FCFFFEEE2DE9F0410D46044610B901202F
:10948800BDE8F081684E336803F007038B4216D3BA
:1094980023689A0727D54FF0B047A268BB6823F026
:1094A800F0031343BB60F9F729FB0646BB68DB03EF
:1094B80019D4F9F723FB831B022BF7D911E0336882
:1094C80023F007030B433360F9F718FB07463368AB
:1094D80003F00703AB42DBD0F9F710FBC01B0228EF
:1094E800F5D90320CCE72368580617D54FF0B047C5
:1094F8006269D7F8083123F00F0343EA1213C7F85B
:109508000831F9F7FBFA0646D7F80831D90305D42C
:10951800F9F7F4FA831B022BF6D9E2E723685A0716
:1095280013D54FF0B047E268BB6823F4E0631343F8
:10953800BB60F9F7E3FA0646BB689B0305D4F9F765
:10954800DDFA831B022BF7D9CBE72368180714D55C
:109558004FF0B0472269BB6823F4605343EAC20363
:10956800BB60F9F7CBFA0646BB68590305D4F9F78F
:10957800C5FA831B022BF7D9B3E72368DA070FD4A0
:10958800294C236803F00703AB4239D8FFF7C8FC1E
:10959800264B1860264BBDE8F0411868F9F7ACBABD
:1095A8006268022A1DD1FFF7C7FB00283FF467AFA6
:1095B8004FF0B04641F28838B36823F003031343F1
:1095C800B360F9F79BFA0746B368626803F00C03C7
:1095D800B3EB820FD4D0F9F791FAC01B4045F3D909
:1095E8007FE7032A02D1FFF7BCFBDEE712B9FFF7DA
:1095F800A9FBDAE74FF0B0431B685B05D8D43EE718
:10960800236823F007032B432360F9F777FA06460C
:10961800236803F00703AB42B8D0F9F76FFA801B51
:109628000228F5D95DE700BF00400058280800204F
:109638002C08002008B5FFF773FC4FF0B043044A2C
:109648009B68C3F3022352F82330D84008BD00BFFB
:109658009052010808B5FFF763FC4FF0B043044A85
:109668009B68C3F3C22352F82330D84008BD00BF1B
:10967800905201084FF0B043D3F89000C0F3400077
:1096880070474FF0B0410209D1F8883002F47F22C8
:10969800000123EA020300F47F200343C1F8883065
:1096A80070474FF0B041020CD1F88830120423EA19
:1096B800020343EA0040C1F88800704770B50668A5
:1096C80016F48036044638D0FFF7C2FAF9F716FACE
:1096D800614E05463368DB0529D54FF0B043616B11
:1096E800D3F8902002F44072914214D0D3F890102D
:1096F800D3F8902042F48032C3F89020D3F8902019
:1097080021F4407022F480328D07C3F89020C3F80A
:10971800900000F190804FF0B042616BD2F8903029
:1097280023F440730B43C2F89030002605E0F9F7A4
:10973800E5F9401B0228CDD903262568E8070AD594
:109748004FF0B0416268D1F8883023EA124392B2F0
:109758001343C1F88830A9070AD54FF0B041A26871
:10976800D1F8883023EA124392B21343C1F8883003
:10977800AA0609D54FF0B0422169D2F8883023F4FF
:1097880040630B43C2F88830AB0502D5206AFFF767
:1097980088FF680502D5606AFFF783FF290502D5AF
:1097A800A06AFFF77EFF6A0602D56069FFF769FFC6
:1097B8002B0602D5A069FFF764FFE80502D5E0692A
:1097C800FFF75FFFE90610D54FF0B042E168D2F825
:1097D800883023F440730B43C2F88830B1F5807F9A
:1097E80002BFD36843F08073D3602A040ED54FF0CC
:1097F800B042216BD2F8883023F040430B43C2F8C3
:10980800883019B9D36843F08073D3606B0410D5DE
:109818004FF0B042E16AD2F8883023F040530B434E
:10982800B1F1005FC2F8883003D1D36843F48033C4
:10983800D360304670BDF9F761F941F288360546C4
:10984800FFF718FF01283FF466AFF9F757F9401BF7
:10985800B042F5D970E700BF0004005830B590F861
:109868002C30012B02464FF0020022D0174B82F811
:109878002D00CA24012582F82C505C6253245C62B6
:10988800B1F5807F146B996914D121F488519961DD
:10989800596C24F0010421F0004159641463DD651A
:1098A8000A4BFF2159620020012382F82D3082F8EB
:1098B8002C0030BD21F408519961D96C24F00204C0
:1098C80021F00041D9641463D865E9E70028004015
:1098D80070B50B4E036B756D1D40EA07044603D542
:1098E8000123F365F9F77BFAAB0704D50223F36587
:1098F800204600F0CBF9012384F82D3070BD00BF5D
:109908000028004038B50A4CE36823F02003E360E0
:10991800F9F7F4F80546E3689B0601D5002038BD41
:10992800F9F7ECF8401BB0F57A7FF4D90320F6E795
:10993800002800402DE9F041114DEC6814F0400476
:1099480007461AD1EB6843F08003EB60F9F7D6F8C5
:109958004FF003080646EB685B0601D4032C02D1DE
:109968002046BDE8F081F9F7C9F8801BB0F57A7F89
:1099780084BF87F82D800324EDE70024F0E700BFBB
:109988000028004038B50F4CE36823F08003E360FB
:10999800A3699B06054606D4FFF7B4FF10B1032060
:1099A80085F82D0038BDA36923F02003A361FFF7D4
:1099B800A9FF10B1032085F82D00A36943F0200307
:1099C800A361EFE70028004038B5044600284BD0D3
:1099D80090F82D3003F0FF021BB980F82C20F8F71F
:1099E8008BFE0223214D84F82D30EB68DB0632D440
:1099F800CA236B6253236B622046FFF79BFF78BB39
:109A0800AB6923F08E6323F04003AB61216963687F
:109A1800AA690B431343A2691343AB61D4E9022338
:109A280043EA02432B61D4E90931EA680B4322F483
:109A3800F8521343EB602046FFF7A4FF80B9D4E93E
:109A48000713AA690B4322F0604213436269134368
:109A5800AB61FF236B62012384F82D30002002E004
:109A6800024BFF225A6238BD0120FCE70028004063
:109A78000023092803D840EA0310C0B270470A3807
:109A88000133C0B2F5E700002DE9F04790F82C301B
:109A9800012B05464FF0020069D0012385F82C30D0
:109AA8004E4B85F82D00DE6806F44076B6F5807FCB
:109AB80078D04C69087891F8019091F802A091F853
:109AC8002470002A55D19B6913F0400308BFCB705E
:109AD800FFF7CEFF80464846FFF7CAFF02465046CA
:109AE800FFF7C6FF81463846FFF7C2FF0B6ACF78FB
:109AF800234343EA875343EA090343EA084343EA13
:109B0800022343EA0063354ACA2050625320506258
:109B18008C6A8869B4F5807F946945D124F48854A7
:109B280094610124D465B6F5807F09BFCB691364BD
:109B38000343536418BF5064284B4A681A672A6B5A
:109B480042F001022A639A6942F488529A61244ACF
:109B5800D2F8803043F40033C2F880301F4BFF2224
:109B68005A620020012385F82D3085F82C00BDE8C5
:109B7800F087B4F1803F07D0B4F5000F04D09B699B
:109B880013F0400308BFCB700B6ACA781C4344EA41
:109B98000A0444EA004343EA092343EA825343EAB6
:109BA8000763B0E70023AEE724F408549461022465
:109BB800D465B6F5807F09BFCB6993640343D3644A
:109BC80018BFD064054B4A685A672A6B42F00202F4
:109BD8002A639A6942F40852B8E700BF0028004097
:109BE8000008005890F82C20012A03464FF0020084
:109BF80012D00A4A83F82D00CA21516253215162BA
:109C0800916941F020019161FF21516200200122F8
:109C180083F82D2083F82C00704700BF00280040EF
:109C280090F82C20012A03464FF0020019D00D4A63
:109C380083F82D00CA2151625321516291690A4863
:109C480041F080019161D0F8801041F48021C0F882
:109C58008010FF2151620020012283F82D2083F813
:109C68002C0070470028004000080058064B5A6D29
:109C7800520610B5044603D54022DA65F9F7B2F862
:109C8800012384F82D3010BD00280040704789005A
:109C980001F1804101F531410A607047890001F105
:109CA800804101F53141086870470000034AD2F845
:109CB800903043F40043C2F89030704700040058D5
:109CC800034AD2F8903023F40043C2F8903070472A
:109CD80000040058074B1A6822F040021A6040F44A
:109CE80041704FF4B85218605A601A6842F0400246
:109CF8001A6070470000015837B5054600284ED055
:109D0800837903F0FF046BB1032C0BD0254B4FF480
:109D180000629A612868FFF7DDFF002401232B7198
:109D2800AC602FE000236B712846F8F7FFFD1E4A50
:109D3800D2F8903043F48053C2F89030002CE5D12B
:109D480002234FF0B042AB71D2F8943023F40043B1
:109D5800C2F89430154B1B681C214B43DB0C642163
:109D68004B430193019B93B90124AC60FFF79EFF1D
:109D78000C4B9A6842F400629A604FF400629A6150
:109D8800002CC7D00123AB71204603B030BD019B26
:109D9800013B0193D2F894305B04E3D4E6E7012455
:109DA800F2E700BF00040058000800582808002007
:109DB80037B5174D2B6802461C204343DB0C642043
:109DC800434314480193019B93B901209060114CBF
:109DD80021732B681C214B43DB0C64214B430193FB
:109DE800019B6BB9012090600A4BDB6803B030BD62
:109DF800019B013B019383689C07E4D50020E6E7BB
:109E0800019B013B0193A368DB07E9D5ECE700BFA1
:109E1800280800200000015837B5184D2B68024665
:109E28001C204343DB0C6420434315480193019BEA
:109E3800A3B901209060124CFF2323732B681C25C3
:109E48006B43DB0C64256B430193019B73B90120C1
:109E580090600B4BDB680B7003B030BD019B013B7E
:109E6800019383689C07E2D50020E4E7019B013B4E
:109E78000193A368DB07E8D5EBE700BF28080020BB
:109E8800000001580F4B13B51B680F4C18225343A1
:109E98001B0D64225343014601936269019B02F042
:109EA800040223B902238B60012002B010BD019B7C
:109EB800013B0193606910F00200F6D0002AECD152
:109EC8001046F2E7280800200004005807B5037977
:109ED800012B0FD10A4B1B68182253431B0C01930B
:109EE800FFF7EEFE019B013B0193019B002BF9D18B
:109EF800FFF7DCFE03B05DF804EBFFF7C3BF00BF5C
:109F080028080020F8B51E468379012B154604461B
:109F18000F46DAB22DD14379012B2AD002234271A0
:109F28008371FFF7D3FF0D212046FFF7C9FEFFF726
:109F38003FFF390A2046FFF73BFFF9B22046FFF7FB
:109F480037FF2E44B5420ED12046FFF7AFFEFFF78C
:109F580099FFA06801230038A3714FF0000318BFD0
:109F680001206371F8BD15F8011B2046FFF720FF9B
:109F7800E8E70220F6E7F8B51E468379012B154677
:109F880004460F46DAB22FD14379012B2CD0427107
:109F9800FFF79CFF1D212046FFF792FEFFF708FF01
:109FA800390A2046FFF704FFF9B22046FFF700FF01
:109FB80000212046FFF7FCFE2E44B5420ED1204674
:109FC800FFF774FEFFF75EFFA06801230038A37156
:109FD8004FF0000318BF01206371F8BD29462046E1
:109FE800FFF71AFF0135E8E70220F6E7F8B51F4644
:109FF8008379012B154604460E46DAB22CD14379F3
:10A00800012B29D04271FFF761FF06F0EF03A3F19E
:10A01800840253425341237131462046FFF750FED4
:10A02800FFF7C6FE2F44AF4210D1FFF73FFE842E44
:10A0380002D02046FFF726FFA06801230038A3714D
:10A048004FF0000318BF01206371F8BD15F8011B1C
:10A058002046FFF7ADFEE6E70220F6E7F8B51E4614
:10A068008379012B154604460F46DAB227D1437986
:10A07800012B24D04271FFF729FF39462046FFF70C
:10A088001FFEFFF795FE00212046FFF791FE2E44A4
:10A09800B5420ED12046FFF709FEFFF7F3FEA06890
:10A0A80001230038A3714FF0000318BF012063712A
:10A0B800F8BD29462046FFF7AFFE0135E8E7022044
:10A0C800F6E737B50023ADF8043001AA02231221C0
:10A0D8000546FFF7C3FFBDF80440022364BA01AA8E
:10A0E800A4B219462846FFF781FFE20702D52846A1
:10A0F80009F076FBA30702D5284609F077FB60072D
:10A1080002D5284609F09CFB210702D5284609F00C
:10A118009DFBE20602D5284609F09EFBA30602D560
:10A12800284609F087FB600602D5284609F064FB3B
:10A13800210606D514F4807118BF0121284609F0BC
:10A1480061FBA20502D5284609F06CFB630402D521
:10A15800284609F087FB03B030BDF8B51E46837961
:10A16800012B154604460F46DAB227D14379012B55
:10A1780024D04271FFF7AAFE0E212046FFF7A0FD6A
:10A18800FFF716FE39462046FFF712FE2E44B54269
:10A198000ED12046FFF78AFDFFF774FEA068012361
:10A1A8000038A3714FF0000318BF01206371F8BD98
:10A1B80015F8011B2046FFF7FBFDE8E70220F6E74C
:10A1C800F8B51E468379012B154604460F46DAB2C8
:10A1D8002BD14379012B28D04271FFF777FE1E213E
:10A1E8002046FFF76DFDFFF7E3FD39462046FFF7F0
:10A1F800DFFD00212046FFF7DBFD2E44B5420ED1DE
:10A208002046FFF753FDFFF73DFEA0680123003805
:10A21800A3714FF0000318BF01206371F8BD2946F0
:10A228002046FFF7F9FD0135E8E70220F6E7026866
:10A2380052E8003F23F0C00342E8003102680029D9
:10A24800F5D102F1080353E8003F23F4000302F1BB
:10A25800080C4CE800310029F3D12023C0F88830DD
:10A268007047000010B5026852E8003F23F490736D
:10A2780042E8003102680029F5D10F4C02F10803C9
:10A2880053E8003F234002F1080C4CE80031002954
:10A29800F4D1C36E012B07D152E8003F23F010031D
:10A2A80042E800310029F7D12023C0F88C30002380
:10A2B800C366436710BD00BFFEFFFFEFF8B5044655
:10A2C8001346D4F88850202D32D1F1B1EAB1E06FAD
:10A2D800A4F85620A4F8542000262122C4F890603F
:10A2E8002165C4F88820226888B1124FC762124FCE
:10A2F8000763124F2832C0E90D76FDF745FE30B1ED
:10A308001023C4F89030C4F8885001200FE0236867
:10A3180040221A62226802F1080353E8003F43F022
:10A32800800302F1080141E800300028F3D1F8BDAC
:10A338000220FCE749A3000891A300089DA3000898
:10A3480008B50346806A1B681B6813F0200317D101
:10A35800A0F85630026802F1080353E8003F23F0E2
:10A368008003083242E8003102680029F2D152E83D
:10A37800003F43F0400342E800310029F7D108BD0F
:10A38800F8F786FEFBE7704708B5806AFFF7FBFF22
:10A3980008BD7047806A38B50468D0F88830D0F8AE
:10A3A8008C50A268120606D5212B04D10023A0F8F0
:10A3B8005630FFF73CFFA3685B0606D5222D04D173
:10A3C8000023A0F85E30FFF74DFFD0F8903043F03F
:10A3D8001003C0F89030FFF7DCFF38BD08B5806A7D
:10A3E8000023A0F85E30A0F85630FFF7D2FF08BD72
:10A3F800704700000368D9691A682DE9F04140F6F2
:10A408000F0631429D68044610D18E0640F19780B0
:10A4180002F0200605F080573E4300F09080436F1D
:10A42800002B00F08580BDE8F0411847AB4EAC48E2
:10A438002E401040304300F08280CF0709D5D00568
:10A4480007D501201862D4F8900040F00100C4F844
:10A4580090008F0709D5E80707D502201862D4F8BD
:10A46800900040F00400C4F890004F0709D5E807B1
:10A4780007D504201862D4F8900040F00200C4F810
:10A4880090000F070BD502F02000304307D00820BA
:10A498001862D4F8900040F00800C4F890000E0547
:10A4A8000AD5500108D54FF400601862D4F89030EE
:10A4B80043F02003C4F89030D4F89030002B37D004
:10A4C8008B0609D502F0200205F080552A4303D0F7
:10A4D800636F0BB1204698472668D4F89020B3687C
:10A4E80002F0280203F0400353EA0205204621D077
:10A4F800FFF7B8FEB3685F0617D5226802F10803B4
:10A5080053E8003F23F04003083242E800310029B5
:10A51800F3D1D4F8800040B1724B8363FDF7ADFDF1
:10A5280030B1D4F88000836B7DE72046FFF731FF18
:10A53800BDE8F081FFF72DFFC4F89050F8E7E06E12
:10A54800012840F08980CE0640F18680D00640F18F
:10A55800838010221A629A6851064BD5D4F880205D
:10A5680011684A6892B2002AE2D0B4F85C009042BE
:10A57800DED9A4F85E200A6892062FD453E8002F8B
:10A5880022F4807243E800210029F7D103F1080280
:10A5980052E8002F22F0010203F1080040E80021F0
:10A5A8000029F3D103F1080252E8002F22F04002FB
:10A5B80003F1080040E800210029F3D12022C4F863
:10A5C8008C20E16653E8002F22F0100243E80021B6
:10A5D8000029F7D1D4F88000FDF71AFD022323677C
:10A5E800B4F85E30B4F85C10C91A89B22046FFF797
:10A5F800FFFE9DE7B4F85E20B4F85E00B4F85C1086
:10A6080080B292B2002893D0891A89B200298FD0DB
:10A6180053E8002F22F4907243E800200028F7D175
:10A62800314D03F1080252E8002F2A4003F10806D1
:10A6380046E800200028F4D12022C4F88C20606766
:10A64800E06653E8002F22F0100243E800200028BB
:10A65800F7D102232367C9E7CF0209D56E0207D5D0
:10A668004FF4801220461A62BDE8F04100F0A0BD08
:10A6780008060BD502F0800005F40005284305D034
:10A68800A36F002B3FF454AF2046CCE64F0611D5FC
:10A6980056060FD553E8002F22F0400243E8002168
:10A6A8000029F7D12023C4F88830A1672046F8F79D
:10A6B800EFFC3DE70D0206D5500004D52046BDE865
:10A6C800F04100F077BDCB017FF532AF002ABFF62D
:10A6D8002FAF2046BDE8F04100F06BBD010000102F
:10A6E80020010004E5A30008FEFFFFEFD0F88C204E
:10A6F800B0F86010222A08B5036855D15B6A826DEC
:10A708000B401370836D01338365B0F85E30013BF5
:10A718009BB2A0F85E30B0F85E309BB2002B42D1FD
:10A72800026852E8003F23F4907342E8003103685E
:10A738000029F5D103F1080252E8002F22F00102A6
:10A7480003F1080C4CE800210029F3D12022C0F8BD
:10A758008C20184A41679342016705D1C26E012ACD
:10A768000ED0F8F7A3FC1EE05A681102F6D553E89C
:10A77800002F22F0806243E800210029F7D1EDE79D
:10A788000022C26653E8002F22F0100243E800219D
:10A798000029F7D1DA69B0F85C10D20644BF10225C
:10A7A8001A62FFF725FE08BD9A6942F008029A610D
:10A7B800F9E700BF00800040D0F88C20B0F86010A6
:10A7C800222A08B5036852D15A6A1140826D22F8CC
:10A7D800021B8265B0F85E20013A92B2A0F85E20B2
:10A7E800B0F85E2092B2002A40D153E8002F22F43C
:10A7F800907243E800210029F7D103F1080252E8DA
:10A80800002F22F0010203F1080C4CE80021002976
:10A81800F3D12022C0F88C20174A41679342016780
:10A8280005D1C26E012A0ED0F8F740FC1EE05A6826
:10A838001102F6D553E8002F22F0806243E8002188
:10A848000029F7D1EDE70022C26653E8002F22F075
:10A85800100243E800210029F7D1DA69B0F85C104A
:10A86800D20644BF10221A62FFF7C2FD08BD9A69DA
:10A8780042F008029A61F9E7008000402DE9F74F9D
:10A888000368B0F86080DF691A689D68D0F88C109A
:10A8980001922229044640F0B480B0F86890DFF8AD
:10A8A8006CA1DFF86CB10026B9F1000F01D0BB062E
:10A8B80021D4B4F85E309BB2D3B1B4F868209A4280
:10A8C80016D9226802F1080353E8003F23F08053A9
:10A8D800083242E8003122680029F2D14D4B636703
:10A8E80052E8003F43F0200342E800310029F7D145
:10A8F80003B0BDE8F08F2368A26D5B6A03EA080322
:10A908001370A36D0133A365B4F85E30013B9BB2AD
:10A91800A4F85E302368DF6978072CD0F9070AD5D8
:10A92800019AD20507D501211962D4F8901041F097
:10A938000101C4F89010B80709D5E90707D5022125
:10A948001962D4F8901041F00401C4F890107A0705
:10A9580009D5E80707D504211962D4F8903043F0E7
:10A968000203C4F89030D4F8903023B12046FFF7A2
:10A9780010FDC4F89060B4F85E309BB2002B93D100
:10A98800216851E8003F23F4807341E800302368D0
:10A998000028F5D103F1080252E8001F01EA0A0174
:10A9A80042E800100028F5D120215B45C4F88C103E
:10A9B800606720670AD05968090207D553E8001F65
:10A9C80021F0806143E800100028F7D1E16E0129E9
:10A9D80013D1E66653E8001F21F0100143E8001088
:10A9E8000028F7D1D969CA0644BF10211962204648
:10A9F800B4F85C10FFF7FCFC56E72046F8F756FB66
:10AA080052E79A6942F008029A6171E7FEFFFFEF88
:10AA180000800040F5A600082DE9F74F0368B0F85C
:10AA28006080DF691A689D68D0F88C10019222292D
:10AA3800044640F0B280B0F86890DFF868A1DFF80B
:10AA480068B10026B9F1000F01D0BB0621D4B4F8D3
:10AA58005E309BB2D3B1B4F868209A4216D9226806
:10AA680002F1080353E8003F23F08053083242E81C
:10AA7800003122680029F2D14C4B636752E8003F4D
:10AA880043F0200342E800310029F7D103B0BDE8C4
:10AA9800F08F2368A26D596A08EA010122F8021BA7
:10AAA800A265B4F85E20013A92B2A4F85E20DF698C
:10AAB80078072CD0F9070AD5019AD20507D50121C4
:10AAC8001962D4F8901041F00101C4F89010B80749
:10AAD80009D5E90707D502211962D4F8901041F089
:10AAE8000401C4F890107A0709D5E80707D50421AE
:10AAF8001962D4F8903043F00203C4F89030D4F8C7
:10AB0800903023B12046FFF744FCC4F89060B4F8B5
:10AB18005E309BB2002B95D1216851E8003F23F4A9
:10AB2800807341E8003023680028F5D103F108025A
:10AB380052E8001F01EA0A0142E800100028F5D196
:10AB480020215B45C4F88C10606720670AD05968DB
:10AB5800090207D553E8001F21F0806143E800107F
:10AB68000028F7D1E16E012913D1E66653E8001FEA
:10AB780021F0100143E800100028F7D1D969CA066E
:10AB880044BF102119622046B4F85C10FFF730FC6E
:10AB980058E72046F8F78AFA54E79A6942F008021B
:10ABA8009A6173E7FEFFFFEF00800040C1A700082D
:10ABB80038B5044603682169A2681D68C0690A435C
:10ABC80061690A437D49024329400A431A605A6869
:10ABD800E16822F440520A435A60794AA1699342D3
:10ABE8001CBF226A11439A6822F06E4222F4306236
:10ABF8000A439A60DA6A616A22F00F020A43DA624B
:10AC0800704A93421CD14FF0B043D3F8883003F018
:10AC1800030343F44033A3F54033013B022B00F216
:10AC2800C780694A9B5CB0F5004F40F08980082BCB
:10AC380024D8DFE803F061C0832380232323650041
:10AC4800624A934209D14FF0B043614AD3F8883041
:10AC580003F00C0343F44023E4E7594A93420DD12F
:10AC68004FF0B043D3F8883003F44063B3F5006F76
:10AC78001AD005D853B1B3F5806F12D0012009E07E
:10AC8800B3F5406FFAD14FF400400EE0FEF7D2FC66
:10AC980058B900204FF00113A3660023C4E91D33FF
:10ACA80038BDFEF7CFF8F3E74A4865684A4B626A51
:10ACB80005EB450133F81220B0FBF2F39942DDD8D9
:10ACC800B3EB053FDAD800231946F6F71DFF090252
:10ACD80041EA10616B080002C0182A464FF00003D1
:10ACE80041F10001F6F710FF3C4BA0F540729A4283
:10ACF800C4D82368D860CCE7FEF79CFC0028C8D0ED
:10AD08006168354B626A33F81220B0FBF2F24B08E7
:10AD180003EB42034FF6EF72B3FBF1F3A3F110011B
:10AD28009142ABD823F00F02216892B2C3F34203D9
:10AD38001343CB60ADE7FEF785F8DFE72548DFE78B
:10AD4800082B9BD801A252F823F000BF9DAD000844
:10AD5800A9AD0008B5AD000885AC0008AFAD000886
:10AD680085AC000885AC000885AC000879AD000802
:10AD78004FF400406368616A174A32F81120B0FB4B
:10AD8800F2F000EB5300B0FBF3F04FF6EF73A0F1D5
:10AD98001002ACE7FEF74EFC00283FF47AAFE9E773
:10ADA800FEF758FCF8E7FEF74DF8F5E70948E1E744
:10ADB800B0F5004FF4D1FEF74DFC9FE7F369FFCFE4
:10ADC8000080004000380140F05201080044004073
:10ADD800F352F5070024F40000530108FFFC0F00AC
:10ADE800836ADA0710B506D50168C46A4A6822F48E
:10ADF800003222434A609C0706D50168046B4A6802
:10AE080022F4803222434A60590706D50168446B10
:10AE18004A6822F4802222434A601A0706D501684C
:10AE2800846B4A6822F4004222434A60DC0606D555
:10AE38000168C46B8A6822F4805222438A609906AA
:10AE480006D50168046C8A6822F4005222438A609D
:10AE58005A060FD50168446C4A6822F480122243CE
:10AE6800B4F5801F4A6005D14A68846C22F4C00298
:10AE780022434A601B0606D50268C16C536823F456
:10AE880000230B43536010BD2DE9F041DDF8188015
:10AE980004460E4615461F462268D36936EA030360
:10AEA8000CBF01230023AB4201D0002027E0B8F1FA
:10AEB800FF3FF2D0F7F722FEC01B4045206802D8BA
:10AEC800B8F1000F1DD150E8003F23F4D07340E8DB
:10AED8000032002AF7D100F1080353E8003F23F0BD
:10AEE800010300F1080141E80032002AF3D12023D0
:10AEF800C4F88830C4F88C3084F884200320BDE876
:10AF0800F08103685A07C7D5C3691B05C4D54FF438
:10AF18000063036250E8003F23F4D07340E8003236
:10AF2800002AF7D100F1080353E8003F23F001039A
:10AF380000F1080141E80032002AF3D12023C4F8C7
:10AF48008830C4F88C30C4F89030D5E773B504461F
:10AF58000026C0F89060F7F7D1FD23681B681A0730
:10AF6800054619D423681B685B070AD56FF07E4332
:10AF7800009300222B464FF480012046FFF784FF00
:10AF8800B0B900202023C4F8883084F88400C4F8BD
:10AF98008C30E06620670CE06FF07E430093324609
:10AFA80003464FF400112046FFF76EFF0028D9D062
:10AFB800032002B070BD10B5044650B3D0F88830F5
:10AFC8001BB980F88430F7F74FFF22682423C4F8B0
:10AFD8008830136823F0010313602046FFF7E8FD6B
:10AFE800012816D0A36A13B12046FFF7F9FE23689B
:10AFF8005A6822F490425A609A6822F02A029A60AB
:10B008001A6842F0010220461A60BDE81040FFF7B6
:10B018009DBF012010BD000030B581658168A0F892
:10B028005C200023B1F5805FA0F85E20436735D12E
:10B038000369002B40F2FF1318BFFF23A0F860300C
:10B048000023C0F890302223C0F88C30016801F149
:10B05800080353E8003F43F00103083141E8003496
:10B068000368002CF2D1456E84680169B5F1005F70
:10B0780034D1B0F86850954230D8B4F5805F1DD10E
:10B08800254A264C002918BF22464267C1B153E819
:10B09800002F42F4807243E80021F7E729B90369D9
:10B0A800002B14BF7F23FF23C8E7B1F1805FC5D110
:10B0B8000369002B0CBF7F233F23BFE7174AE4E750
:10B0C80003F1080252E8002F42F0805203F1080011
:10B0D80040E800210029F3D1002030BDB4F5805F9D
:10B0E8000FD10F4A0F4C002918BF2246426751B1B1
:10B0F80053E8002F42F4907243E800210029F7D169
:10B10800EAE7084AF2E753E8002F42F0200243E852
:10B1180000210029F7D1DFE721AA000885A8000847
:10B12800C1A70008F5A60008D0F88C30202B30B451
:10B1380015D1B9B1B2B100230468C3660A4B9C4269
:10B148000AD063681B0207D554E8003F43F08063C8
:10B1580044E80035002DF7D130BCFFF75DBF022071
:10B1680030BC70470120FBE700800040436E30B5DB
:10B178002BB90123A0F86A30A0F8683030BD036805
:10B18800094D9A689968094C490FC2F342626B5C91
:10B19800615CDB00B3FBF1F3A0F86A30AB5CA25C46
:10B1A800DB00B3FBF2F3E7E720530108185301086B
:10B1B8007047704770471FB504AB03E9060090F865
:10B1C8008430012B04463AD0012380F884302423AC
:10B1D800C0F8883003681A6822F001021A609A6879
:10B1E80022F440120A439A6071B95A68BDF80C00FB
:10B1F8009DF80E1022F0100202435A605A6822F09D
:10B208007F4242EA01625A601A6842F001021A60FB
:10B21800F7F774FC6FF07E42034600924FF480010A
:10B2280000222046FFF730FE38B92023C4F88830C2
:10B23800002384F8843004B010BD0320F8E702200E
:10B24800F9E790F88430012B0FD0012380F884307F
:10B25800016851E8002F42F0020241E80023002B68
:10B26800F6D180F88430184670470220704710B530
:10B2780090F88430012B044617D02423C0F8883076
:10B2880003681A68196821F00101196042F0005238
:10B298004FF0005141661A60FFF768FF2023C0F89D
:10B2A8008830002084F8840010BD0220FCE770B5C7
:10B2B80090F88430012B044617D005682423C0F881
:10B2C80088302E682B6823F001032B60AB6823F0CD
:10B2D80060431943A960FFF749FF20232E60C0F897
:10B2E8008830002084F8840070BD0220FCE770B527
:10B2F80090F88430012B044617D005682423C0F841
:10B3080088302E682B6823F001032B60AB6823F08C
:10B3180060631943A960FFF729FF20232E60C0F856
:10B328008830002084F8840070BD0220FCE700000B
:10B3380038B5084D052455F8043B2BB9013C14F0E9
:10B34800FF04F8D1204638BDDB6898470028F5D0BF
:10B35800F9E700BF64100020034BD870034B1B684B
:10B368001B6C03B11847704778100020601000204C
:10B37800034B1874034B1B685B6C03B11847704789
:10B388007810002060100020F0B5314D314B95F950
:10B398000420314E91B00C46012795F905108DF81F
:10B3A800047002288DF809208DF80A1010D18DF844
:10B3B8000800D8711C7202F09FFD337803B114B1F4
:10B3C80001A803F003FA254B059A1A6011B0F0BDE5
:10B3D80059714FF480711A71D9801C7233788DF8C5
:10B3E800087053BB1F2306A88DF81C208DF8183051
:10B3F80002F064FF20238DF8183006A82B798DF809
:10B408001C3002F05BFF22238DF8183006A86B79F8
:10B418008DF81C3002F052FF21238DF8183006A851
:10B428006B798DF81C3002F049FF29238DF818300C
:10B4380006A80B4B079302F041FF02F05DFD0123C4
:10B4480006A88DF818308DF81C3002F037FFB4E7E5
:10B4580078100020300800205410002058100020D8
:10B46800000400017FB5092301A88DF8043003F01A
:10B47800ADF90038044B059A1A6018BF0120404204
:10B4880007B05DF804FB00BF5810002070B50446F3
:10B498000B46134962784A700020A2780A72087035
:10B4A8001A884A729A788A72DB780B746368CB6060
:10B4B8000C4B1B68DA6A2AB1237803F0FB030A2BCA
:10B4C80000D09047084E052556F8043B1BB15B6A2F
:10B4D8000BB120469847013D15F0FF05F4D170BD2A
:10B4E8003C080020601000206410002070B504465D
:10B4F80010480123037063784370A3788372E3686C
:10B50800C360E378037623694376237943720A4B51
:10B518001B689B6A03B19847084E052556F8043BFB
:10B528001BB19B690BB120469847013D15F0FF05FB
:10B53800F4D170BD50080020601000206410002075
:10B54800014B1868704700BF5810002000B58BB039
:10B55800012368468DF8003002F088FD38B99DF85F
:10B568000400003818BF01200BB05DF804FB002070
:10B57800FAE7000008B501F073FE48B9FFF7E6FFE7
:10B58800012806D0054BD879197AFFF7FDFE01206E
:10B5980008BDBDE80840FFF7CBBE00BF300800205B
:10B5A8002DE9F04186B005460E46174601F058FED3
:10B5B80000287FD101F06CFE044640B9FFF7C6FFB2
:10B5C800012807D03D4B197AD879FFF7DDFE6FF0D7
:10B5D800020462E0DFF8E88088F80860003E18BFDF
:10B5E80001268DF80460374E687833798DF812306B
:10B5F800694602F0D9FC00283ED08DF80440039437
:10B60800ADF810406FF0060495E803002E4B83E870
:10B618000300337988F80A30394601A803F0DAF9CB
:10B628002A4B059A1A60112841D801A353F820F033
:10B6380097B60008BDB60008B7B60008B7B6000848
:10B64800B7B60008B7B60008B7B60008D7B50008FF
:10B65800B7B60008B7B60008B7B60008B1B6000814
:10B66800B7B60008B7B60008BDB60008BDB60008F2
:10B67800BDB60008ABB600082B788DF808306B789B
:10B68800ADF810306B6803934FF0FF34BCE7104BF4
:10B6980000221A70E31D18BF1446204606B0BDE804
:10B6A800F0816FF00404F8E76FF00504F5E74FF058
:10B6B800FF34F2E76FF00104EFE700BF3008002025
:10B6C8005008002078100020600800205810002042
:10B6D8005C10002037B501F0E5FD144D052455F840
:10B6E800043B5BB11B694BB155F8043C9B682BB11B
:10B6F800984718B155F8043C1B699847013C14F069
:10B70800FF04ECD1FFF714FE68B9094D2B7853B14B
:10B71800084BADF80040D978019422466846FFF7F7
:10B728003FFF00B92C7003B030BD00BF641000208B
:10B738005C1000207810002030B58BB0054601F071
:10B748008FFD0446002839D1FFF700FF012838D1C2
:10B7580068468DF8004002F089FC10B14FF0FF30C8
:10B7680004E09DF80430AB4202D100200BB030BD9C
:10B77800012DF3D0022D11D0002DF7D1002BF4D0DC
:10B7880068468DF8045002F099FD0028E6D10E4B6A
:10B798001B681B6B002BE8D09847E6E7002BDDD130
:10B7A80068468DF8045002F089FD0028D6D1064B72
:10B7B8001B681B6B002BD8D02846EDE76FF0010003
:10B7C800D4E76FF00200D1E76010002010B50446FE
:10B7D8008AB018B94FF0FF300AB010BD0023684690
:10B7E8008DF8003002F042FC0028F3D19DF80430B7
:10B7F8002370F1E77FB500220B4620498DF807201A
:10B8080001220A7042784A700446002A33D102792C
:10B818000A721A884A729A788A72DB780B740369FA
:10B82800CB60C378164D8DF80830037B8DF809304E
:10B83800836803932B68DB6A0BB102A898472B68CF
:10B848009B6B13B1227E02B198470E4E052556F820
:10B85800043B1BB1DB690BB120469847013D15F04D
:10B86800FF05F4D10DF10700FFF7B0FF637913B1BD
:10B87800054B01221A7004B070BD00BF3C080020BF
:10B8880060100020641000205C10002010B50446F1
:10B898008AB018B94FF0FF300AB010BD20236846AF
:10B8A8008DF8003002F0E2FB0028F3D1024A9DF93E
:10B8B800043023701371EFE77810002000B58BB0C7
:10B8C8002323019068468DF8003002F0F7FC003819
:10B8D80018BF012040420BB05DF804FB70B5654C01
:10B8E80001468EB01822204606F0ECF8624B002282
:10B8F8001A70F8F73DFE23784068012202FA03F136
:10B90800014004D15D4B084608F0D2F8FEE75C49D7
:10B918005C481A4602F032F918B14FF0FF300EB009
:10B9280070BD272304A88DF8103002F0C7FC564ECE
:10B93800564D002870D1012333702B68DB690BB199
:10B9480000209847272304A88DF8103002F08EFBBA
:10B95800059B93F84820227093F8182193F81A3120
:10B968006270A370464BD3E9020105F09DFF0546BE
:10B978000028D2D1464E062304A88DF8103002F0D4
:10B9880075FB059B736104A802F098FC022304A8C8
:10B998008DF81030059602F069FB0836032304A8D9
:10B9A8008DF81030059602F061FB0F2606F040F87E
:10B9B800012304A88DF814308DF8106002F07EFC85
:10B9C80010230DEB03008DF810308DF8145002F0A1
:10B9D80075FC04238DF8103004A8A3788DF8143072
:10B9E80002F06CFC3A238DF8103004A863690593C3
:10B9F80002F064FC02A920788DF8086004F0E4F8ED
:10BA0800003818BF0120E0711420FFF757FFE079D4
:10BA180003F0A4F9284682E728238DF810302B6814
:10BA28001B6943B104A802F021FB2B6805981B6928
:10BA380040F2C4519847272304A88DF8103002F02B
:10BA48003DFC50B9012304A88DF8103002F00EFB1C
:10BA58009DF81430002B7FF46EAF3378002B7FF401
:10BA68006CAF052204A88DF81020059302F026FC7F
:10BA780078E700BF781000205C10002028530108E8
:10BA8800A0100020B81000205410002060100020E2
:10BA98003C10002037B500230D4601930446D0B969
:10BAA80000F0A8FB0190019BD3B10F4A42F8243063
:10BAB8000E4A9A620E4A1268916B1963916C596327
:10BAC80092690C49D9625A6128465B680A49F22290
:10BAD8009847002006E001A900F092FB0028E2D078
:10BAE8004FF0FF3003B030BD6410002091B3000860
:10BAF800601000206DB40008480F0020194B07B5EE
:10BB08001860194B194A1A60194A5A60194A9A60FA
:10BB1800194ADA60194B02681A6042685A608268EA
:10BB28009A60C268DA60164A1A6182695A61154BCE
:10BB3800C26B5A60144A019119609A601946134AF7
:10BB4800DA600020FFF7A6FF48B901A800F056FB0D
:10BB5800003818BF0120404203B05DF804FB4FF0E5
:10BB6800FF30F9E760100020B8100020F5B4000895
:10BB7800FDB7000815BC000895B40008A010002007
:10BB880081FB00089010002061B3000879B3000819
:10BB980051B118B1012804D000207047044B0B6044
:10BBA8007047044B0B60F7E74FF0FF30704700BF5A
:10BBB800000400010100010208B503F0EBF80028B9
:10BBC80014BF6FF00100002008BD08B502F0BCF9F1
:10BBD800002814BF6FF00100002008BD10B504460E
:10BBE8008AB018B94FF0FF300AB010BD212368465B
:10BBF8008DF8003002F03AFA0028F3D1024A9DF994
:10BC0800043023705371EFE7781000202DE9F041DC
:10BC18002E4D2F4F00232B7043786B703B689B6A27
:10BC28008AB004460BB128469847DFF8A880052655
:10BC380058F8043B1BB11B6A0BB120469847013EDC
:10BC480016F0FF06F4D12378052B2FD00B2B35D017
:10BC5800012B25D1204C062368468DF8003002F0D0
:10BC680005FA0199E07905F065FE10B91B4B019AB8
:10BC78005A611B48FFF70AFE1A48FFF7AFFF6B78B7
:10BC88008BB9A371184B5878FFF756FD3B685B6A70
:10BC98000BB1114898476B7813B9E07905F0DAFED3
:10BCA8000AB0BDE8F081FF23A371EFE70F4B012233
:10BCB8005A74227A9A74627ADA74F1E76378002BFC
:10BCC800EED00AB0BDE8F041FFF7CCBB5008002029
:10BCD8006010002064100020300800203C10002074
:10BCE8003408002035080020781000203C08002087
:10BCF80030B58BB0FFF769FF0446F0B903F044FF95
:10BD0800831C1DD0F8B9134D2B685B69DBB1272361
:10BD180068468DF8003002F0A9F92B6801985B6934
:10BD28004FF4B961984703F041FF78B92CB9094B32
:10BD38001B68DB690BB10120984720460BB030BD6A
:10BD48006FF00704EFE74FF0FF34ECE74FF0FF34F4
:10BD5800F3E700BF60100020014B1878704700BF60
:10BD6800CC100020014B5878704700BFCC10002041
:10BD780070470000044B9A7A0AB101225A70034BAB
:10BD88005B6903B118477047CC1000206C0800208D
:10BD980073B5224C6378002B33D008F073F96668CA
:10BDA8000546FFF7CDFB0644AE4214D2A37A93B101
:10BDB800E0228DF800208DF80130217AE3680193A4
:10BDC80001226846FFF7ECFB08B1073010D10023C9
:10BDD8006370A372656094F83430EBB1002384F883
:10BDE80034300F4B5B6BBBB102B0BDE870401847F5
:10BDF80040F2DC510B4808F011FA0A4808F0D4F96F
:10BE0800E8E794F83520002AE5D094F8360084F85D
:10BE18003530FFF791FCDEE702B070BDCC10002092
:10BE28006C0800200411002037B5104D104CC8B123
:10BE3800C1B10123627200222860E16023700D48BD
:10BE48000D4B00924FF0FF3108F002F900250B4826
:10BE580025822022294605F049FE6570A574A5862D
:10BE680003B030BD00232B602370EFE7C81000201B
:10BE7800CC100020041100207DBD0008E010002037
:10BE88002DE9F0478E4C23788CB0002B56D0C27821
:10BE98000AB9837B13B1238A01332382437B002BA6
:10BEA8004CD0E02A4AD10023A372876897F8008013
:10BEB800B8F1220F27D8B8F1220F30D8DFE818F0F0
:10BEC8004100FB0052005A0061006E0075008E00B0
:10BED8009D00B400C7002F002F002F002F002F0057
:10BEE8002F002F002F002F002F002F002F002F00D2
:10BEF8002F002F002F002F002F002F002F002F00C2
:10BF0800C900D000D400B8F17E0F00F0CC80B8F1A1
:10BF18007F0F00F0DF80B8F17D0F00F0AB80A57ACD
:10BF2800002D00F05B81674C637A3BB94FF47A715E
:10BF3800204608F073F9204608F036F90CB0BDE841
:10BF4800F087E36801220021A2721970A37AE168E0
:10BF58009818A0720620C854A37AE1689818A072AD
:10BF6800CA54DCE7584B9B6A002BD8D00121022029
:10BF78009847D4E77B7884F83630012384F8353045
:10BF8800CDE704238DF804307B78003B18BF0123EC
:10BF980001A88DF8083002F091F9C0E778780038E8
:10BFA80018BF012002F0DAFEB9E7484E0FCE01AD06
:10BFB8000FC50FCE0FC596E8070085E807007B7808
:10BFC8000A2BACD8424A12685268002AA7D00CA99A
:10BFD80001EB830353F82C0C9047A0E77878431EB5
:10BFE800012B9CD83A4B01381B6818BF01202072DE
:10BFF8009B68002B93D0984791E7E26801230821BA
:10C00800A3721170627A057BA17AAA4228BF2A46D8
:10C01800934284D285685A1CEB5CE56801334E1C58
:10C02800A6726B54D3B2EDE7E3680122A27209222B
:10C038001A70A37AE268218A581CA072D154A27A95
:10C04800238AE1681B0A501CA0728B5467E723827D
:10C0580065E705238DF8043001A802F0B7FB5EE719
:10C06800194BDB6A98475AE7194B78781B68607553
:10C07800DB68BEE7037B072B7FF451AF06238DF8FF
:10C088000430B7F80130ADF808307B793A791B04F1
:10C0980043EA0223FA781343642253430393BB7998
:10C0A8008DF81030D8E73B2201A88DF804208DF8D0
:10C0B800083002F003F9012384F834302FE700BF79
:10C0C800CC100020041100206C080020F446010860
:10C0D800C81000202A2301A88DF8043001F0C6FFFB
:10C0E80094F80A90E6689DF808009DF809509DF8B4
:10C0F8000A709DF80BC09DF80D309DF80E209DF834
:10C108000F109DF80CE009F1010A84F80AA006F85E
:10C118000980354E94F80A903668D4F80C8009F1F5
:10C12800010A84F80AA096F803A008F809A094F870
:10C138000A90D4F80C8009F1010A84F80AA096F84C
:10C1480002A008F809A094F80A90D4F80C8009F124
:10C15800010A84F80AA096F801A008F809A094F842
:10C168000A9009F1010A84F80AA096F80080E668A6
:10C1780006F8098094F80A80E66808F1010984F84D
:10C188000A9006F808C094F80AC0E6680CF101089D
:10C1980084F80A8006F80C70A77AE66807F1010CA3
:10C1A80084F80AC0F555A57AE6686F1CA772705521
:10C1B800A07AE568461CA6722954A17AE0684D1C4D
:10C1C800A5724254A27AE168501CA0728B54A37ADB
:10C1D800E268591CA17202F803E0A0E6034807F0E0
:10C1E80095FF6570AAE600BFC81000200411002062
:10C1F80070470000004870476C0800200020704716
:10C208004FF0FF3070470000044B054A93F818318F
:10C21800022B18BF062382F890347047E0160020DE
:10C22800A81C0020034BD3F8483313B15B6903B152
:10C2380018477047A81C0020034A137843F00403EA
:10C248001370FFF7EFBF00BFA41C00201FB50A4BF7
:10C258008DF8090093F87C208DF80A2093F88C203B
:10C2680093F848000D3202A98DF8082003F0ACFCC1
:10C27800C0B205B05DF804FBE016002010B5074C0D
:10C2880004F5806007F042FF94F81A3413B10123D3
:10C2980084F81934BDE81040FFF7C4BFA81C00207B
:10C2A80010B50C4CD4F8403343F08003C4F8403345
:10C2B80094F81A3413B10020FFF7E0FF94F8913492
:10C2C80023F0120343F0120384F89134BDE81040C0
:10C2D800FFF79ABFA81C00202DE9F041DFF8AC80D9
:10C2E80098F81831022B06460D4602D0284BDB6A17
:10C2F800984702F0E9FD044628B1022002F0DAFD71
:10C30800002002F0DCFD98F81831012B17D102F05B
:10C31800DDFD074630B1002002F0CDFD002002F01F
:10C32800CFFD3C4602F0D4FD48B1002002F0C4FD28
:10C33800002002F0C6FDBDE8F041FFF765BF002C04
:10C34800F9D1144C94F8902494F81A34BAB90BB172
:10C3580084F84164304602F065FFD8F82C0007F0F5
:10C368009BFED4F8B4339842E5D30B4807F0CEFED1
:10C3780094F8913443F0100384F89134DBE70BB15F
:10C3880084F84154284602F04DFFF1E7E0160020FA
:10C39800A85A0108A81C00204020002073B5164C9C
:10C3A800164D04F57A76EB6C95F8502095F97810CF
:10C3B80095F84800009603F02DFC95F8303184F884
:10C3C800FC3395F8480040F2012304F22442314638
:10C3D800A4F8FA3303F02AFC58B194F8243484F80A
:10C3E8006A34074B00205B6B984794F8FB3384F85A
:10C3F800903402B070BD00BFA81C0020E0160020D9
:10C40800A85A0108074A10B5137843F002031370BD
:10C41800FFF708FFBDE81040034B0122002102206E
:10C4280007F046BBA41C002071530108074A10B549
:10C43800137843F008031370FFF7F4FEBDE81040CB
:10C44800034B01220021022007F032BBA41C00206C
:10C45800815301082DE9F0410F4616461D468046D6
:10C4680007F010FE0B4A0C4C1378278123F01103B8
:10C4780043F011031370C4E9000866812573FFF7C0
:10C48800D1FEBDE8F041054B01220021022007F052
:10C498000FBB00BFA41C00205422002091530108A8
:10C4A80013B507F0EFFD0D4B6C461860204607F0FA
:10C4B8003DFD94E803000A4A0A4B83E80300137819
:10C4C80043F020031370FFF7ADFE074B0122002154
:10C4D800022002B0BDE8104007F0EABA642200204A
:10C4E800A41C0020E01F00209E530108F8B5334D1E
:10C4F80095F81841012C06464BD0022C51D064B94E
:10C5080038B9D5E91B0105F1740383E80300204617
:10C51800F8BD01283DD0022801D00324F7E7284FB1
:10C5280085F8180107F5747EBEE80F0007F57A7CD8
:10C53800ACE80F009EE8030095F8E9308CE80300AA
:10C5480087F8FB63E3B195F80031022B18D1D5F8D1
:10C5580004316B67C7F8EC3395F87D3095F80821FE
:10C5680087F8F83395F88C3085F8782087F8F93310
:10C5780097F81B2487F8E82340F20133A7F8FA3329
:10C58800002387F81A340F4BDB6A9847FFF706FF3A
:10C59800BDE702F0A4FC04460028B8D185F818616C
:10C5A800B5E70028B9D1064B85F81801062283F8AB
:10C5B8009024044BDB6A98473446A8E7E01600202D
:10C5C800A81C0020A85A01082DE9F04192B006469F
:10C5D80002F07AFC002840F05981AD4D95F81831E9
:10C5E800012B09D02B6BAB4C93B194F80431BBB140
:10C5F800042B6FD0032003E002F068FC18B10F2071
:10C6080012B0BDE8F08102F063FC0028EAD0F6E73A
:10C61800B5F82031D4F81C24013B53432B63E4E7DD
:10C628009D4803F008FA002840F02C8194F80C315A
:10C6380023802B6B0C930DF1180895F839308DF881
:10C648003830404695F81C318DF83A3007F094FCA4
:10C65800D5F82831009302AF98E80600D5F82431C0
:10C66800384607F020FC97E803000FAB83E8030087
:10C67800EB6A0D9300238DF844302388ADF84630DB
:10C6880095F8303101228DF839201BB98DF84420F6
:10C698008DF83930814B0093814B95F84800A3F110
:10C6A80079020CA903F005FBC0B10B28A8D1D4F876
:10C6B800941499B1002EA3D0D4F84033794843F0AC
:10C6C8002003C4F8403307F0A9FD764807F06CFD55
:10C6D800002095E7704803F0E2F9A4E795F8487060
:10C6E80095F9693095F9392095F87D106E4E3846E0
:10C6F80003F0ECFA009641B2EB6C95F850203846FE
:10C70800183603F087FA0096EB6C95F8502095F9E7
:10C71800701095F8480003F07DFAD4F8C413AB6D97
:10C72800D4F8DC230B44C4F8B033EB6D1344C4F8DD
:10C73800B43394F80431042B07D02B6E0B44C4F89F
:10C74800B0336B6E1344C4F8B4330023089395F8E0
:10C75800303183B108A802F095FC00284ED195F934
:10C76800390094F837629DF82070FFF76FFD3E445A
:10C7780080B2B04240D300238DF8133095F8393099
:10C788008DF8213095F838308DF82230D5F8803082
:10C798000993D5F884300A932388ADF82C3095F89E
:10C7A800303194F81B648DF82E3095F848003F4BD3
:10C7B8008DF820600DF1130208A903F03FFA012358
:10C7C80084F8413495F8393084F842349DF81330B0
:10C7D80084F84334D4F81C34C4F85064C4F848349A
:10C7E800C4F8583402F076FB50B1D4F81C0402F0B7
:10C7F80083FB28B1102003E7082001E71320FFE698
:10C8080095F81831012B01D102F078FB02F065FB95
:10C818000023059394F8043195F9395094F81B6472
:10C828009BB1042B7FF4E6AE05A802F067FE58BB67
:10C8380094F8183413B1059B013B0593164B0598E2
:10C848003246E9B202F0BCFE02E0134802F090FE64
:10C85800C0B9D4F8403394F80C11218043F0020396
:10C86800C4F8403394F8183411480133DBB284F823
:10C87800183484F845340F4B00259B6AC4F8985443
:10C88800984725E71120BBE61220B9E60E20B7E647
:10C89800E0160020A81C0020B01D00201017002062
:10C8A8003C2100201020002060200020C42000200F
:10C8B800AA1C0020A85A0108F0B5504C504EB4F8F4
:10C8C800DC202287D4E92D0194F8B12084F869206E
:10C8D80004F16C0282E80300D4E92F0104F1740228
:10C8E80082E80300B4F8C420A4F87C2091B0D4F8FE
:10C8F800CC20D4F8C810C4F884200025D4F8D0205F
:10C90800C4F888200123A4F82031C4F8801084F8E2
:10C918003051A56284F81B5184F83A5084F81D51AF
:10C9280084F81E51C4F83451C6F89854A6F818541F
:10C9380086F81A54A4F838518DF8183004F509739C
:10C94800039304F50A7394F84800A4F84651049335
:10C9580003A92C4B84F84551C4E94F55059303F0BE
:10C9680041F9E36EC6F8D43394F87D3086F8E033A5
:10C9780094F88C3086F8E1334FF48073A6F8E233EC
:10C9880086F8D05394F8303186F8E43306F5747796
:10C998000FCF06F57A740FC497E8030040F201231D
:10C9A80084E80300A6F8FA33D6F8483386F81B540F
:10C9B800CDE901551BB15A685B6901920293124B8C
:10C9C8000793A3F148020892A3F1140209920F4AAF
:10C9D8000B9229330A93A2F19C030C93A2F19803BA
:10C9E8000D93131D0E9301A902F14C0307A802F53C
:10C9F80099620F9302F05DFA11B0F0BDE0160020C5
:10CA0800A81C0020C421002010210020C4170020E9
:10CA1800F8B50D4F0D4C0E4E0D4607F077FB3B6BEE
:10CA2800984796F8480004F22442294603F0FEF895
:10CA380048B194F8243484F86A34706D7B6B984755
:10CA4800EB7C84F89034F8BDA85A0108A81C002093
:10CA5800E01600200F4890F81B3480F8B8330E4BCE
:10CA680093F8692080F8BB2393F87D2080F8C823C9
:10CA780093F88C2080F8C92393F8303180F8CC33B0
:10CA88000022A0F8CA2300F56E7100F56070FFF768
:10CA9800BFBF00BFA81C0020E0160020114890F876
:10CAA8009034EBB190F81B3480F8D0330E4BDA6E2B
:10CAB800C0F8D42393F87D2080F8E02393F88C20E5
:10CAC80080F8E12393F8303180F8E4334FF4807232
:10CAD800A0F8E22300F5747100F56670FFF798BFBF
:10CAE800704700BFA81C0020E016002070B5344C29
:10CAF8002421204604F0FCFF636A984218BF606254
:10CB08004FF01C012F4814BF0125002504F0F0FF49
:10CB1800636C984218BF60644FF480712A4818BF4C
:10CB280045F0020504F0E4FFD4F84831984218BFF4
:10CB3800C4F848014FF0D401244818BF45F0040553
:10CB480004F0D6FFD4F82032984218BFC4F8200267
:10CB58004FF000011E4818BF45F0080504F0C8FF53
:10CB6800D4F82432984218BFC4F824024FF46071F4
:10CB7800184818BF45F0100504F0BAFFD4F8A835D6
:10CB8800984218BFC4F8A8054FF01401124818BFFE
:10CB980045F0200504F0ACFFD4F8C03598420F4B9F
:10CBA80018BFC4F8C005D3F8483318BF45F040058E
:10CBB8002BB11B691BB12846BDE87040184770BDF2
:10CBC800E016002008170020281700202C18002045
:10CBD80004190020081900208C1C0020A81C002023
:10CBE8002DE9F04F91B04FF00008012B05460F4694
:10CBF80002928DF81580ADF8188003D8C84EC1464A
:10CC0800B94502D311B0BDE8F08F15F8090002F05C
:10CC180077FA4844B842F5DC15F8093009F10104FF
:10CC2800023BE4B2112BEDD801A252F823F000BF69
:10CC380081CC0008B3CC0008B3CD0008DDCD0008D6
:10CC480065CE00088DCE0008FFCE000831CF000861
:10CC5800ADCF00080DCC00080DCC00080BD00008A3
:10CC68000DCC00080DCC0008C9D00008F1D0000890
:10CC780035D1000873D10008052002F0EDFA90B113
:10CC88000521002002F0ACFA2A5DA64B09F1030445
:10CC980009F102095FFA89F983F85C2415F809207B
:10CCA80083F85D24E4B2A146AAE700238DF8163084
:10CCB8008DF817308DF81C308DF82030B8F1000F42
:10CCC8006CD14FF0050896F87C208DF83920631E4A
:10CCD80096F839208DF83B202B4496F838200D9390
:10CCE8008DF83C2096F81A3196F868208DF83D208A
:10CCF800D6F82C218DF83A300C9273B37B1C1B1B91
:10CD0800DBB28DF8383008AB019307AB009396F887
:10CD180048000DF117030DF116020CA902F09AFF55
:10CD28008DF8150000F00700072813D196F939206F
:10CD38009DF9163086F839309A429DF8173086F8F2
:10CD48003830B8BF01229DF81C30B8BF86F81D21C5
:10CD580086F868304FF0000909E00523D1E7012281
:10CD68000DF11501032002F0DBF809F101095FFA62
:10CD780089F29DF82030B3FBF8F19142EFD82344B3
:10CD8800DCB2631EDBB29F420DD9EA5C032A9AD05B
:10CD9800A74288BF1C464FF0010884E709F105093E
:10CDA8005FFA89F4F7E71C46F5E72B5D012203F0EB
:10CDB8000F0309F1020986F81B3102FA03F35FFA3F
:10CDC80089F9A6F82031002206A9042002F0A8F863
:10CDD8004C4668E707238DF815302B5D96F8480018
:10CDE800C3F3021203F00F038DF8303009F1030387
:10CDF800DBB28DF83120EA5C09F10403DBB209F1FA
:10CE08000504EB5C09F102095FFA89F91B0443EA9E
:10CE1800022315F809201343642253430CA90D93E8
:10CE280002F027FF00F00703072BE4B28DF8150086
:10CE38000CD19DF8303086F8703086F878300D9B2C
:10CE4800F36673679DF8313086F869308DF81800FD
:10CE5800012206A9052002F063F824E7314BD3F834
:10CE680048336BB11B685BB19847029B8DF818007B
:10CE780003F03F038DF81930022206A90620EAE7DD
:10CE8800FF20F2E703238DF815302B5D8DF8243051
:10CE98000CAB089309F10303DBB209F10604EA5C61
:10CEA80096F8480009F10403DBB208A9EB5C1B04FF
:10CEB80043EA022309F10202D2B209F10509AA5C88
:10CEC8001343642253435FFA89F90C9300230D93AB
:10CED80015F809308DF8383002F0D1FEC3B20028B9
:10CEE800E4B28DF81530FFF6DEAE8DF81830012269
:10CEF80006A90720AFE72B5D03F00F03012B4FF4C2
:10CF08007A7238BF0123534309F10209B365134408
:10CF18005FFA89F9F365002206A9082056E700BFE1
:10CF2800E0160020A81C00202B5D96F84800C3F3EB
:10CF380040128DF81D2007A9C3F3001203F00F0358
:10CF48008DF81C208DF81E3002F09FFE09F10209B1
:10CF580001305FFA89F93FF43BAFBDF81C30914AC4
:10CF6800A6F87C309DF81E309DF81C40D05CF4F784
:10CF78004DFD0223C6F880000CA996F848008DF8EC
:10CF880030308DF8324002F01FFE96F939300890A3
:10CF980040B29842B8BF184686F83900002206A960
:10CFA800092013E703238DF815302B5D8DF83030F9
:10CFB80009F10303DBB209F10504EA5C96F84800BD
:10CFC80009F10403DBB209F10209EB5C5FFA89F9A4
:10CFD8001B0443EA022315F8092013436422534330
:10CFE8000CA90D9302F057FEC3B20028E4B28DF8E5
:10CFF8001530FFF658AE8DF81830012206A90A2020
:10D0080029E7092002F028F9DFF89CA1002854D06C
:10D018000921002002F0E4F80023ADF8263009F1D8
:10D028000203DBB24FF47A71EA5C09F10303DBB265
:10D038000DF1300BEB5C1B0443EA02232A5D13431A
:10D0480009F10402D2B209F1060409F10509AA5C42
:10D058005FFA89F943EA026315F8092003934A4302
:10D0680012125846ADF8242006F060FF039B03F126
:10D07800965303F5A91303F5EC530893DAF83C33F8
:10D0880000930DF1200999E80600DAF838330AA868
:10D0980006F009FF0B9B00939BE806000A9B484695
:10D0A80006F0E6FE99E8030006F018FF01F021FFFC
:10D0B8000123E4B28AF83834F5E58AF83804F2E551
:10D0C8000C2002F0C9F800283FF4EDAD0C21002037
:10D0D80002F086F8344B93F89034043B012B7FF62A
:10D0E800E2AD01F002FFDEE509F10203DBB22A5DE1
:10D0F800E95C09F10303DBB209F10504EB5C09F112
:10D1080004095FFA89F91B0415F8090043EA0123A9
:10D1180013436421594300F00F0001F0E7FEE4B225
:10D128008DF81800012206A9112094E60D2002F0BE
:10D1380093F800283FF4B7AD0D21002002F050F815
:10D1480009F10203DBB2194AE85C2B5D126809F1A8
:10D15800040409F103095FFA89F943EA002015F884
:10D168000910E4B201F0C4FE9DE52A5D09F102034D
:10D1780009F1040409F10309DBB25FFA89F9E95CF2
:10D1880015F809301B0443EA01231343642058436C
:10D1980001F0B0FEE4B28DF81800012206A91320B0
:10D1A80059E600BFAB530108A81C002054220020F8
:10D1B8000E4B93F89124920703D593F88F24012AF4
:10D1C80008D90B4991F81A2122B18A6A501C18BF54
:10D1D80001328A620022A3F8182483F81A24D3F8AB
:10D1E800402322F00202C3F840237047A81C002005
:10D1F800E016002070B5184C184D04F55A7006F06A
:10D2080085FFD4F84033D4F89804D5F8906023F01B
:10D218002003C4F8403338B106F03EFF864203D2FB
:10D22800002385F83A3070BD0120FFF7CDF90028BA
:10D23800F9D00B28F7D095F8393084F84234092012
:10D2480094F8183484F8453484F8410401F0EAFF6E
:10D25800BDE87040FFF7ACBFA81C0020E016002016
:10D26800094BD3F84023012A0AD008490978C9078D
:10D2780008D43AB993F89204013818BF01207047CE
:10D288000020704701207047A81C0020A41C002023
:10D29800034BD3F84003431E58425841704700BF20
:10D2A800A81C00202DE9F04FA9B0EFF3108272B648
:10D2B800DFF8F4820021D8F80030C8F8001082F3B3
:10D2C8001088BA4C002B00F0E480DAB29B06039277
:10D2D80064D5B74D95F81831022B02D0B54BDB6AEF
:10D2E8009847EFF3108972B6B34F06F0CBFE3E684D
:10D2F800D4F8B013361A3144B04806F08FFFAF485F
:10D3080006F052FFD4F8B413AD48314406F086FF56
:10D31800AB4806F049FF89F3108894F81A34002BBB
:10D3280000F06D81152312A995F848008DF8483052
:10D3380002F04AFCD4F8B4130F900144A14806F057
:10D348006DFFA04806F030FF3B6894F81B24EB62A1
:10D358000DAF38468DF870201D9306F00DFED5F8F8
:10D368002831009306AE97E80600D5F824313046F8
:10D3780006F099FD96E803001FAB83E80300D4F894
:10D388001C341E9395F8303195F84800003B18BFBF
:10D3980001231CA98DF8713002F01FFC039BDF06E6
:10D3A8004BD5834DDFF820A2D5F8E420BAF90A302E
:10D3B800059298F800200493002363F300020A936F
:10D3C80088F8002084F84434049AA4F8223484F8B5
:10D3D8002534C4F82834A4F82C3484F82E34C4F83E
:10D3E800303484F82034C4F8343484F83834C4F839
:10D3F8003C34704B9AF90C90A4F88C2494F890243F
:10D40800DB6A84F88E9484F88F24DAF80470BAF80A
:10D418000860984794F88F3413B9694806F076FE87
:10D428003146384601F04EFD8346002800F0EA8078
:10D43800049BA4F87E3484F88094039B19071AD5BA
:10D448005B4B93F81831022B02D05A4BDB6A984792
:10D458000220FEF7D9FE84F8410401F0E3FE94F8B7
:10D468001A3413B1012384F8193494F8913443F031
:10D47800100384F89134039B5A0703D5062105202D
:10D48800FEF72AFF039B9B0703D504210320FEF721
:10D4980023FF01F035FD94F89124D7065FD50023CA
:10D4A80084F89234D4F840331E0644BF23F0820334
:10D4B800C4F8403312F0050F00F0FC820B2001F095
:10D4C800CBFE002800F0F68294F89134DD0700F1D5
:10D4D800F182580740F10883D4F8403323F002035F
:10D4E800C4F84033D4F8402382BB94F8915415F023
:10D4F80001011EBF2B4662F3000384F8913494F8AF
:10D5080091345E0744BF6FF3820384F8913401239A
:10D5180084F8923421B1D4F844332C481B689847D6
:10D528006D070BD52A4801F0A3FE01F0D1FE28B102
:10D5380094F8913443F0040384F8913401F0CEFC5C
:10D5480094F891346FF3041384F89134012384F828
:10D55800923494F8913443F0200384F8913494F889
:10D56800913418070AD56FF3C3031A4984F8913424
:10D57800D4F84433A1F12400DB68984794F8913437
:10D5880099070AD56FF34103124984F89134D4F806
:10D598004433A1F16C005B68984794F89034022BEF
:10D5A8001AD1FEF7FBFE17E0A41C0020A81C0020DF
:10D5B800E0160020A85A0108642200202820002034
:10D5C80040200020A820002054220020E82000202D
:10D5D800FC2000203421002094F891349A0640F170
:10D5E800C6826FF3451384F89134D4F84033002B86
:10D5F80040F0BD8229B0BDE8F04FFFF777BA84F854
:10D608004134A1E695F81821012A0CD101F05EFCFD
:10D61800804668B1584601F04EFC584601F050FC6F
:10D62800042384F88F347EB9012384F8213450E12F
:10D6380001F04EFC0028F6D0404601F03DFC404683
:10D6480001F03FFC0523ECE73B7804935B09013BC1
:10D65800062B00F21882DFE813F007001602950087
:10D668001602920016020702102EDDD995F8303105
:10D678001297F6B28DF84C60002BD5D11CA804F097
:10D688004BF912AA1CA9FF2002F0AEF89DF85830F9
:10D69800C3F3030307468DF82C3095F8480095F836
:10D6A8007D308DF82D3007220BA902F0A0FA002F4B
:10D6B8005DD100285BD09DF853309DF85220159914
:10D6C800C5F8E4101B0443EA02239DF85120022008
:10D6D8001343C5F8E03004F02DF99DF8583095F85B
:10D6E800480085F82E71C3F30212C3F3030385F8CB
:10D6F800703085F878309DF8593085F86920012B0D
:10D7080038BF01234FF47A725343AB651344EB657A
:10D718000DF15A034FF001081093113E94F81B3491
:10D728008DF83C300FA985F868808DF8446002F0C8
:10D7380066FA0223404685F8303101F08DFD18B1B4
:10D748004146384601F04CFD94F88F34012B00F225
:10D75800A88194F81A34002B40F09B8194F89134F6
:10D7680043F0100384F89134FEF74EFD65E601207E
:10D7780001F072FD0028E7D001210720E2E701232C
:10D7880084F8203495F87D308DF82E3094F82434C0
:10D798008DF82D3095F88C3095F848000D330BA98D
:10D7A8008DF82C3002F010FAA6F10D031BB2099087
:10D7B80023EAE37300B283423FF736AF0B2E7FF6BE
:10D7C80033AFBB4B25931CA8FF231C978DF87460BF
:10D7D8008DF8983002F0D4F8074600287FF424AF7B
:10D7E80095F81831012B13D101F070FB002873D084
:10D7F800384601F060FB384601F062FB04239DF8CF
:10D808007C101E9884F88F34C1F3001101F077FB67
:10D818009DF87C301E99C4F8341413F00F0203D01D
:10D828009DF89000002863D19DF89800002862D0E8
:10D83800002A7FF4F9AE9DF89020002A0CBF4FF023
:10D8480002084FF0030800220A92D5F8EC20914212
:10D8580054D195F8E910002950D0D5F80C1195F855
:10D86800EAB009680A9195F81811022902D1032132
:10D8780084F88F14B8F1030F7FF4D6AE13F0600F5D
:10D888007FF4D2AE0592012795F82E31BBF1000F37
:10D8980037D0BBF1010F38D1012B34D16FF0090615
:10D8A80046FA08F606F00106C6F10206F6B2BDF819
:10D8B8007E100AAA304601F02DFE40B307280CBF9F
:10D8C8000823012384F821340A9BC4F83034C4F8AF
:10D8D8006C34FEF7E5FCB0E501F0FAFA002897D0C1
:10D8E800384601F0E9FA384601F0EBFA052386E7F5
:10D8F8004FF00008A7E74FF00108A4E74FF0010B2D
:10D90800C2E70426D3E70326D1E70123DAE71CABF5
:10D91800009305990A9B3246584601F0B7FE20B19C
:10D9280002280CBF0A230B237FE60A9BC4F8303475
:10D93800C4F86C349DF87C3084F82104C3F3401398
:10D9480084F82E3484F8443494F88F3484F822749C
:10D95800012B9EBF0122A86285F81E21012FC4F861
:10D96800280484F82C0484F8410438D1022284F86D
:10D97800202495F83A20002A4AD19DF87C20D60622
:10D9880046D4012B94F840149DF87C2005D8012931
:10D9980001D1900601D501F05FFBB8F1020F94F8B0
:10D9A8008F3443D0B8F1030F0AD09DF87C10B8F13A
:10D9B800010F4A4601F00F0120A83BD0FFF710F9EC
:10D9C8009DF8903084F82334259BC4F828349DF8BA
:10D9D800983084F82C34012384F82D3430E0049AEC
:10D9E80002F0E002A02A1BD195F82E11012285F839
:10D9F8003A2009B927996963012B84F8202407D9AB
:10DA0800D5F89020C4F83C24DAF80020C4F898240B
:10DA180095F81821002AB4D1012284F82524B0E70A
:10DA2800002285F83A2084F82024A6E79DF898106B
:10DA380025984A46FFF7D4F89DF8903084F82334A7
:10DA48009DF89020E02A08D195F81F312BB984F869
:10DA58002324C4F82834A4F82C3494F8913443F0DF
:10DA6800020384F891346FE6114D013EB2B2791C7D
:10DA7800284604F027F80323A4F82034C4F82854CF
:10DA880084F82C64E9E7012384F82134FEF708FCC4
:10DA98005AE694F84434002B3FF460AE0020FEF7B9
:10DAA800EDFB94F88F34022B3FF45EAE56E600BFD0
:10DAB800E01E002094F89134590715D5012001F093
:10DAC800CBFB60B1012001F09DFB08B984F8180474
:10DAD800D4F8403323F00203C4F8403304E00620AE
:10DAE80001F0BAFB0028F3D194F89134DA077FF5F6
:10DAF800F9AC94F840240AB1032A18D11D4A94F8C5
:10DB0800181492F86820914205D29B0723D594F8FF
:10DB18008F34012B1FD8184806F0F8FAD4F8403390
:10DB280023F02003C4F84033FFF742FBDAE4012A6C
:10DB380011D194F81924002A3FF4D4AC0D4A94F872
:10DB4800181492F868209142E5D29F0703D594F8FB
:10DB58004434002BDFD194F8913400206FF3041380
:10DB680084F8913484F81904FFF744FBBAE429B027
:10DB7800BDE8F08FE0160020102000202DE9F04FBE
:10DB880089468DB090460746002800F08F8100290D
:10DB980000F08C810368002B00F088814368002B1B
:10DBA80000F084818368002B00F08081C368002B1B
:10DBB80000F07C81104602F003F8002800F078811C
:10DBC800BD4CBE4D384601F0C1FA40F2C4520021A6
:10DBD800204603F08BFF40F21C520021284603F038
:10DBE80085FFB74BC4F82C3104F50973089304F585
:10DBF8000A7300264046099308A9B24B84F8488066
:10DC08000A9384F8186184F88C608DF82C6001F010
:10DC1800E9FF0F2306A994F848008DF8183001F0A1
:10DC2800D3FF801B18BF01204FF00A0B84F81C019A
:10DC380006A994F848008DF818B001F0C5FF4FF018
:10DC4800060A84F8DC0006A994F848008DF818A0A4
:10DC580001F0BAFF102384F8DD0006A994F8480003
:10DC68008DF8183001F0B0FF1123C4F89C0006A904
:10DC780094F848008DF8183001F0A6FF1223C4F874
:10DC8800A00006A994F848008DF8183001F09CFF10
:10DC98001323C4F8A40006A994F848008DF8183096
:10DCA80001F092FF1423C4F8A80006A994F84800CC
:10DCB8008DF8183001F088FF1623C4F8AC0006A9C7
:10DCC80094F848008DF8183001F07EFF172384F887
:10DCD800B10006A994F848008DF8183001F074FFD7
:10DCE80018230DEB0301C4F8B400C4F8BC0094F881
:10DCF80048008DF8183001F067FFC0B21D2384F882
:10DD0800B80084F8C00006A994F848008DF81830C7
:10DD180001F05AFF1E2384F8C40006A994F84800AD
:10DD28008DF8183001F050FF1F2384F8C50006A9AC
:10DD380094F848008DF8183001F046FF2023C4F805
:10DD4800C80006A994F848008DF8183001F03CFF87
:10DD58000B23C4F8CC0006A994F848008DF81830B5
:10DD680001F032FF0C2306A9A4F8D00094F848006B
:10DD78008DF8183001F028FFD4F89C306365D4F88A
:10DD8800A030A365D4F8A430E365D4F8A83023669E
:10DD98004FF00108D4F8AC300590A4F8D2006366BF
:10DDA80084F8B080C4F894B084F898A0C4F84CB053
:10DDB80084F850A084F8688084F81F81C5F84893D7
:10DDC800FEF77AFD404B009632464FF0FF3105F5DD
:10DDD8005A70C5F84473C4E90B6684F8198185F84C
:10DDE8009164C5F8408306F033F9384B0096324603
:10DDF8004FF0FF3105F5607006F02AF9344B0096B4
:10DE080032464FF0FF3105F5667006F021F902AF92
:10DE1800304B009632464FF0FF3105F5806006F032
:10DE280017F9384606F0A8F897E8030004F5927346
:10DE380083E80300284B294F1E60294BC5F84C3353
:10DE4800284BC5F85433284BC5F85C33274BC5F825
:10DE58005033274BC5F8583305F553703B6898473E
:10DE680004F5A67003F084FB20B1112630460DB0EE
:10DE7800BDE8F08F204601F01DFB0028F5D101F028
:10DE880041F8B8B91B4801F067FB06460028ECD1F9
:10DE98007B69984703F0F4FDBB6D94F81901984726
:10DEA800FB6A9847012385F89234DFE70326DDE70C
:10DEB8000926DBE71326D9E7E0160020A81C002076
:10DEC80000040001C4210020FDD100085DCA00083B
:10DED800A5CA000885C20008A41C0020A85A010889
:10DEE800A9C400085DC4000841C2000835C4000880
:10DEF8000DC40008C817002008B5034B0020C3F85C
:10DF08004003FEF781F908BDA81C002010B5FFF7F3
:10DF1800A7F90A4C60B90A4B93F81831022B02D1C1
:10DF2800084BDB6A98470123C4F84033002010BD32
:10DF3800D4F84003013818BF0120F8E7A81C0020D6
:10DF4800E0160020A85A010838B5134C04F55A7099
:10DF580006F0DCF804F5607006F0D8F804F5667091
:10DF680006F0D4F804F5806006F0D0F800F0B5FFAC
:10DF78000A4B0025DB6A9847C4F84053FEF7B6FD04
:10DF88000749084840F2C45203F09CFD0123C4F835
:10DF98004033284638BD00BFA81C0020A85A0108F5
:10DFA800E01600201C11002070B52E4B8AB00546E3
:10DFB80093F8DD008DF8090093F8DC008DF80A006D
:10DFC80029489A6A90F81804039200268DF80B00E5
:10DFD80004960C46002940D00692D3F88820079270
:10DFE8001A8F93F81A118DF8151052BAADF820202F
:10DFF80093F87C2093F848308DF8243003AB8DF8E3
:10E0080022008DF8232000930DF10A020DF10B0375
:10E018000DF1090105A88DF8146000F0DDFE9DF9E9
:10E028000900FEF713F9607004A801F02BF8B0B9E5
:10E03800049A0F2A0DD863789A420AD81544AB423D
:10E04800A3EB02012CBF002001202170C0000AB000
:10E0580070BD002323700820F9E70320F7E7132099
:10E06800F5E700BFE0160020A81C00201FB50446F5
:10E07800002800F012810078412800F20881DFE8CA
:10E0880010F0420048004D00520056005A005F0050
:10E098000601060106010601060106010601060140
:10E0A80066006A006E0079008000830086008B009D
:10E0B80089008D009100940097009A009D00A000AF
:10E0C800AF00B300BB00B700BF00C200C600CF005E
:10E0D800CB00CD000601D3000601060106010601AA
:10E0E80006010601060106010601060106010601F0
:10E0F800060106010601DB00DF00E300E800EC0092
:10E10800F000F400FD00674B93F81831237104B058
:10E1180010BD644B93F83031237102E0606803F05E
:10E12800B5FB0020F3E7606803F0F6FBF9E75D4B09
:10E1380093F81A31F0E75B4BD3F8E0306360F0E70F
:10E14800584B211D93F8300103F0FEFBE9E7554BCE
:10E1580093F81931E0E7534B93F88C30DCE71C2334
:10E168008DF808304F4B02A993F8480001F02CFDB8
:10E178006060D6E74C4B043493E8030084E803005E
:10E18800CFE74A4B0434F7E7494B0434F4E7494BEB
:10E198000434F1E71A23E3E71923E1E7414B93F845
:10E1A8006830B9E73F4B5B6DC8E73E4B9B6DC5E7F1
:10E1B8003C4BDB6DC2E73B4B1B6EBFE7394B5B6EDD
:10E1C800BCE702238DF80830364B02A993F87C206F
:10E1D80093F848008DF80A2001F0F6FC2071A0E7BA
:10E1E800304B93F8DD3097E72E4B93F8393093E7AF
:10E1F8002C4B93F8DC308FE72A4B93F838308BE7B9
:10E20800284BDB6C9AE7274B93F8503084E7254B73
:10E21800D3F88430636084E7224B8FE7264B8DE781
:10E22800204BD3F8CC30F5E71E4BD3F82C31636084
:10E2380001F058FDA06074E71A4BD3F890307DE7E1
:10E24800184B93F81F3167E7164BB3F88830A38053
:10E2580067E7144BB3F88A30F9E7124BB3F8D030BC
:10E26800F5E7104BB3F8D230F1E70E4B93F848209E
:10E278000AB1062A13D1B3F8A035E8E7094B93F899
:10E2880048200AB1062A0AD1D3F8A43556E7204611
:10E2980004B0BDE8104000F024BE032037E7182082
:10E2A80035E700BFE01600204C1700209417002027
:10E2B800541700209C1700201C1100207FB504462D
:10E2C80010B9032004B070BDA44DD5F840339A07A7
:10E2D80000F171820278412A00F26A82DFE812F0C6
:10E2E8004200480056005C00600065006A00770044
:10E2F800820088008E0094009A00A000A600AC005E
:10E30800B6006802BB00DD00F000170139012A01E0
:10E3180044014D015101550159015D016802610136
:10E3280073019B018901AD01B301BA01BF01C401A9
:10E3380068022A02680268026802680268026802C3
:10E348006802680268026802680268026802680275
:10E358006802680236023B02400245024A024F0246
:10E3680054025E020079FEF7C1F80028AAD105E040
:10E378000379022BA5D07A4A82F8303195F8913486
:10E3880043F0200385F8913400209BE7406803F0B0
:10E398006FFA0028F2D094E7406803F0ADFAF8E786
:10E3A8006F4B027983F81A21E8E76D4B4268C3F88E
:10E3B800E020E3E76A4E416896F8300103F0BAFAC4
:10E3C80000287FF47EAF6368C6F8E430D6E741687A
:10E3D80000293FF476AF002001F0EAF90028CDD0FB
:10E3E80011206FE7416800293FF46BAF0120F3E784
:10E3F800416800293FF465AF0820EDE7416800292E
:10E408003FF45FAF0920E7E7416800293FF459AFBF
:10E418000C20E1E7416800293FF453AF0D20DBE70A
:10E42800416800293FF44DAF0E20D5E74168002927
:10E438003FF447AF0F20CFE74A4C494B007983F8A8
:10E448001901A36D9847E36A984797E7444B027907
:10E4580083F88C2092E7424E037A8DF8043096F8C0
:10E46800480096F87D308DF80530072201A901F0A3
:10E47800BEFB00283FF425AF636896F84800019377
:10E48800002201A901F0B3FB00283FF41AAF6C3653
:10E49800D4E9010186E8030070E7314E037A8DF86C
:10E4A800043096F8480096F87D308DF8053007223C
:10E4B80001A901F09CFB00283FF403AFB436E7E75D
:10E4C800274E037A8DF8043096F8480096F87D3088
:10E4D8008DF80530072201A901F089FB00283FF4D7
:10E4E800F0AED4E9010106F1740383E8030096F85D
:10E4F8001831022B7FF442AF96F83031002B3FF4ED
:10E508003DAF184BDB6A9847FDF748FF36E7144ED6
:10E51800037A8DF8043096F8480096F87D308DF827
:10E528000530072201A901F062FB00283FF4C9AEBB
:10E53800BC36ADE74368029301238DF80C30084BD5
:10E5480002A993F8480001F05FFB00287FF416AF9A
:10E55800B7E6436802930023EFE700BFA81C00203A
:10E56800E0160020A85A010803795A1E0E2A3FF621
:10E57800A8AE934A82F8683000E7914B42685A6522
:10E58800FCE68F4B42689A65F8E68D4B4268DA657F
:10E59800F4E68B4B42681A66F0E6894B42685A6685
:10E5A800ECE6874C037994F848008DF8043006228D
:10E5B80001A901F01CFB00283FF483AE9DF804304C
:10E5C80084F8DD30DAE67E4C03798DF8043094F86F
:10E5D800480094F87C308DF80630052201A901F036
:10E5E80006FB00283FF46DAE9DF8043084F83930FE
:10E5F800C4E6734C037994F848008DF804300A2275
:10E6080001A901F0F4FA00283FF45BAE9DF804304C
:10E6180084F8DC30B2E66A4C037994F848008DF847
:10E628000430092201A901F0E2FA00283FF449AEBA
:10E638009DF8043084F83830A0E6614B4268C3F88E
:10E648009420DA649AE65E4B027983F8982083F87E
:10E65800502093E65A4B4268C3F884208EE6584B04
:10E668004268C3F8CC2089E6012B40F0A480554CC1
:10E678002421204603F03CFA636A984201D017200F
:10E6880020E61C2104F1280003F032FA636C98425A
:10E69800F5D14FF4807104F1480003F029FAD4F859
:10E6A80048319842EBD1D42104F5A67003F020FA42
:10E6B800D4F820329842E2D1002104F5097003F021
:10E6C80017FAD4F824329842D9D14FF4607104F57E
:10E6D8000A7003F00DFAD4F8A8359842CFD1142166
:10E6E80004F2AC5003F004FAD4F8C0359842C6D10D
:10E6F800334E2146304640F2C45203F0E3F9204637
:10E7080040F2C452002103F0F1F995F81B3485F862
:10E71800E833736FC5F8EC3396F87D3085F8F83335
:10E7280040F20123A5F8FA33274B96F819019B6D9F
:10E73800984723E68379012B3FF6C3AD204B426807
:10E748004068C3F82C2100F0D1FE47E61C4B426814
:10E75800C3F8902012E61A4B027983F81F210DE6C0
:10E76800174B8288A3F8882008E6154B8288A3F8FF
:10E778008A2003E6124B8288A3F8D020FEE5104BCE
:10E788008288A3F8D220F9E50D4B93F848200AB106
:10E79800062A12D1A288A3F8A025EFE5084B93F822
:10E7A80048200AB1062A08D16268C3F8A425E5E51D
:10E7B80000F099FBD9E5012084E5182082E500BF27
:10E7C800E01600201C110020A85A01082DE9F0438A
:10E7D80087B00023ADF800300646002800F0ED8031
:10E7E8000361FEF73DFD20B10124204607B0BDE8D6
:10E7F800F08300F073FD0028F6D100F069FD0146B2
:10E8080018B96F48142203F071F96E4D95F89134D8
:10E81800012243F0040385F8552485F891343378B0
:10E828008DF804300021013B8DF80520ADF8061065
:10E838000C2B00F2BA80DFE803F007B8B8B878818B
:10E84800B8B88FB8AC99A800D5F8407317F020076E
:10E85800CAD196F80480B8F1020F45D1DFF8688173
:10E868005A4CFEF729F896F9051098F848003A46E8
:10E8780001F017FA88F83900B37988F83830384643
:10E8880007238DF80530FDF731FEFF2304F5867068
:10E89800A5F80C31C5F8084185F8047103F03CF877
:10E8A80004F58A7002F0F2FF3846FDF78DFE044643
:10E8B80040B196F9051098F84800012201F0F1F9E5
:10E8C80088F83900D5F894343361002C71D000F001
:10E8D800FFFC002889D195F8913485F81A0460F373
:10E8E800820385F8913480E7B8F1010F4FF00204F4
:10E8F800E8D1DFF8D4908DF8144099F8480089F8E9
:10E908001D7102A901F06EF9337989F830318DF85B
:10E9180005708DF80680FDF785FC95F8913443F075
:10E92800100385F891340024CCE7002269460220C0
:10E9380000F0F6FA0028F6D01324C3E7244BB28877
:10E94800DB6B96F90C10B0689847D5F8403343F064
:10E958000203C5F84033E6E702A90D2000F060FB8A
:10E968000028E0D0002269460D20E1E7164B93F815
:10E978001831D3B9347904F0070000F0ADFA8DF8F6
:10E988000040012269461020D2E700226946122081
:10E99800CEE78DF8072000F090FA044638B900F069
:10E9A80089FA204600F08BFA8CE702248AE70124D2
:10E9B80088E701A800F0DEFB17E7032415E700BF8E
:10E9C800FC200020A81C0020E0160020AA1C002023
:10E9D800A85A01082DE9F04F99B08046059118B959
:10E9E800032019B0BDE8F08F00230361FEF738FC5F
:10E9F8000646002840F0AB8045460FCD0EAC0FC44C
:10EA08005A4C98F800A0B8F80C7098F90EB0142277
:10EA180004F58860314603F069F8012284F841243E
:10EA2800534C94F83021022A35460BD194F818211A
:10EA3800022A07D194F81E2122B9BAF1010F38BF72
:10EA48004FF0010ABAF1010F2DD0BAF1030F2CD003
:10EA5800BAF1000F35D102229DF83C30DDF8409024
:10EA6800029362F34715012694F87C108DF8321052
:10EA780002220CA994F848008DF8302001F0A4F87F
:10EA880094F81A3194F830C194F81D1140B202225A
:10EA9800002B6FD0BCF1010F65D1002963D1002E86
:10EAA8006DD1104627E00422D6E70023DDF83C901C
:10EAB800BDF840709DF942B0029365F01F0501262C
:10EAC800D2E74FF0000BD946CDF808B0CCE74FF0AD
:10EAD800010084F81A04DDE005F29A420BA900F05F
:10EAE800DDFA002800F020811320049B33871F4B98
:10EAF800002283F81A241D4BD3F89434C8F8103038
:10EB08006FE705F29A452A460BA900F0C7FA0028D4
:10EB1800EAD10B9B84F82801C4F82C5184F83031D1
:10EB280002E1B9F1000F00F0FF80002A00F0FC803C
:10EB38004946E01C02F0C6FF94F8373201332380BF
:10EB4800F2E01220D1E70220CFE70720CFE701202B
:10EB580047E7064B93F8912483F840A442F001025A
:10EB680083F89124C7E7EEB90220C4E7A81C002067
:10EB7800E0160020002E94D05845B8BF584694F8A7
:10EB88007C308DF82000052294F848008DF822305A
:10EB980008A901F02CF800283FF422AF9DF8203096
:10EBA80084F83930694A6A4BD2F89804D3F890400F
:10EBB80038B105F071FA664B84423CBF002283F8F5
:10EBC8003A20198F1A8F93F830010491996A0991A4
:10EBD80052BA0028B9D093F81B0100B9186393F80A
:10EBE8001801ADF85820013893F87C2093F81A41A1
:10EBF8001491D0F1000BD3F888108DF85B204BEB03
:10EC0800000B93F8482093F83A0093F868308DF891
:10EC18005A3009AB00934F4B03904FF001008DF829
:10EC28004C0015918DF85C20A3F12F01A3F130025F
:10EC380013A88DF84D4000F0CFF8039B4FEA0B1B4B
:10EC48004BEA431B00264BEA801B4BEAC413B14531
:10EC58003E4C039308BF37463A46494604F59C7034
:10EC6800CDE90A669B46268084F81A6402F02AFFDA
:10EC7800E9B2A570C5F34215FAB2042D344E039BD0
:10EC880084F837223FF423AF072D3FF44AAF022D13
:10EC98007FF459AF304D84F80D110420029984F89F
:10ECA8000401FF2084F80C0184F8281184F8143139
:10ECB800D6F8E410C4F8085105F59B730AA8C4F8FF
:10ECC800101184F83021C4F82C3100F017FC00280A
:10ECD8007FF437AF0A9BA4F844040BA8A4F81631B4
:10ECE800C4F84C3400F0CEF900287FF4FDAE0B9B3D
:10ECF800D3B196F93900FDF7A9FA94F83732002B09
:10ED08003FF4FFAE0B9B0F2B3FF6E6AE05F58B727B
:10ED18000BA90F2000F0C2F900287FF4E5AE0B9B89
:10ED280063F3030B84F814B10598FDF74DFC002834
:10ED38007FF4DBAE099B86F83A00B36200F07EF9F7
:10ED480000283FF406AF1320D1E600BFA81C00201E
:10ED5800E016002048170020AA1C002037B50B4DEC
:10ED68008DF8040004460F2295F8480001A900F028
:10ED78003EFF40B1064A85F81C4192F8913443F0B1
:10ED8800200382F8913403B030BD00BFE0160020A4
:10ED9800A81C002010B5FFF7B9F8044688B90A483E
:10EDA80005F0B4F9094805F0B1F9094805F0AEF9DC
:10EDB80000F093F8FDF780FD064BDB6A9847204684
:10EDC80010BD0124FBE700BF1020002028200020F0
:10EDD80040200020A85A01082DE9F04F8BB0477851
:10EDE8000093149B90F90C8090F90D6090F80E90A8
:10EDF8008B464168196004469246002F57D002237B
:10EE08008DF8103004A9C37B007C8DF8123000F017
:10EE1800DBFEB4F808C0618943B26068984545468E
:10EE28006144B8BF1D46604534BF002701278842AA
:10EE380009D30A218DF81010207C019304A900F051
:10EE4800C3FE019B46B2B4F808C0608961680CEB48
:10EE5800400E714520D3A1EB0C01B1FBF0FC00FB87
:10EE68001C11C9B998450ADC237833B10223207CE8
:10EE78008DF8243006A900F0B5FE4FF001092123D2
:10EE88008DF81030207CE37B8DF8115004A98DF8A3
:10EE9800123000F099FE45B2009B8BF800503846BE
:10EEA8008AF8006083F800900BB0BDE8F08F454603
:10EEB800F2E7704770477047704700207047704707
:10EEC8007047704700207047002070470020704747
:10EED8000020704700207047704770477047022035
:10EEE8007047022070470220704770470020704723
:10EEF8007047704700207047002070477047704780
:10EF08007047000010B5054C4FF4037220460021ED
:10EF180002F0ECFD0020C4E9000010BD68220020CA
:10EF28002DE9F8438146174600293FD0244B002598
:10EF380003F1010C1A462801103312F8018FB8F1B9
:10EF4800000F36D19A42F8D11E4E33680BB9C6F875
:10EF580000C073680BB1C3F800C033180024013532
:10EF68009C6083F80C900D302B01BAB206EB0515A6
:10EF78003044F750C6F804C002F0A4FDB9F1110FEF
:10EF88004FF0000398BF104C6B71D6F8083298BF49
:10EF980024FA09F403F1010398BF04F001043B4487
:10EFA8002C71C6F808324046BDE8F8834FF00108D6
:10EFB800F9E70135202DBBD14FF00208F3E700BF78
:10EFC8006F220020682200202007020010B510B32D
:10EFD800124A1368984204D103681360002304E0BE
:10EFE8000B4613B119688842FAD15168884208BFA4
:10EFF80053600BB101681960D2F808328168013B8F
:10F0080000245B1A04602146C2F80832102202F07C
:10F018006DFD204610BD0120FCE700BF68220020DE
:10F02800054B1B6813B11A798242FAD1002B0B6089
:10F038000CBF0320002070476822002010B5054B44
:10F04800186800B910BD037B04680BB9FFF7BEFF51
:10F058002046F6E76822002038B5084B084C1868A7
:10F0680000B938BD03790568112B05D824FA03F3D4
:10F07800DB0701D5FFF7AAFF2846F1E76822002041
:10F088002007020028B1044BD3F80832036000209F
:10F0980070470120704700BF682200202DE9F04129
:10F0A80007460E4615463AB331B3144B1C68002385
:10F0B8002CB93046FFF7E6FF0020BDE8F081A268D2
:10F0C800F91A0132914210D32279EA54581C228944
:10F0D8005FFA80F8611D55FA80F002F0F3FCA3682E
:10F0E800246898445FFA88F3E2E720462468FFF72B
:10F0F8006DFF002CF9D1DCE70120DEE76822002053
:10F108000238C0B211289ABF014B185C0020704722
:10F11800BB53010830B50B4B93F820200446084632
:10F1280072B100211C330578A54208D001319842FC
:10F13800CDB20CBF04480430AA42F4D8002030BD38
:10F148001046FCE7742400208024002010B5084CE9
:10F1580000232060142204F10C00FF2184F82030E1
:10F16800C4E9010002F0C2FC012384F8213010BD7B
:10F178007424002010B50E4A92F82010042915D8DE
:10F18800936804781C7044785C70C47880789870B0
:10F198000131DC7082F8201002F11C018B4214BF8F
:10F1A800043302F10C039360012010BD0020FCE73A
:10F1B80074240020094B93F8200068B15A6803F1C1
:10F1C8001C018A4200F1FF3014BF043203F10C0223
:10F1D80083F820005A600120704700BF7424002083
:10F1E80010B5074B93F820200446084632B15968F9
:10F1F800FFF790FF10B101234470837010BD00BF6A
:10F208007424002008B5064B93F820202AB15968C9
:10F21800FFF780FF08B1407808BD0120FCE700BF78
:10F228007424002030B50A4A92F82010536882F8F6
:10F23800210061B1916801241C32DD78587005B94C
:10F248009C7093420CBF034B04339942F5D130BDF7
:10F25800742400208024002008B5044B5968FFF767
:10F2680059FF003818BF012008BD00BF74240020D2
:10F278002DE9F3410422154E044600210DEB02004E
:10F2880096F8208002F032FC0025EBB2984502D8AF
:10F2980002B0BDE8F0817368197821705A786270FD
:10F2A8009F785FB1336820469B689847FFF782FFD5
:10F2B80017B901A8FFF75EFF0135E6E7DB788DF89F
:10F2C80004108DF805208DF80730EFE7742400202E
:10F2D800014B93F82000704774240020034B93F8E7
:10F2E8002000042894BF00200120704774240020C7
:10F2F8001FB50024CDE90244C41F8DF800408DF8E5
:10F3080001100C0AADF80420090C120C8DF803103A
:10F318008DF806208DF8073002461B0A0121684641
:10F328008DF802408DF8083002F04BFA002818BF1B
:10F338000E2004B010BD2DE9F04188B017460D46E7
:10F348000F9A064600284DD000240121CDE9044437
:10F358008DF810109DF838108DF81510ADF816308E
:10F36800190CCDE900441B0ECDE902448DF8193083
:10F37800ADF81A20130C120E07948DF818108DF89A
:10F388001C308DF81D20E3B24FEA0318002D5FFAF8
:10F3980088F803DC002008B0BDE8F08101331021B3
:10F3A8008DF81F303A466B460DEB010002F09FF9CD
:10F3B8000346C8B9102DAC46A8BF4FF0100CDAB2FE
:10F3C800624503F1010303DB103D2DB20134DAE796
:10F3D80008EB020020326A44315C12F8202C4A40C3
:10F3E8003254ECE70920D6E70E20D4E70138032889
:10F3F80015D8DFE800F002080C100A4B1B681B69DF
:10F408000B6000207047074B1B685B69F8E7054BEA
:10F418001B689B69F4E7034B1B68DB69F0E7052071
:10F42800704700BF982400202DE9F041C4B00C4675
:10F438004A9E17461D468046B8B3B1F5807F36D838
:10F448004FF488720021684602F050FB492300936C
:10F458004FF48073ADF804302B0C8DF80830330C62
:10F46800ADF80650ADF80A608DF80C30224600233E
:10F47800414604A82D0E360E8DF80E308DF8095031
:10F488008DF80D608DF80F4002F01CFB04F110019F
:10F498004B9A3B4689B2684602F013F910B101282D
:10F4A80018BF0E2044B0BDE8F0810920FAE70D200E
:10F4B800F8E7000010B590B10A4C2822002120601E
:10F4C80002F014FB2368084A1A6000204FF0FF324C
:10F4D800C3E90302C3E90522C3E9072210BD0820D6
:10F4E800FCE700BF9824002000010101024B1B68C3
:10F4F80018600020704700BF9824002030B1044BEA
:10F508001B68DB68013303600020704709207047DF
:10F518009824002013B500230C460193D2B101A909
:10F52800FFF764FF18B9019B591C02D1146002B09F
:10F5380010BD99B2611A002902DD0B441360F6E789
:10F5480002D113600720F2E71B0C1B0403F580337C
:10F558002344F3E70920EAE728B1044B1B681C336E
:10F568004362002070470920704700BF982400209C
:10F5780013B50446D8B1114B1A68938801339BB26E
:10F588009380C38200F057FA98B904F118030093E6
:10F5980021680123132202F08BF860B9204600F09D
:10F5A8004AFA003818BF0120000102B010BD092036
:10F5B800FBE71020F9E70E20F7E700BF98240020AA
:10F5C800F0B5054687B01C463BB32F4E3368DB6861
:10F5D800834257D894F82020002A14BF0922082211
:10F5E800834205D3204600F05AFA70B110200AE091
:10F5F800002301900093A36894F82810606AFFF72D
:10F608009AFE0028EED007B0F0BD23792168B4F83F
:10F6180008C0A768043B9AB209B90920F3E7B2F514
:10F62800807F2DD8ADF80EC08DF817304FEA174CF3
:10F6380004F12C033F0E8DF8117000932F0C082352
:10F648004FF0490EADF80C008DF814708DF81600C7
:10F658002F0E0DEB0300CDF808E08DF810C0ADF8C3
:10F6680012508DF8157002F023F808B10E20CAE781
:10F67800204600F014FA0028B8D13368DD60C2E7EC
:10F688000D20C0E70620BEE7982400202DE9FF41A1
:10F698000A9D80460F4616461C46002D5AD0002368
:10F6A80003A910460393FFF7A1FE18B1062004B082
:10F6B800BDE8F081039B9C4201D80133F6D128466E
:10F6C80000F05EF9002847D1264B1A78424503D04E
:10F6D8001A79424542D10120AA68BA4240D103EBC7
:10F6E8008002EB6A92F801802979CDE90043043958
:10F6F800927828683B4689B2FFF796FE0028D6D153
:10F7080095F820300194002B4FF00103009314BFAB
:10F718004246082295F82810686A3B46FFF70BFE18
:10F728000028C4D1013E032EC1D8DFE806F0020745
:10F738000B0F0D4B1B681C611C62B8E70A4B1B685A
:10F748005C61F9E7084B1B689C61F5E7064B1B6891
:10F75800DC61ACE70920AAE70F20A8E70B20A6E7A1
:10F768000220A4E7A4080020982400201FB50A4618
:10F778000B2A4FF00001CDE90011CDE9021107D0A5
:10F788000C2A13D00A2A0FD00A2005B05DF804FB12
:10F79800012802D120238DF80030684602F011F8C4
:10F7A800002818BF0E20F0E73023F4E70B21F4E718
:10F7B80038B5054602F000F8044678B97DB9094B1A
:10F7C8001B680B219878FFF7D1FF38B90C21FFF798
:10F7D800CDFF18B90A21FFF7C9FF00B10E24204652
:10F7E80038BD00BF982400202DE9F04380468FB033
:10F7F8000C461746002A6BD0002969D000252946F7
:10F808001D2206A8059504F093FE8DF81350344D7B
:10F818002B680DF114099E88CDF804900DF113039F
:10F8280002933B7900933B6832462146404601F0FB
:10F83800E4FF00284ED138683A79494602F042F987
:10F84800384600F04FF8002846D13C7AFA79BB795F
:10F85800240444EA02241C432B689A6894423DD944
:10F868009C609DF813000B21FFF780FF034658BBEF
:10F878000C21FFF77BFF034630BB0A21FFF776FF19
:10F88800034608BB7B7ABA7AFF7A3F0447EA022725
:10F898001F433A46334621460920FFF729FD034610
:10F8A80090B933463A4621460820FFF721FD034622
:10F8B80050B92A689DF8131091700021D1604FF05B
:10F8C800FF31C2E90411916118460FB0BDE8F08319
:10F8D8000923F9E70E23F7E70F23F5E70323F3E7F7
:10F8E8009824002010B50446002845D00168002956
:10F8F80042D011F8013B43710322063002F0E2F8CE
:10F908002046032250F8091B043102F0DBF8216875
:10F91800CB79E3600A7A43EA0223E3604A7A43EA4E
:10F928000243E3608A7A43EA0263E360CB7A237492
:10F938000B7B63742379212B1AD110220D3104F12A
:10F94800120002F0BFF81D222168501C8B5C636214
:10F95800085C43EA0023901C6362085C033243EAB4
:10F96800004363628A5C43EA02636362002010BD5D
:10F97800112B03DC0D22E7E70220F8E70120F6E768
:10F9880010B50446002854D00168002951D00B78DE
:10F9980043714B7883608A7843EA02238360CA788C
:10F9A80043EA024383600A7943EA026383604B793E
:10F9B80003738B79C381CA7943EA0223027BC3812B
:10F9C80002F00F020831103002F07CF8237B00228D
:10F9D80003F00F0384F8202084F82820227903F10B
:10F9E8000800111A04290DDD21680933043AD21AD6
:10F9F800085C84F82000D2B2606A84F82820194490
:10FA080002F060F8237922681A44002012F8043CB6
:10FA1800E36212F8031C43EA0123E36212F8021CB2
:10FA280043EA0143E36212F8012C43EA0263E3620A
:10FA380010BD0220FCE710B5044660B3036853B359
:10FA48000279162A29D942791A700146082251F8F2
:10FA5800060B013002F040F82146082251F80E0B3F
:10FA6800093002F039F82368E28A5A74E38A226876
:10FA78001B0A93742368A269DA74A36922681B0AB3
:10FA880013752368628B5A752368E27E9A7517236B
:10FA98002371002010BD0120FCE70220FAE738B5E9
:10FAA8000446002863D00168002960D0037B90F8E1
:10FAB800282003F00F03002A57D108332079043295
:10FAC8001344984255D363790B702368A2685A701F
:10FAD800A36822681B0A937023686289DA70236816
:10FAE800E27A1A712368227B5A712368E2899A7133
:10FAF800E38922681B0A2146D371227B51F8100B37
:10FB080002F00F02083001F0DDFF237B94F8282073
:10FB180003F00F0303F108052AB1226894F82010B6
:10FB2800515503F10905206894F82820616A284492
:10FB380001F0C8FF94F828302268E16A2B44D154B8
:10FB48005A1CE16A206892B2090A81549A1C2168F9
:10FB5800E08D92B28854DA1C216894F82F0092B292
:10FB6800043388542371002038BD0933A6E70120E7
:10FB7800FAE70220F8E70000024B1A8810431880C1
:10FB8800704700BF9C24002008B5074B1B883BB179
:10FB9800FEF7BCF900280CBF00206FF0020008BD7A
:10FBA8006FF00100FBE700BF9C24002010B5034B59
:10FBB80000241C80FEF7A0F9204610BD9C240020DC
:10FBC800B0FA80F04009704782B018B9084602B010
:10FBD80000F0CAB8002002B0704710B9084600F01B
:10FBE80077B9704710B9084600F08EB970470346D8
:10FBF800084611460BB900F0E5B90020704710B966
:10FC0800084600F071BD704710B9084600F006BA02
:10FC18000020704710B40446084611461A46019B56
:10FC280014B910BC00F018BA10BC70470346084657
:10FC380011460BB900F042BA0020704710B40446D0
:10FC4800084611461A4614B910BC00F0AFBA002095
:10FC580010BC704730B40546084611461A46DDE91F
:10FC680002341DB9029430BC00F02EBB002030BC19
:10FC7800704710B9084600F0DFBB0020704710B984
:10FC8800084600F06FBD0020704710B9084600F024
:10FC9800EEBB0020704710B9084600F0EBBB00200F
:10FCA80070470346084611460BB900F005BC002012
:10FCB800704710B40446084611461A46019B14B909
:10FCC80010BC00F0FBBB092010BC704710B4044600
:10FCD800084611461A4614B910BC00F063BDC8B2F4
:10FCE80010BC70470048704701000102064B10B570
:10FCF8001B6A0446984730B10448054B2044984293
:10FD08008CBF0020012010BDA85A010840C220C99C
:10FD180080B92A00F0B5114B85B00C4610491F5622
:10FD2800054601F049F80F4BE4B25E6A072D4FF023
:10FD38000103CDE9024301460AD105220023CDE99A
:10FD480000234FF47A727A431846B04705B0F0BDE5
:10FD580008220020CDE900203A46F5E7F7530108CC
:10FD6800D0530108A85A01081FB50023009303784F
:10FD7800013B372B21D8DFE803F01C242020201E6C
:10FD8800202020204143454E2055585B5E61642069
:10FD98006C1E6E73787A20207D81262020202020FA
:10FDA800202020202020202083858A2020838A204C
:10FDB8008C90C3780BB102230093009805B05DF8CE
:10FDC80004FB8378F6E743788DF8043005238DF833
:10FDD80005308378003B18BF01235B008DF806309F
:10FDE80010238DF80730304B1B6801A803F55872B3
:10FDF800CDE9022300F0C0FF0090DEE74023DBE7F7
:10FE08002023D9E7827890F9013012B9274AD35CC8
:10FE1800D2E7274AFBE7827890F90130002AF8D127
:10FE2800244AF4E740F6B833C6E74FF47A73C3E7D9
:10FE38004FF4FA63C0E741F28833BDE741F27073CB
:10FE4800BAE71D484FF47A7101F020FE00F5FA6018
:10FE5800D2E71A4BB0E7144B1B6803F55873ABE7AE
:10FE6800114B1B6803F55B73A6E71023A4E70E4B41
:10FE78001B68A1E74FF0834300939EE7104BFBE715
:10FE8800104B99E740F21113ADF8003095E70323C2
:10FE980092E790F901300C4AB9E70C4990F9010052
:10FEA80000F08AFFA8E700BFA42400207F540108BF
:10FEB800875401088F54010818FCFFFF00EA063731
:10FEC8009A99094040F70937F7530108D0530108B8
:10FED80037B50B4B02781B680C2101FB02335B7AA8
:10FEE80003EB4304074B1D6803690093C36842781A
:10FEF800816805EBC40000F0DFFC03B030BD00BF33
:10FF0800A4240020A024002070B586B0027B6423BE
:10FF1800ADF80030012A4FF00003CDE90133CDE9F7
:10FF280003338DF802308DF8143030D0022A39D0DE
:10FF38005ABB03684BB343683BB31F4D80682B60C3
:10FF48001E4B18226946186001F0BCFD1C4B2C683A
:10FF580093E807000C3384E8070093E8070004F1EE
:10FF68000C06032386E80700A4F86C33012204F585
:10FF78005B7104F5587000F090FC2B684FF6B07276
:10FF8800A3F878230522C3F87C2306B070BD0A497C
:10FF980008684360036100F55B7100F5587000F074
:10FFA8007CFCF2E7044B1B68B3F86023B3F86C13CE
:10FFB8000A43A3F86023E8E7A4240020A024002033
:10FFC8002047010808B503460A2924D8DFE801F0CC
:10FFD80006232323230B161B23212100BDE80840F9
:10FFE8000068FFF783BE90F900009978052271B97F
:08FFF80000F013FC003818BFF3
:020000040801F1
:10000000012008BD052293F900000021F4E790F9D2
:1000100000005978EEE70221EEE70722F3E700201F
:10002000EFE7000010B504791CB1012C0BD00020C3
:1000300010BD0A4B01681B68012203F5587000F0DF
:1000400030FC0120F4E7054B01681B68224603F5EC
:100050005B7000F026FC2046EAE700BFA4240020E5
:10006000F7B50528144D1C46A8BF052058700E464C
:100070002946174600F0A4FE94F90130A070072B22
:1000800013D1322000F09CFD0C4BDB6D05469847E8
:1000900004F10C0208340346019200943A463146BA
:1000A000284600F092FD03B0F0BD054A55F8231034
:1000B000D05C00F07DFDE7E7D0530108A85A0108A5
:1000C000F75301082DE9F04F344F90F901607B6838
:1000D000D0F804908BB0044688469847054600281F
:1000E00059D1E37C73B92E4A2378126803EB43039A
:1000F000990002EB8303D3F80490B9F1000F01D10A
:1001000052F80190274B484613F906B0FB68984710
:10011000A37CD7F818A022890993072E28D10023A1
:100120000121CDE90223204A0693CDE90431CDE92E
:1001300007330521CDE900214FF47A7202FB0BF25F
:100140004CF250311846D047637C13B3174B995D7E
:100150007B6D0D31C9B228469847E07C324649464E
:1001600000F040FE88F8006001200BB0BDE8F08F81
:10017000002101250823CDE90013CDE90715CDE9BC
:100180000511CDE903110292A1782B465A46284663
:10019000D9E7074BDBE70020E7E700BFA85A0108D3
:1001A000A4240020F7530108854501008F5401085D
:1001B0007F5401082DE9F04F8DB090F90130DFF840
:1001C000FCA0DFF8FC90CDE90A123E4A12F903B018
:1001D0000278DAF800300C2505FB02333A4A5B7AE4
:1001E000126803EB430302EBC303044693F90210C6
:1001F00090F9020000F0DFFD3449064694F9010051
:1002000000F0DEFDA26861688046304600F005FD22
:100210002178DAF80020D9F80C30694307465058A5
:100220009847D9F81C309C4694F901300025072BDB
:100230004FF47A63CDE90753CDE905552DD101235C
:10024000CDE903530523CDE901534FF47A7303FB42
:100250000BF300933946434646F2A81228466746F8
:10026000B8472378DAF800200C214B4394F90110A9
:10027000D05800F0D9FDA18994F90100FFF74EFD97
:100280000B9B217B1860D9F85430284698470A9B6D
:1002900001201E700DB0BDE8F08F01200823CDE9CC
:1002A0000350CDE901032A46CDF800B06546434628
:1002B0003946A84701200546D3E700BFA424002003
:1002C000A85A0108F7530108A0240020D0530108C0
:1002D0002DE9F04F8FB0002405468A469146984696
:1002E0000494ADF81440ADF8024007264FF0010B1E
:1002F0002B7AA34206D9686804A9204400F0F2FBD7
:1003000000285ED102238DF8083002A86B7A8DF8A0
:100310000A30FFF72DFDAB7A8DF81D309DF81130B6
:100320008DF81E309DF812308DF81F309DF810307A
:100330008DF82030EB7A8DF821302B7B8DF8223030
:100340006B7B8DF8233010238DF81C608DF82430E2
:100350003A4E8DF82C000DF102030A9305238DF817
:100360002D3033680C930723ADF834302B68069397
:100370000DF1120204AB0DF1110106A800F0CCFB47
:10038000072805460BD130680C22002100F5587073
:1003900001F0B0FB3368BDF80220A3F860239DF89C
:1003A00011308AF800309DF8123089F800309DF83D
:1003B000103088F80030189B28461C700FB0BDE83C
:1003C000F08F9DF81330BDF81470ADF80270204422
:1003D000C4B2F3B917B3194A0020116807260246C0
:1003E0004FF00C0C062B1BD10CFB00FE51F80EE05D
:1003F000BEF1000F04D00BFA00F23A4397B201228B
:1004000001301028EED1002A3FF472AFADF802702F
:100410006EE75A1E042A01D9062BDCD0062667E7B0
:1004200047FA00FE1EF0010FEAD00CFB00FE51F867
:100430000EE0BEF1000F08BF0626E1E7A42400206D
:1004400038B505464068FFF755FC0522841D00219C
:1004500095F90000E4B200F0E4F908B904F0FD04F5
:1004600095F901000722002100F0DBF908B904F03A
:10047000FB04204638BD00207047000010B503780B
:100480000F2B044618D84068FFF734FC22780B493C
:1004900002EB42020968831C01EB820051F8222022
:1004A000DBB21AB903F0FD0358B210BD032B06BF2F
:1004B000626842600223F7E70020F6E7A4240020E8
:1004C000022070472DE9F04FDFF838810446D8F854
:1004D000000099B08946174600211E4601220323D9
:1004E00000F55870CDE90611CDE908118DF814100A
:1004F0008DF81510ADF8163000F0B5F938B9D8F808
:100500000020B2F8603343F00303A2F86033D8F858
:100510000020637A8DF8283002F55871CDE90B126E
:10052000394A94F9083012680D920DF116020F92B3
:100530002268109262681192D4E90301A27A8DF8C0
:10054000482001228DF8492013AA82E803001025D3
:10055000227DE18A8DF8293018468DF85420ADF8B7
:100560003850FFF7DBFB0AAB17930DF1150316901C
:1005700000933146019705AB06AA10A800F0BCFB1A
:10058000064698BB9DF81410204F013901F082FAFD
:100590001F4B1B690393C4B24FF00C0B04F16003B3
:1005A0006B44D8F8000013F848AC9DF814300BFBEE
:1005B0000AFC01343946B4FBF3F203FB1244D0F8D1
:1005C0007C33B0F9782350F80C00DDF80CC0E4B2AD
:1005D000E04728B189F800A0304619B0BDE8F08F97
:1005E000013D15F0FF05D9D10D26F5E70C2801BF17
:1005F000D8F80020B2F8603343F00303A2F8603368
:10060000EAE700BFA4240020A0240020400D03003E
:10061000A85A0108F8B50679012E054601D806202A
:10062000F8BD0F2E2BD80368187A40F3030005227B
:10063000002140B200F0F5F82B680446187A40F328
:1006400003100522002140B200F0EBF8A8B1B4FA83
:1006500084F4640929680B7A086843F3030243F3BE
:10066000031352B25BB29A42C8BF0124FFF742FBA8
:1006700048B9002CD3D10420D2E70124EAE70320B3
:10068000CEE70520CCE7002CFBD10C4F29683B6856
:1006900006EB460003EB80000C2201F017FA3A68E3
:1006A0000C2303FB062320465C72B2F8601301237F
:1006B000B3400B43A2F86033B2E700BFA42400208C
:1006C00010B4017801290ED9084B18680C234B434C
:1006D000C4180022C250C4E9012200F5587010BCB1
:1006E000102200F0A7B8002010BC7047A4240020FE
:1006F0002DE9F04186B050238DF81430037A102B89
:10070000074630D14368DD7B6DBB0224A8466426D2
:10071000062C14D87A68535D03932A44517843EA2F
:1007200001230393927843EA02437343CDE90338EC
:1007300063B968468DF80040FFF7C2FF0DE0CDF8C1
:100740000C808DF81480CDF81080F2E703AB01A87F
:1007500001938DF80840FFF75DFF0134E4B2102CDF
:1007600005F10305D4D106B0BDE8F0811FB50268DC
:100770000379116851B901A88DF80430FFF7A0FF83
:1007800078B9002040B205B05DF804FB02A80292DF
:100790008DF80C30FFF73EFF0628F2D8024B185CAC
:1007A000F0E70320EEE700BFF0530108C90020B9CD
:1007B000034B0B449856C0B27047024BF9E700BF99
:1007C000FF5301083F540108F0B59A42069D03DB30
:1007D0009DF914309A4220DD0020F0BD03EB430365
:1007E00031F814C005EB830300264CFA06F7FF0727
:1007F00007D51F7A07F00F0E724502DBB2EB171F09
:100800000DDD0136102E03F10C03EED10134E4B2FC
:100810002301DBB29842E1D8DEE70024F8E70120AB
:10082000DBE7884204DB9042CCBF00200120704708
:100830000020704710B51409B4EB111F03464FEAAE
:1008400011100ED391420CD202B201F00F0133F815
:100850001240012000FA01F124EA010123F81210EC
:1008600010BD0020FCE7F0B528B100EB41050127E1
:100870000020914200D3F0BD002435F802CB23467E
:1008800007FA04F636EA0C0608BF013304F1010446
:1008900008BFDBB2102CF3D118440131C0B2C9B289
:1008A000E7E710B500B149B910BD31F8134020F8A1
:1008B00013400133DCB2A242F7D8F5E70023F9E791
:1008C00082B030B5048804936AB9B3F5616F18D368
:1008D00049F6AF2542F21072AB4298BF4FF47A72DC
:1008E000944238BF1446012C38BF01246143BDE84F
:1008F0003040C3688B428CBF5B1A0023C36002B0D8
:1009000070476422ECE700002DE9F04F91B01546E6
:10091000DDF86C8004939DF8683009930C46064618
:1009200003F0B4FB684ADFF8A4B10590A8F5F633EC
:10093000303BB3FBF2F3534303F5F63203F5A83330
:1009400003F5C0730393182313FB0543303206925B
:10095000089300254FF0FF3A089BA34207D1002DD2
:1009600014BF50464FF0FF3011B0BDE8F08FBDF915
:100970007030ADF82C300B99CDF86C804046CDF836
:10098000288003F013FBB4F800906EB9B8F5616FDE
:100990005BD349F6AF2242F21073904598BF4FF4F3
:1009A0007A73994538BF99464B46012B38BF0123CE
:1009B0000793002E52D1B9F1640F48D1A0605F4671
:1009C000A1680EA803F014FB0F9B0093DDE90A1247
:1009D0000E9B0CA803F06BFA049B0C9A0BB9099BB5
:1009E0002BB12369BB4202D1394B9A420DD9394B05
:1009F000E760984509D90023ADF83430069B0D997E
:100A00000C93184603F0D2FAA060606800B9E76062
:100A1000276126B103F044FBE3680344E360D4E9B3
:100A200003329342059B1D996360079B88BFE26078
:100A30004B43E168994202D20498A8B9A6B10123B8
:100A40001D442375EDB2183486E76423A9E7B9F590
:100A50007A7F0ABF204F214FA060B1E7049B0BB9FA
:100A6000C4F80CB05F46D0E700209342207506D84A
:100A70005B1A9A4505F1010528BF9A46EDB2002E92
:100A8000E1D1B9F1640F164AADF8346019D049F6D6
:100A9000B023B9F57A7F18BF1346904584BF039AF7
:100AA0009B180C931C9B00930CAF97E806001B9BB4
:100AB000384603F0FCF997E8030003F077FA824622
:100AC000C1E74FF46163E8E78051010040771B0004
:100AD0007F5101002FEC010080A81201002E93022B
:100AE00030EC01000378032B14D1437803F00F029C
:100AF0001B098A704B7083788B80C27843EA02238B
:100B00008B800379C3F3021203F00F03CA700B70DA
:100B100005207047002070472DE9F3479846437938
:100B2000057990F907609146044690F906208A46B7
:100B300083B190F9087075B30F2A12D194F9092086
:100B40000F2E1ED194F90A60072D24D1002F08BF63
:100B5000012720E090F90B7090F9092090F90A60C4
:100B6000E9E7A369019394F915300093216994F999
:100B70001430207BFFF728FE0028E1D105F0FD05A9
:100B8000DEE794F91D30B3420FDC94F91C30B34218
:100B9000DADA05F0FB0528468AF8002089F80060BB
:100BA00088F8007002B0BDE8F0871E46CCE7000070
:100BB000024B03FA00F0B0FBF1F0704740420F0027
:100BC0004FF4FA53B3FBF0F0704730B54FF47A7539
:100BD0000C1F6A4300FB042252001EBF00F1FF34C9
:100BE0001219B2FBF0F2914238BF1146039A11601C
:100BF000820048431CBF013040084FF47A71121A3A
:100C000001FB1323002BCABF03F2E73393FBF1F17F
:100C1000B3FBF1F1049B196030BD38B540001446B8
:100C20000D46F0F7F7FE01462846F0F741FE214653
:100C3000F0F73EFEF0F730FD03F0CAFCF0F70CFED3
:100C400040B238BD2DE9F74F019300231F469C4663
:100C50001C01058A5FFA84FE04F0F004A54206D860
:100C6000019B82F800C01F7003B0BDE8F08F0EEB4F
:100C70004E054FEA4309AD000024466836F8096086
:100C80002641F60727D5866806EB050A765916B37E
:100C9000067836B9466926B136F809602641F60766
:100CA00019D59AF8086090F901B046F303084FFA95
:100CB00088F8D8450FDC46F3031676B25E450ADBAA
:100CC0009AF8096006EB4608C66806EBC806367D4A
:100CD0004EB90137FFB20134102C05F10C05CCD10F
:100CE0000133DBB2B4E70CF101060EEB040801F8A6
:100CF0000C805FFA86FCEEE72DE9FF47044640686A
:100D0000DDE90C671D468A46914603F0C9F9236860
:100D10001B1A3B604FF000080123337085F80080F8
:100D2000636813B12368834224D8CAF80080D4F8DA
:100D30001CC0A3699CF800E00393D4E9030101AB54
:100D400083E80300237D0093DCF80C10237A627A99
:100D50007046FFF7D9FD334638602A46E0694946B8
:100D6000FFF770FF2B782BB1C7F80080002004B08C
:100D7000BDE8F0873378002B14BF0B200C20F6E77A
:100D800037B590F9002090F90250954204460FD0F3
:100D9000013A52B295420BD0A368019394F9013005
:100DA00000936168E0782B46FFF70EFD0028EFD036
:100DB000104603B030BD8842B8BF084670470000F7
:100DC00051F82000054B984205D0054BC31A5842F4
:100DD0005841400070470120704700BF90D0030089
:100DE00020A1070005281FB50ED80C4B53F8203062
:100DF0000093CDE901120A4B01220021022002F0EA
:100E00005BFE05B05DF804FBCDE90012054B012245
:100E10000021022002F050FEF3E700BF0055010858
:100E200097540108B654010807B5054BCDE90001F8
:100E300001220021022002F03FFE03B05DF804FB16
:100E4000D254010810B5102204460021F13000F000
:100E500051FE0021C4F814112046F022BDE81040D4
:100E600000F048BE02460846102100F0A5B92DE961
:100E7000F0430446D0F8140185B00E46154604F23E
:100E8000011988B3C0F110089045474628BF17469E
:100E9000BAB2484400F01AFED4F814313B440F2B88
:100EA000C4F814312DD9A8452BD204F1F00304F570
:100EB000807113F8012F187C8B4282EA00021A70AD
:100EC000F7D104F1F10810224146684600F0FEFD1A
:100ED00022466946684600F0E9F910226946404614
:100EE00000F0F4FD3E44ED1B04F5807804F1F107B9
:100EF000102D09D8AAB23146484600F0E7FDC4F8E3
:100F0000145105B0BDE8F08304F1F003711E13F82D
:100F1000012F11F8010F434582EA00021A70F6D141
:100F200010223946684600F0D1FD224669466846DF
:100F300000F0BCF910226946384600F0C7FD1036B3
:100F4000103DD5E7F0B589B00C46102200210546CA
:100F5000684600F0CFFD22466946684600F0A6F9D3
:100F60009DF90030002B6A464FF0000143DA1378F8
:100F700012F8010F01315B0043EAD0130F2902F888
:100F8000013CF4D19DF80F305B0083F08703D4F867
:100F90001401DBB210288DF80F303BD104F58073BB
:100FA000694604F5887013F8016F11F8012B984217
:100FB00082EA06021A70F6D104F1F00304F580719A
:100FC00013F8012F187C8B4282EA00021A70F7D1C5
:100FD00010220DEB020004F1F10100F077FD224632
:100FE000294604A800F062F910220021684600F0AA
:100FF00081FD09B0F0BD137812F8010F01315B00DB
:1010000043EAD0130F2902F8013CF4D19DF80F30C8
:101010005B00BCE79DF90030002B6A464FF00001F1
:1010200037DA137812F8016F01315B0043EAD61307
:101030000F2902F8013CF4D19DF80F305B0083F0DA
:101040008703471CDBB28DF80F30102F04EB000331
:10105000C0F10F064FF0800288BF002600F58170B6
:1010600083F801210021324620443E4403F064FA13
:10107000C4F8146104F58073694604F5887013F8A8
:10108000016F11F8012B984282EA06021A70F6D11C
:1010900092E7137812F8016F01315B0043EAD6132F
:1010A0000F2902F8013CF4D19DF80F305B00C8E72E
:1010B0000A780378534003704A784378534043706A
:1010C0008A78837853408370CA78C3785340C3705A
:1010D0000A790379534003714A7943795340437144
:1010E0008A79837953408371CA79C3795340C37134
:1010F0000A7A037A534003724A7A437A534043721E
:101100008A7A837A53408372CA7AC37A5340C3720D
:101110000A7B037B534003734A7B437B53404373F7
:101120008A7B837B53408373CA7BC37B5340C373E7
:10113000704710B50B7814786340037054784B787F
:101140006340437094788B7863408370D478CB7815
:101150006340C37014790B796340037154794B7900
:101160006340437194798B7963408371D479CB79EF
:101170006340C371147A0B7A63400372547A4B7ADA
:10118000634043728B7A947A63408372D47ACB7AC9
:101190006340C372147B0B7B63400373547B4B7BB4
:1011A00063404373947B8B7B63408373CB7BD27BA5
:1011B0005340C37310BD0000A1F11003DBB2102B2C
:1011C0002DE9F04704D8374C24FA03F3DB0705D4A4
:1011D000002382F8F030FF20BDE8F087531E44184A
:1011E000A0424ED101F11C039B005FFA83F9C3F3C7
:1011F0000313013B2C4D82F8F03001240B46D61826
:10120000B3FBF1F001FB103010F0FF0016F804AC56
:1012100016F803EC16F802CC16F8017C36D115F856
:101220000E8015F80CE015F807C015F80A70E009F3
:1012300000EB400084EA080800EBC0006400C0B284
:10124000E4B24440C246581AC0B212F800808AEA9A
:10125000080A02F803A01044043390F801808EEAD3
:10126000080E86F801E090F802E08CEA0E0C86F891
:1012700002C0C078DBB247409945F770BFD8002064
:10128000AAE710F8015B03F8015FA9E71829DAD98A
:10129000102801BF15F80AA015F80EE015F80CC0CB
:1012A000EF5DD0E701010100185701082DE9F04F6B
:1012B000A3B092F8F0301D911B920193002B00F027
:1012C000538101461EA8FFF734FF1B9BA74CA84D76
:1012D000A84E10330293002303939DF87C000490E2
:1012E0009DF886000590205C06909DF87B00079095
:1012F000205C089004989DF881C0205C099014F847
:101300000C000A909DF880000B909DF885009DF8D8
:1013100078809DF87DE09DF882A09DF887900C90E4
:101320009DF87A00029B1C9314F80A2014F80930E7
:1013300014F8081014F80E700D90205C0E909DF8B3
:101340007F000F90205C10900B98205C11900C98FF
:10135000205C12909DF8840013909DF87900149001
:101360009DF87E001590205C16909DF883001790E4
:10137000205C18901398205C19901498205C1A90A7
:101380000398013003900298DDF804B01030029009
:101390009DF80C00834536D88DF878108DF87A20AA
:1013A00009990E9A8DF87C108DF882201199069A71
:1013B0008DF880108DF87E201999169A8DF884107A
:1013C0008DF886200A99189A8DF87D108DF887205F
:1013D0001299109A8DF87B301B9B8DF881108DF837
:1013E00083201A99089A1D988DF885108DF87F2012
:1013F0001EA903EB0B128DF87970FFF79AFE0020FF
:1014000023B0BDE8F08F15F808B082EA03008BEA3C
:10141000000016F80EB080EA0B008DF8780015F881
:101420000E004B40434016F80A0043408DF87930D7
:1014300081EA070315F80A10594016F80930594097
:1014400016F808308DF87A107A40534015F80920C4
:1014500053408DF87B30089A069B5340049AAA5C4F
:10146000534016F80C2053408DF87C30DDE90832EB
:101470005A4015F80C305340059AB25C53408DF831
:101480007D30DDE909325A40059BEB5C5340079AF9
:10149000B25C53408DF87E30069B0A9A5340049A02
:1014A000B25C5A40079BEB5C5A408DF87F200E9B44
:1014B000109A53400B9AAA5C53400C9AB25C53406A
:1014C0008DF88030DDE910325A400C9BEB5C5340C4
:1014D0000D9AB25C53408DF88130DDE911325A40EB
:1014E0000D9BEB5C53400F9AB25C53408DF88230F9
:1014F000129A0E9B53400B9AB25C5A400F9BEB5CC6
:101500001C995A408DF88320169B189A5340139AC1
:10151000AA5C5340149AB25C53408DF88430DDE9E4
:1015200018325A40149BEB5C5340159AB25C5340FE
:101530008DF88530DDE919325A40159BEB5C53403C
:10154000179AB25C53408DF886301A9A169B534016
:10155000139AB25C5340179AAA5C1EA853408DF8A8
:101560008730FFF7A5FDB8E6FF2049E718570108C7
:10157000185501081856010808B538B1044A05493C
:101580001060D82200F0A2FA002008BD0220FCE77B
:10159000A8240020485C01080A4B1A6870B5002393
:1015A00002F1180503EB03142E5D864204D11834B2
:1015B00022440A60002070BD01330B2BF2D10320BE
:1015C000F9E700BFA82400202DE9F041CCB0064681
:1015D000DDF8488117461C460D4631B3B8F1000FBF
:1015E00023D006A8FFF72EFC204601A9FFF7D4FF61
:1015F0000446B0B9019906A80131FFF733FC26B1C2
:101600001022314606A8FFF732FC3A46294606A8C2
:10161000FFF72DFC06A902A8FFF794FC029BC8F86F
:10162000003020464CB0BDE8F0810224F9E700000C
:1016300030B595B013A90446FFF7AEFF002830D1AE
:101640001B490C2303FB00F2555CA5422BD1139BD5
:10165000187C1090D87B0F90987B0E90587B0D9043
:10166000187B0C90D87A0B90987A0A90587A099047
:10167000187A0890D879079098790690587905904B
:1016800018790490D8780390987802900A445B788F
:101690000193936800930022064B1146022002F04A
:1016A0000BFA15B030BD01300B28CBD1F9E700BFE4
:1016B00090590108185801080B2B10B402D810BC1F
:1016C000FFF782BF032010BC704730B50D4685B0D0
:1016D0001446014668B103AA002000922A460390EE
:1016E000FFF772FF18B90398001B18BF012005B05F
:1016F00030BD0220FBE72DE9F0430D46BFB0144694
:101700009946804620B31BB311F00F0122D1F0227D
:1017100001A800F0EFF920466946FFF73DFF0446B7
:1017200048B9009801AA10210130FFF745FD2E4667
:10173000AF1BFFB21EB920463FB0BDE8F08301AA3F
:1017400009EB070108EB0700FFF7B0FD103EEFE7DC
:101750000224F0E70524EEE7F0B5184E346802469F
:1017600085B00846002304F1180103EB03154F5D13
:1017700097421ED10D2A05F1190513D10023CDE999
:101780000033CDE902330C2210216B46FFF7B3FF83
:101790000446306810226946284400F097F9204634
:1017A00005B0F0BD01461022601900F08FF9002449
:1017B000F5E701330B2BD8D10324F0E7A824002050
:1017C00009B1FFF7C9BF022070471FB51446A0B189
:1017D0000C2A01D10B2912D10023CDE90033CDE928
:1017E00002330A466B461021FFF785FF18B9694698
:1017F0002046FFF7B1FF04B010BD0220FBE7032035
:10180000F9E7F8B51E46DDE907479DF818505BB3C8
:1018100054B34FB3212D29D819462A46204600F04B
:1018200055F90122631C691EB018FFF764FFF8B96F
:10183000E37ADB093B70EBB96319204613F8012CFE
:1018400013F8021C120642EA014213F8041C0A4370
:1018500013F8031C012342EA0122291FFFF735FF79
:10186000003818BF0120F8BD0220FCE70520FAE788
:101870000720F8E70420F6E708B5014630B1044B2D
:101880000822186800F022F9002008BD0220FCE7B9
:10189000A824002008B530B1044B0822196800F0D4
:1018A00015F9002008BD0220FCE700BFA824002095
:1018B0007FB5124E0023044602A801930D46FFF7A0
:1018C000E9FF33685B6901936CB102AA082312F83F
:1018D000011B41B9013B13F0FF03F8D102A8A04757
:1018E00002A8FFF7C9FF35B1019B23B901A8A8479A
:1018F0003368019A5A61002004B070BDA82400200A
:1019000008B5014638B1054B18680822104400F0AC
:10191000DDF8002008BD0220FCE700BFA82400205D
:1019200008B538B1044B19680822114400F0CEF80C
:10193000002008BD0220FCE7A8240020034B1B6800
:1019400002280CBF1961596100207047A8240020AB
:1019500041B1054B1B6802280CBF1B695B690B601A
:101960000020704702207047A824002030B58FB0B7
:10197000002405460CA80994FFF78CFF9DF837302A
:1019800007939DF8363006939DF8353005939DF802
:10199000343004939DF8333003939DF83230029332
:1019A0009DF8313001939DF8303000932246214656
:1019B0001E4B022002F080F80AA8FFF7B1FF9DF845
:1019C0002F3007939DF82E3006939DF82D30059308
:1019D0009DF82C3004939DF82B3003939DF82A300A
:1019E00002939DF8293001939DF8283000932246F8
:1019F0000F4B2146022002F05FF809A92846FFF7A5
:101A0000A7FF9DF8243003939DF8253002939DF89D
:101A1000263001939DF8273000932246054B21463E
:101A2000022002F049F80FB030BD00BF7458010821
:101A3000B2580108F058010808B50020FFF7F8FD7A
:101A40000120FFF7F5FD0920FFF7F2FD0820FFF761
:101A5000EFFD0020FFF78AFF002008BD10B5044607
:101A60000B20FFF7E5FD0C20FFF7E2FD0920FFF753
:101A7000DFFD0820FFF7DCFD0A20FFF7D9FD204637
:101A8000FFF774FF002010BD014B1860704700BFC6
:101A9000AC0800200B4A30B514680B4D43F23903F3
:101AA00005FB04331360091A6FF00042B3FBF2F236
:101AB000C2EBC27201319B1A93FBF1F201FB1233AC
:101AC000184430BDAC0800206D4EC64101380A44B0
:101AD000914200D1704711F8013B00F8013FF7E750
:101AE00010440A44914200D1704711F8013B00F8BC
:101AF000013DF7E702F020BD30B530B10A4D014499
:101B00004FF0FF33814201D1D84330BD10F8012B93
:101B10005340082243F30004013A2C4092B284EA75
:101B20005303002AF6D1EDE72083B8ED012070477A
:101B3000054B4FF400529A62044B1B6813B15B686B
:101B400003B11847704700BF00040048AC250020CF
:101B5000054B4FF480529A62044B1B6813B1DB684B
:101B600003B11847704700BF00040048AC250020AF
:101B7000012070470120704701F048B901F036B9E3
:101B800010B501F019FE0E21044640F61F1001F0B9
:101B90002DF92046012101F0F9FDBDE8104001F0CA
:101BA000D7BA000070B50C4E01EB40030D46B3658B
:101BB0004FF6FF71002304461A46084601F05EFB0B
:101BC00096F85600002101F0E1FD29462046BDE8C7
:101BD000704001F095BA00BFC825002010B504463A
:101BE00001F0AAFE01281CD101F0AEFE34B112486A
:101BF000214602F017FB104802F0DAFA0F4C104BA6
